:020000040800F2
:10000000000001107108040875040308D1D9000824
:100010007509040875090408750904080000000042
:10002000000000000000000000000000BD0A0308FE
:10003000B90A030800000000B50A030859F00008D7
:100040007509040875090408750904087509040888
:100050007509040875090408D99D0008059F000862
:10006000C99E00088D9E0008519E00089DBA000898
:100070008DBA00087DBA00086DBA00085DBA0008A4
:1000800049BA000835BA000875090408750904085A
:10009000750904087509040875090408159E000807
:1000A000D9E0000839E10008C9E0000861E1000872
:1000B00029E1000819E1000809E1000889C40008E5
:1000C00091C400087DC4000885C4000875090408AF
:1000D000750904082193000885920008E991000839
:1000E0009D9D000875090408CD15030875090408CD
:1000F000E9E0000875090408F9E0000821BA0008E1
:1001000075090408750904087509040875090408C7
:1001100081F10008E5F000089DE2010881E2010894
:100120000DBA0008F9B90008E5B90008D1B900080E
:10013000BDB90008750904087509040875090408A3
:100140007509040875090408750904087904030889
:10015000A9B9000895B9000881B900087509040813
:1001600071C4000879C400087509040875090408F9
:100170007509040875090408750904087509040857
:08018000750904087509040863
:0801880008040400010000005E
:1001900002020300802600207C26002000000000D0
:1001A00000000000160008008C2600209426002085
:1001B000000000004006000803000100182C002089
:1001C000202C002000000000000000001D000100A5
:1001D000302C0020C02C0020000000004806000841
:1001E00027000400502C0020C42C00200000000038
:1001F0004A0600080A020A00282E0020382E002095
:10020000000000004E06000801010400802F0020BD
:100210006446002000000000000000000802090001
:10022000AE45002068460020000000001F82000844
:1002300006020C0024460020744600200000000046
:1002400019900008070202004C460020804600205A
:100250000000000058060008FF0101006146002070
:1002600084460020000000005A06000802000C002E
:1002700034460020884600200000000000000000F6
:10028000F7010600A8450020944600200000000069
:100290005C0600082C001000C44B0020B44B00206A
:1002A00000000000A11E02082B002400F84B0020D3
:1002B000D44B002000000000711E020829005000ED
:1002C000005000203C510020000000000000000011
:1002D00014000200FC4F00208C51002000000000A0
:1002E0006206000810000300704F002090510020AB
:1002F000000000006406000828000C00644F002085
:10030000945100200000000068060008230010003F
:10031000544F0020A0510020000000006D1502087D
:10032000190005004C4F0020B051002000000000D3
:1003300074060008F8110100484F0020B851002051
:10034000000000007A06000800010400444F00206D
:10035000BC510020000000007C06000800020500DF
:10036000C0510020A857002000000000000000003D
:100370001E000400FC520020B057002000000000C6
:100380008006000822000C007C520020B457002098
:100390000000000084060008090201001458002033
:1003A0001C65002000000000900600080C002400DE
:1003B000F66400202065002000000000B9E201087A
:1003C0001B00F4004C650020D866002000000000EF
:1003D000595A020812100C00CC660020CC6700208D
:1003E00000000000920600082F001100B0660020F7
:1003F000D8670020000000009E06000803123300AA
:100400005F6900202C69002000000000B006000891
:1004100025005A0078680020D26800200000000003
:1004200000000000F6110C006C68002060680020DD
:1004300000000000E4060008012008006C6A0020AB
:10044000B86A002000000000F00600081A0008004A
:10045000506A0020C06A002000000000F806000872
:100460000E20EA004A6B0020D86C0020000000003B
:1004700055B0020813000400786C0020C46D002001
:10048000000000000007000802010300356B002097
:10049000C86D002000000000E1E201081F000E000E
:1004A000106F00204C6F00200000000004070008BF
:1004B00005020100F86E00205C6F002000000000C3
:1004C00012070008030106008A6E0020606F0020FA
:1004D00000000000140700080A1012004C960020CB
:1004E00074960020000000001A070008060016009D
:1004F0001C930020889600200000000075B00208C0
:10050000340010008C910020A09600200000000014
:10051000C1A103080D00340058910020B0960020BE
:1005200000000000817A030811000C00EC85002017
:10053000E496002000000000CD790308FD011E00B4
:10054000D47F0020F096002000000000A181000868
:10055000FE010800C07F002010970020000000006E
:100560008DC5000804008000D4B3002088B50020A9
:100570000000000000000000F9010400C098002005
:1005800008B60020000000001182000818102C009E
:10059000909800200CB6002000000000C52A020838
:1005A000FB0101005898002038B600200000000030
:1005B00085C50008FC010900249700203CB60020F6
:1005C0000000000051C50008050006008CB700209F
:1005D00004B90020000000002C070008F51162009B
:1005E00024B700200CB9002000000000858E02080E
:1005F00026000E0080B9002070B900200000000025
:10060000818F03082A006000F4C0002094C00020FD
:100610000000000099A1030815007000CCBA00206A
:1006200054C1002000000000000000000B2010005A
:1006300004C400203CC40020000000003207000871
:10064000C409000019012828000020030000000050
:100650004A01B400D6010000013C00003F01000047
:100660000000030000010500000000010000000080
:1006700000000000000028010000040090010000BC
:1006800000000100C800141E010064002C012800B5
:100690001300000000010005535034450000000025
:1006A000000000000000000000000000000000004A
:1006B000000000000000000000000000000000003A
:1006C000000000000000000000000000000000002A
:1006D000000000000000000000000000000000001A
:1006E0000000010000000000000000000000000009
:1006F000E8036400040A00017E05EA05B40532003F
:100700000884250000000000000001000000000532
:100710000000000004010100000000300100005A48
:100720000000000090012C01C800640020000200BD
:1007300001002B21231E64010200000001000A01B8
:0207400029008E
:100742005001000007000000020000000000803F8E
:100752000000803F0000803F000000000000000019
:10076200010203040607080901010000506704089A
:10077200F889040800000000000000006067040817
:100782006867040800000000012000006C6704088C
:100792007467040800000000014000007867040844
:1007A200B07B0408000000000120000084670408F8
:1007B2009067040800000000040000009467040829
:1007C200B4A604080000000004000000A0670408AA
:1007D200E099040800000000010000000201FF008F
:1007E2000000803F0000803FC8380408050804006C
:1007F20000000000605A04083C5A0408B438040897
:1008020000000000F438040805080A000000000097
:10081200605A04083C5A0408BC580408000000004E
:10082200FFFFFFFF01010000ED1A020800000000B7
:100832000000000000010101303030302D30312D38
:1008420030315430303A30303A303000010000005C
:100852000000803F00000101FFFF00000000803F18
:10086200006002401060024000000000000B000027
:1008720000002000000000000000000000600240B4
:100882002860024000000000060C0000000020006A
:1008920000000000000000000060024040600240D2
:1008A20000000000100D0000000020000000000009
:1008B200000000000060024058600240000000009A
:1008C200160E0000000020000000000000000000E2
:1008D200006002407060024000000000200F000033
:1008E2000000200000000000000000000060024044
:1008F2008860024000000000261000000000200076
:10090200000000000000000000600240A060024001
:100912000000000030110000000020000000000074
:100922000000000000600240B860024000000000C9
:10093200362F000000002000000000000000000030
:100942000064024010640240000000000038000011
:1009520000004000000000000000000000640240AF
:100962002864024000000000063900000000400038
:1009720000000000000000000064024040640240E9
:1009820000000000103A00000000400000000000DB
:1009920000000000006402405864024000000000B1
:1009A200163B0000000040000000000000000000B4
:1009B200006402407064024000000000203C00001D
:1009C200000040000000000000000000006402403F
:1009D200886402400000000026440000000040003D
:1009E200000000000000000000640240A064024019
:1009F2000000000030450000000040000000000040
:100A02000000000000640240B864024000000000E0
:100A12003646000000004000000000000000000018
:100A220001010100D0A304080F000000D9D202087E
:100A3200000000000000000064040020A4A30408D9
:100A420000000000000000000000000000000000A4
:100A5200F8890408000000000000000018050020CA
:100A620004000000F89A04080D000000EDD9020805
:100A7200D01D002000000000209D04080D00000091
:100A8200BDD90208C41D002000000000109E040809
:100A92000800000000000000B81D00200400000053
:100AA2008C9D04080D000000D5D80208AC1D002062
:100AB20000000000209E040803000000DDDE0308A1
:100AC200941D002000000000B4A3040803000000ED
:100AD200DDDE03087C1D002000000000AC9A040843
:100AE2000100000000000000000000000000000003
:100AF200000000000E0000000000000000000000E6
:100B020000000000A4A30408000000000000000090
:100B12000000000000000000F88904080000000046
:100B22000000000018050020040000001CA30408B7
:100B32000300000079D80208641D002008000000AC
:100B42008C9D04080D000000D5D80208AC1D0020C1
:100B520000000000209E040803000000DDDE030800
:100B6200941D002000000000B4A30408030000004C
:100B7200DDDE03087C1D002000000000AC9A0408A2
:100B82000100000000000000000000000000000062
:100B9200000000000E000000000000000000000045
:100BA20000000000BCA304080000000000000000D8
:100BB2000000000000000000F889040800000000A6
:100BC20000000000180500200400000024A304080F
:100BD20003000000DDDE0308DC1D00200000000031
:100BE200AC9A0408010000000000000000000000B0
:100BF20000000000000000000E00000000000000E5
:100C0200000000000000000020700020702D720023
:100C120098A304080F00000000000000000000007C
:100C22000000000014190020FFFFFFFFFA0000007F
:100C320001000000010000002D202D2D202D2D2D62
:100C42002D202D2D2D2D00000000000000000000A1
:100C520000000000000000002D202D2D202D2D2D44
:100C62002D202D2D2D0000000000000000000000AE
:100C72000000000000000000949A04089C9A0408F6
:100C8200A49A040800000000000000000000000018
:100C920000000000659A04080400000009D8020858
:100CA2000000000000000000AC9A040801000000EF
:100CB2000000000000000000000000000000000032
:100CC2000E00000000000000000000000000000014
:100CD2003EB500200100C409000000003CB5002020
:100CE2000100C409000000003AB500200100C40957
:100CF2000000000038B500200100C4090000000017
:100D020034B500200100C4090000000036B50020FF
:100D12000100C4090000000032B500200100C4092E
:100D22000000000030B500200100C40900000000EE
:100D3200E66A00200100C80001000000E46A002009
:100D42003200307532000000E36A0020055A0500C7
:100D5200DE6A002000FF0100E26A002001000000BC
:100D620038050020E06A002002000000E462040866
:100D7200DD6A002000FF0100E16A0020010000009E
:100D820038050020DF6A002002000000E462040847
:100D92000C9B04080F00000000000000000000008F
:100DA2000000000040050020C86E00209CFF2C01BE
:100DB20000000000E20200200A000000BC58040803
:100DC200C86A0020E0150C1700000000E1020020B4
:100DD200080000003C5A0408E00200200500000060
:100DE200605A0408CA6A002002000000D4580408AD
:100DF200DC6A002001000000345A0408DB6A00208B
:100E020001080100DA6A002004000000E05804082A
:100E1200666C00200100FF7F01000000646C00206E
:100E220002000000F45804083E6B0020030000009A
:100E3200045904083D6B0020030000000459040813
:100E42003C6C00200000F401010000003A6C00201C
:100E52000000F40101000000386C00200000F401E1
:100E620001000000366C00200000F40101000000C7
:100E7200346C002000FF0100506C0020E803D00712
:100E82000A0000004E6C0020006401000A0000000D
:100E92004F6C0020006401000A000000486C002032
:100EA200006401000A0000004D6C00200064010093
:100EB2000A0000004C6C0020006401000A000000DF
:100EC2004B6C0020006401000A000000476C002007
:100ED20000FF01000A000000466C002000FF010034
:100EE2000A000000466B00200000F401010000002F
:100EF200446B00200000F40101000000426B00205E
:100F02000000F40101000000406B00200000F40129
:100F120001000000436C002000C80100426C002068
:100F220000C80100416C002000C80100406C002094
:100F3200006401000A0000003F6C002000FF010075
:100F42000A0000005B6C002000C801005A6C0020FF
:100F520000C80100596C002000C80100586C002034
:100F620000C80100576C002000C80100566C002028
:100F720000C80100556C002000C80100546C00201C
:100F820000C80100536C002000C80100149B040833
:100F9200000000000000000000000000000000004F
:100FA200249B04080900000000000000E405002062
:100FB200040000002C9B040809000000000000004F
:100FC200D805002004000000F0A004080900000079
:100FD20000000000CC05002004000000CC8A0408B8
:100FE2000900000000000000C0050020040000000D
:100FF200349B04080900000000000000B405002032
:10100200040000003C9B04080900000000000000EE
:10101200A805002004000000449B04080900000009
:10102200000000009C050020040000004C9B040806
:1010320009000000000000009005002004000000EC
:10104200AC9A04080100000000000000000000004B
:1010520000000000000000000E0000000000000080
:101062000000000000000000249C040800000000B2
:1010720000000000000000000000000034A6040888
:101082000700000000000000080600200000000029
:10109200349C04080800000000000000FC05002049
:1010A20000000000409C040808000000000000004E
:1010B200F005002000000000AC9A040801000000C6
:1010C200000000000000000000000000000000001E
:1010D2000E00000000000000000000000000000000
:1010E200489C04080000000000000000000000000E
:1010F20000000000589C04080D00000000000000E1
:101102004406002000000000609C04080D0000005E
:10111200000000003806002000000000689C04085F
:101122000700000000000000300600200000000060
:10113200709C04080D00000000000000240600203E
:1011420000000000789C04080D0000000000000070
:101152001806002000000000809C04080700000020
:10116200000000001006002000000000AC9A0408F5
:10117200010000000000000000000000000000006C
:10118200000000000E00000000000000000000004F
:1011920000000000889C040800000000000000001D
:1011A200000000000000000034A604080C0000004B
:1011B20000000000E86A0020000000009C9C040877
:1011C2000C00000000000000EA6A0020000000009D
:1011D200AC9C04080C00000000000000206B002002
:1011E20000000000BC9C04080C000000000000008D
:1011F200146B002000000000D09C04080C000000CA
:1012020000000000EC6A002000000000DC9C0408E2
:101212000C00000000000000EE6A00200000000048
:10122200E49C04080C00000000000000F06A0020AA
:1012320000000000F89C04080C0000000000000000
:10124200F26A002000000000009D04080C0000006B
:1012520000000000F46A002000000000089D04085D
:101262000C00000000000000F66A002000000000F0
:10127200149D04080C00000000000000F86A002021
:10128200000000002C8C04080C000000000000008C
:10129200FA6A0020000000001C9D04080C000000F7
:1012A20000000000FC6A002000000000289D0408E5
:1012B2000C00000000000000FE6A00200000000098
:1012C200349D04080C00000000000000006B0020A8
:1012D20000000000409D04080C0000000000000017
:1012E200026B0020000000004C9D04080C0000006E
:1012F20000000000046B002000000000589D04085C
:101302000C00000000000000186B0020000000002C
:10131200609D04080C00000000000000166B002015
:1013220000000000689D04080C000000000000009E
:10133200246B002000000000749D04080C000000D3
:1013420000000000266B002000000000809D0408C1
:101352000C000000000000002C6B002000000000C8
:1013620058A604080C00000000000000066B0020D4
:10137200000000008C9D04080C000000000000002A
:101382000E6B002000000000949D04080C00000079
:1013920000000000086B002000000000A09D04086F
:1013A2000C000000000000000A6B0020000000009A
:1013B200AC9D04080C000000000000000C6B002033
:1013C20000000000B49D04080C00000000000000B2
:1013D200106B002000000000EC8804080C000000E4
:1013E200000000001A6B002000000000C09D0408ED
:1013F2000C00000000000000126B00200000000042
:10140200DC8B04080C00000000000000226B0020AE
:1014120000000000CC9D04080C0000000000000049
:101422001C6B002000000000D49D04080C0000008A
:10143200000000001E6B002000000000DC9D04087C
:101442000C00000000000000286B002000000000DB
:10145200E49D04080C000000000000002A6B00203C
:1014620000000000AC9A0408010000000000000027
:101472000000000000000000000000000E0000005C
:10148200000000000000000000000000EC9D0408C5
:10149200000000000000000000000000000000004A
:1014A200FC9D040805000000000000003C6B0020C9
:1014B20000000000AC9A04080100000000000000D7
:1014C2000000000000000000000000000E0000000C
:1014D200000000000000000000000000049E04085C
:1014E20000000000000000000000000000000000FA
:1014F200F88904080000000000000000F804002041
:1015020004000000C88A04080D00000051D8020837
:10151200A406002000000000F89A04080D00000054
:1015220085D202089806002000000000209D0408D1
:101532000D00000051D202088C06002000000000BD
:10154200109E040808000000000000008006002031
:10155200040000008C9D04080D0000003DD202082A
:101562007406002000000000189E04080900000014
:10157200000000006806002004000000209E04080D
:1015820003000000DDDE030850060020000000001A
:10159200AC9A0408010000000000000000000000F6
:1015A20000000000000000000E000000000000002B
:1015B2000000000000000000249E0408000000005B
:1015C200000000000000000000000000F89A04087B
:1015D2000D00000000000000C40600200000000012
:1015E200309E04080700000000000000BC06002036
:1015F200000000008C9D04080D00000000000000A7
:10160200B006002000000000AC9A040801000000AF
:1016120000000000000000000000000000000000C8
:101622000E000000000000000000000000000000AA
:10163200389E0408000000000000000000000000C6
:1016420000000000489E04080D0000000000000099
:10165200DC06002000000000509E04080A00000082
:10166200000000007C6C0020000000005C9E04086A
:101672000A00000000000000846C0020000000004E
:10168200649E04080A000000000000008C6C002028
:10169200000000006C9E040808000000000000002A
:1016A200D006002000000000AC9A040801000000EF
:1016B2000000000000000000000000000000000028
:1016C2000E0000000000000000000000000000000A
:1016D200749E0408000000000000000000000000EA
:1016E20000000000889E04080D00000000000000B9
:1016F200F406002000000000989E04080400000088
:1017020059DB02080000000000000000A09E04084F
:101712000D00000000000000E806002000000000AC
:10172200B49E04080400000035DB0208000000003B
:1017320000000000AC9A0408010000000000000054
:101742000000000000000000000000000E00000089
:10175200000000000000000000000000BC9E040821
:101762000000000000000000000000000000000077
:10177200D09E04080700000000000000300700208F
:1017820000000000DC9E04080800000000000000C9
:101792002407002000000000E89E04080800000062
:1017A200000000001807002000000000F49E04085A
:1017B20008000000000000000C07002000000000EC
:1017C200009F04080800000000000000000700203D
:1017D20000000000AC9A04080100000000000000B4
:1017E2000000000000000000000000000E000000E9
:1017F2000000000000000000000000000C9F040830
:101802000000000000000000CB04002000000000E7
:10181200189F04080B000000000000009807002039
:1018220000000000209F04080B00000000000000E0
:101832008C070020000000002C9F04080B00000011
:10184200000000008007002000000000389F04080C
:101852000B000000000000007407002000000000E0
:10186200449F04080B0000000000000068070020ED
:1018720000000000509F04080B0000000000000060
:101882005C07002000000000589F04080B000000C5
:10189200000000005007002000000000649F0408C0
:1018A2000B000000000000004407002000000000C0
:1018B200709F0408080000000000000038070020A4
:1018C20000000000AC9A04080100000000000000C3
:1018D2000000000000000000000000000E000000F8
:1018E2000000000000000000000000007C9F0408CF
:1018F20000000000000000000000000000000000E6
:10190200909F04080800000000000000C8070020A3
:10191200000000009C9F0408080000000000000076
:10192200BC07002000000000A89F04080800000077
:1019320000000000B007002000000000B49F04086F
:101942000800000000000000A407002000000000C2
:10195200AC9A040801000000000000000000000032
:1019620000000000000000000E0000000000000067
:101972000000000000000000BC9F040800000000FE
:1019820000000000C804002000000000CC9F0408F2
:101992000B00000000000000F8070020000000001B
:1019A200D89F04080B00000000000000EC07002094
:1019B20000000000E49F040807000000000000008F
:1019C200E407002000000000F09F04080700000068
:1019D20000000000DC07002000000000FC9F04085B
:1019E2000700000000000000D407002000000000F3
:1019F200AC9A040801000000000000000000000092
:101A020000000000000000000E00000000000000C6
:101A1200000000000000000008A004080000000010
:101A220000000000C80400200000000014A0040808
:101A32000700000000000000440800200000000031
:101A42001CA0040807000000000000003C08002061
:101A52000000000024A004080700000000000000AD
:101A620034080020000000002CA004080700000039
:101A7200000000002C0800200000000034A0040830
:101A82000700000000000000240800200000000001
:101A92003CA0040807000000000000001C08002011
:101AA2000000000044A0040807000000000000003D
:101AB20014080020000000004CA0040807000000E9
:101AC200000000000C0800200000000054A00408E0
:101AD20007000000000000000408002000000000D1
:101AE200AC9A0408010000000000000000000000A1
:101AF20000000000000000000E00000000000000D6
:101B020000000000000000005CA004080F000000BC
:101B12000000000045D50208000000004C0800202B
:101B22003A6B00201700000014590408396B00209A
:101B32000A320100386B002001FA0100346B0020E8
:101B420000C80100326B0020E803D007010000004A
:101B52005350524143494E47463445564F000000C8
:101B620064A004080F00000069D4020845D40208EA
:101B7200000000002809002070A004080F000000E7
:101B82000DD40208CDD3020800000000A0090020F5
:101B92007CA004080F000000A5D402088DD402081E
:101BA20000000000540A002088A004080F00000072
:101BB2005BD502080000000005DB02084C0D002086
:101BC20090A004080F0000009DD102080000000050
:101BD200000000009C0D002098A004080F000000E7
:101BE200A1D3020895DA020800000000780E002056
:101BF200A0A004080F0000004DDC0208B5D70208BF
:101C0200C5D30208F00E0020A8A004080F000000AF
:101C120081D502080000000000000000900F0020A3
:101C2200B0A004080F00000025D60208F5D502086E
:101C3200000000001C100020B8A004080F000000E3
:101C4200A1D60208E9D6020800000000BC1000205C
:101C5200446C002001030100C4A004080F0000002E
:101C6200C1D5020895D5020800000000AC11002081
:101C7200CCA004080F00000055D602087DDB020844
:101C82000000000038120020D8A004080F00000055
:101C920019D70208C9DB020800000000D812002090
:101CA2003E6C002001030100E0A0040800000000D7
:101CB200000000000000000000000000ECA004088A
:101CC20008000000000000000414002000000000D2
:101CD200F4A004080700000000000000FC1300202C
:101CE2000000000004A1040807000000000000003A
:101CF200F41300200000000010A1040807000000F7
:101D020000000000EC130020000000001CA10408E9
:101D12000D00000000000000E013002000000000A1
:101D220028A1040803000000DDDE0308C813002018
:101D320000000000AC9A040801000000000000004E
:101D42000000000000000000000000000E00000083
:101D520000000000000000000000000030A10408A4
:101D62000000000000000000000000000000000071
:101D720040A104080A00000000000000AC6704084B
:101D82000000000048A104080A0000000000000052
:101D9200306704080000000050A104080A00000097
:101DA200000000005C6C00200000000058A1040844
:101DB2000A000000000000001014002000000000D3
:101DC200AC9A0408010000000000000000000000BE
:101DD20000000000000000000E00000000000000F3
:101DE200000000000000000060A1040800000000E4
:101DF2000000000000000000000000006CA10408C8
:101E020003000000DDDE0308501400200000000083
:101E120074A0040803000000DDDE0308381400206B
:101E22000000000068A0040803000000DDDE0308D3
:101E32002014002000000000AC9A040801000000F9
:101E42000000000000000000000000000000000090
:101E52000E00000000000000000000000000000072
:101E620078A104080000000000000000000000004B
:101E7200000000008CA1040803000000DDDE03085E
:101E8200B0140020000000009CA004080300000021
:101E9200DDDE0308981400200000000098A1040869
:101EA20003000000DDDE0308E40200200000000061
:101EB200A0A1040803000000DDDE03088014002056
:101EC20000000000A8A1040803000000DDDE0308F2
:101ED2006814002000000000AC9A04080100000011
:101EE20000000000000000000000000000000000F0
:101EF2000E000000000000000000000000000000D2
:101F0200B4A104080000000000000000000000006E
:101F120000000000C0A104080700000015DC020850
:101F22006015002000000000B09D040803000000BE
:101F3200DDDE03084815002000000000CCA10408E3
:101F420003000000DDDE0308301500200000000061
:101F5200D4A1040803000000DDDE030818150020E8
:101F620000000000DCA1040807000000F9DB020801
:101F7200101500200000000040A304080300000028
:101F8200DDDE0308F814002000000000E8A10408C8
:101F920003000000DDDE0308E01400200000000062
:101FA200F4A1040803000000DDDE0308C8140020C9
:101FB20000000000AC9A04080100000000000000CC
:101FC2000000000000000000000000000E00000001
:101FD20000000000000000000000000000A2040851
:101FE2000F00000001D50208BDD402080000000065
:101FF2006815002008A204080F00000089D7020813
:1020020000000000000000001C16002014A20408BA
:102012000F000000C9D30208C1D30208000000006B
:10202200A81600201CA204080F00000000000000F7
:102032000000000000000000201700202CA204086D
:102042000F00000061D7020831DC02080000000026
:10205200C017002034A204080000000000000000A5
:102062000000000000000000D48804080300000003
:10207200DDDE0308FC1800200000000020A2040896
:1020820003000000DDDE0308E41800200000000069
:1020920018A2040803000000DDDE0308CC180020AB
:1020A2000000000040A2040803000000DDDE030877
:1020B200B4180020000000004CA204080300000035
:1020C200DDDE03089C1800200000000054A2040872
:1020D2000200000039DD02080000000000000000DC
:1020E2005CA204080200000039DD020801000000C1
:1020F2000000000068A204080200000039DD0208A6
:102102000200000000000000000000000E000000BD
:10211200000000000000000000000000D66A00205D
:1021220088130C1701000000D86A002088130C17CE
:102132000000000074A2040800000000000000007B
:10214200000000000000000084A204080800000053
:1021520000000000E81900200400000090A204081A
:102162000800000000000000DC1900200000000050
:10217200209E040804000000B9D8020800000000F4
:1021820000000000AC9A04080100000000000000FA
:102192000000000000000000000000000E0000002F
:1021A200000000000000000000000000D46A0020CF
:1021B20088130C1701000000D26A002088130C1744
:1021C20000000000CCA204080F00000031D3020876
:1021D2000000000000000000F4190020766C0020CE
:1021E2000100000074590408D16A002001000000B7
:1021F20080590408F46E0020020000008859040887
:102202009AB40020000000000000000098B40020F2
:10221200000000000000000096B400200000000052
:102222000000000094B40020000000000000000044
:1022320092B40020000000000000000090B40020D2
:102242000000000000000000401E0020000000000E
:1022520000000000D06A0020020000009459040827
:10226200D4A20408000000000000000000000000EA
:102272000000000084A20408080000000000000022
:10228200781A00200400000090A204080800000050
:10229200000000006C1A002000000000209E0408CC
:1022A2000400000011D3020800000000000000003A
:1022B200AC9A0408010000000000000000000000C9
:1022C20000000000000000000E00000000000000FE
:1022D2000000000000000000E4A20408000000006A
:1022E200000000000000000000000000F4A204084A
:1022F2000D0000005DD90208B41A0020040000009D
:1023020000A304080D00000055D30208A81A0020FB
:10231200040000000CA304080D0000001DD90208EF
:102322009C1A00200000000018A30408030000000B
:1023320099D80208841A00200800000024A3040887
:1023420003000000DDDE0308DC1D002000000000A9
:10235200AC9A040801000000000000000000000028
:1023620000000000000000000E000000000000005D
:102372000000000000000000A49A04080000000011
:10238200000000000000000000000000659A040840
:10239200040000001DDA0208000000000000000036
:1023A200AC9A0408010000000000000000000000D8
:1023B20000000000000000000E000000000000000D
:1023C20000000000000000002CA304080000000030
:1023D2000000000000000000000000007C930408E0
:1023E2000D00000000000000141B0020040000008B
:1023F2003CA304080800000000000000081B0020A5
:102402000400000048A304080800000000000000C7
:10241200FC1A00200400000050A304080800000079
:1024220000000000F01A00200400000058A3040875
:102432000800000000000000E41A00200400000070
:1024420060A304080800000000000000D81A002061
:102452000400000068A30408080000000000000057
:10246200CC1A00200400000070A304080800000039
:1024720000000000C01A002004000000AC9A04080A
:102482000100000000000000000000000000000049
:10249200000000000E00000000000000000000002C
:1024A2000000000078A304080F00000021D30208F6
:1024B2000000000000000000201B002080A3040890
:1024C2000F000000000000000000000000000000FB
:1024D200981B002088A304080F00000000000000E1
:1024E2000000000000000000381C0020756C002075
:1024F20004000000A0590408CC6A0020E0150C1763
:1025020000000000CF6A0020080000003C5A0408C6
:10251200CE6A002005000000605A040890A3040857
:102522000F0000000000000000000000000000009A
:10253200881C002000FFFF0000000000AA550300D5
:102542009FAA5505010000AA5507010000000000DE
:10255200441E00200508020000000000605A040822
:102562003C5A0408345A04080000000001AA550B22
:10257200010000AA5509020000000000010000004D
:10258200C0120000D9EF020859ED020855ED020809
:1025920065FC020871F0020853ED020851ED0208D1
:1025A20039ED020829ED020821ED020825ED0208A5
:1025B200040309041201000202020040830440578E
:1025C2000002010203010000A5690308C5680308AF
:1025D2002DBB03089564030871680308A56403080A
:1025E200C1640308856403087564030800000000E1
:1025F200000000000101000009024300020100C0C6
:102602003209040000010202010005240010010544
:1026120024010001042402020524060001070582A8
:10262200030800FF09040100020A00000007050177
:10263200024000000705810240000000FF00000088
:10264200DD67030895670308E566030800000000DC
:102652005164030839660308B9660308A1650308D3
:10266200000000000000000045640308890103081F
:10267200850103088101030875010308710103083C
:102682007D01030879010308990103088D010308FC
:10269200C5020308D9020308B10203089D02030818
:1026A20089020308010000000C91040800000000E8
:1026B20000000000F5E20108A0860100040000000D
:1026C2000000000000000000000000000000000008
:1026D200000000000000000000000000B09D04089F
:1026E2003C85040800000000015901087D0000003B
:1026F20006000000000000000000000000000000D2
:1027020000000000000000000000000000000000C7
:10271200D0A60408000000000000000085D70308CE
:10272200E8030000030000000000000000000000B9
:102732000000000000000000000000000000000097
:1027420000000000D8A604080000000000000000FD
:1027520085B10208102700000300000000000000FD
:102762000000000000000000000000000000000067
:102772000000000000000000149C0408000000009B
:10278200F91C020891370108204E000005000000E4
:102792000000000000000000000000000000000037
:1027A2000000000000000000000000007C9204080D
:1027B20000000000000000002DD2030810270000D6
:1027C2000100000000000000000000000000000006
:1027D20000000000000000000000000000000000F7
:1027E200E4A6040800000000000000001DC5000867
:1027F200E8030000050000000000000000000000E7
:1028020000000000000000000000000000000000C6
:1028120000000000F0A60408000000000000000014
:1028220021E30108204E0000030000000000000028
:102832000000000000000000000000000000000096
:10284200000000000000000000A7040800000000D3
:102852000000000059EE0108204E000003000000B5
:102862000000000000000000000000000000000066
:1028720000000000000000000000000010A7040893
:10288200000000000000000091560108400D030006
:102892000300000000000000000000000000000033
:1028A2000000000000000000000000000000000026
:1028B200C09104080000000000000000658B0308BE
:1028C20010270000010000000000000000000000CE
:1028D20000000000000000000000000000000000F6
:1028E20000000000588504080000000000000000FD
:1028F200ED6A02081027000003000000000000003B
:1029020000000000000000000000000000000000C5
:10291200000000000000000020A7040800000000E2
:1029220000000000EDF80308A0860100010000008D
:102932000000000000000000000000000000000095
:1029420000000000000000000000000048850408AC
:1029520000000000000000000DF8030850C3000052
:102962000100000000000000000000000000000064
:102972000000000000000000000000000000000055
:1029820058A60408000000000000000075F30308C8
:10299200A86100000100000000000000000000002B
:1029A2000000000000000000000000000000000025
:1029B2000000000028A7040800000000000000003A
:1029C200C9750208A0860100010000000000000095
:1029D20000000000000000000000000000000000F5
:1029E20000000000000000008492040800000000C3
:1029F200000000001DF20008A00F0000010000000E
:102A020000000000000000000000000000000000C4
:102A120000000000000000000000000034A70408CD
:102A2200000000000000000051930208102700007F
:102A32000100000000000000000000000000000093
:102A42000000000000000000000000000000000084
:102A5200E89104080000000000000000F17803087B
:102A6200A00F0000010000000000000000000000B4
:102A72000000000000000000000000000000000054
:102A82000000000018A2040800000000000000007E
:102A9200DD8F03081A410000010000000000000061
:102AA2000000000000000000000000000000000024
:102AB2000000000000000000E8920408000000008E
:102AC2000000000081ED0208102700000100000054
:102AD20000000000000000000000000000000000F4
:102AE200000000000000000000000000788C0408D4
:102AF200000000000000000095DE02081A410000FC
:102B020001000000000000000000000000000000C2
:102B120000000000000000000000000000000000B3
:102B220040A7040800000000000000005D7A0308CE
:102B3200400D030000000000000000000000000043
:102B42000000000000000000000000000000000083
:102B52000000000048A70408000000000000000078
:102B6200197A0308400D0300000000000000000075
:102B72000000000000000000000000000000000053
:102B8200000000000000000050A704080000000040
:102B92000000000031E50108A086010003000000EA
:102BA2000000000000000000000000000000000023
:102BB2000000000000000000000000000000000013
:102BC200010203040102030406070809685E0C00FF
:102BD20043000000000000000000000000000000B0
:102BE20000000000000000000000000000000000E3
:102BF2004300000000000000000000000000000090
:102C020000000000000000000000000000000000C2
:102C1200430000000000000000000000000000006F
:102C220000000000000000000000000000000000A2
:102C3200430000000000000000000000000000004F
:102C42000000000000000000000000000000000082
:102C5200430000000000000000000000000000002F
:102C62000000000000000000000000000000000062
:102C7200430000000000000000000000000000000F
:102C82000000000000000000000000000000000042
:102C920043000000000000000000000000000000EF
:102CA2000000000000000000000000000000000022
:102CB200E10B0408210A04080000000025A9040809
:102CC200609A040884A5040884A5040884A504085D
:102CD20084A5040884A5040884A5040884A504081E
:102CE20084A5040884A50408FFFFFFFFFFFFFFFF80
:102CF200FFFFFFFFFFFF000001004153434949006E
:102D020000000000000000000000000000000000C1
:102D12000000000000000000000041534349490048
:102D220000000000000000000000000000000000A1
:102D3200000000000000000000000000002600204B
:102D42000000000000000000000000000000000081
:102D52000000000000000000000000000000000071
:102D62000000000000000000000000000000000061
:102D72000000000000000000000000000000000051
:102D82000000000000000000000000000000000041
:102D92000000000000000000000000000000000031
:042DA200010000002C
:1080000070B4EFF31186502383F31288436B1A6820
:10801000D20720D45D686DB9446A826A944217D051
:1080200081691144D9600ED9A21A5A608462002273
:1080300080F858201A6842F00102F1B21A6081F308
:10804000118870BC704701698A1A5A608562EEE730
:10805000012380F85830F3B283F3118870BC704765
:10806000436A8269D154436A0169426B01338B428E
:1080700028BF00234362002A2FD0EFF31182502340
:1080800083F31288436B1968C9072CD470B45E68F7
:108090006EB9456A816A8D4217D084690C44DC60F0
:1080A0000ED9691A59608562002180F85810196844
:1080B00041F00101D2B2196082F3118870BC70479F
:1080C0000469611A59608662EEE7012380F858302E
:1080D000D2B282F3118870BC7047426DD36843F00E
:1080E0008003D3607047D2B282F31188704700BF1B
:1080F000026B10B462B1836CC2684469D11A013B4F
:10810000615C5DF8044B08BF13468364C8B27047D6
:10811000016A4369C4685B5C0131A14228BF114612
:1081200001625DF8044BD8B2704700BF436B13B1D6
:1081300090F858007047836A406A181AB0FA80F0C5
:1081400040097047416A836A99420AD3CB1A416B4E
:10815000026961B14968501E0B4483420AD2C01AB9
:10816000704702691144CB1A416B0029F2D1501EAD
:10817000C01A704700207047036B43B1826C5B6884
:1081800093422FBF981AC0689B1AC0187047C269E3
:10819000036A9A422FBFD01AC0688018C01A70476D
:1081A0000A4B30B503F1140493F900205D78072AD7
:1081B000C8BF143A811804338D7213F8025C8554D9
:1081C00013F8012C0A75A342EED130BDDC3104084E
:1081D00003682DE9F041DF691FB13B46BDE8F0417E
:1081E0001847002A164611DD04460D460E4400E0ED
:1081F00023689B68204698470028F9D0236815F823
:10820000011B1B6820469847AE42F1D1BDE8F081C2
:1082100000231022027043708370C370704710B542
:10822000074B03F10C0193F900205C78845402445D
:108230009C78D470DC78947104338B42F3D110BDF8
:10824000F031040830B4846814B12368A5885D83D4
:10825000436840F2E93001E0002833D01D8901383D
:1082600015F0020F80B2F7D089B2998140F2E9315E
:1082700001E0002950D01889013910F0010F89B2AE
:10828000F7D0998940F2E93101E000292FD018890F
:10829000013910F0020F89B2F7D092B29A8140F200
:1082A000E93201E0002A4BD01989013A11F0010F9F
:1082B00092B2F7D09B8914B12368A2881A83012057
:1082C00030BC70472C498B4208D0A1F578418B42D5
:1082D0004CD001F580618B42D4D10220274901EBBB
:1082E00000104189013189B241814189CAE7224A9E
:1082F000934208D0A2F57842934235D002F58062CD
:108300009342D8D102211D4B03EB01114B8901335C
:108310009BB24B814B89CEE71748834207D018495F
:108320008B4227D001F580618B42ABD102211348EB
:1083300000EB01114889013080B248814989A1E7E9
:108340000D498B4207D00E4A934211D002F580624C
:108350009342B0D10222094B03EB0212538901333D
:108360009BB253815389A6E70121CCE70120B5E7F1
:108370000122F0E70121DAE700300140DCC60020ED
:1083800000380040002870B51EDB0928044620DDB7
:10839000012303EB83035B00B0FBF3F2092AF8D857
:1083A0007BB10E4EB4FBF3F00928CCBF572230222C
:1083B000A6FB03E5024403FB1044EB0801F8012B84
:1083C000F0D100230B7070BD2D230B7040420131A2
:1083D000DBE7303001F8010BF3E700BFCDCCCCCCAC
:1083E000884230B44FF001042ED301FB04F4B0FBFB
:1083F000F4F58D42F9D284B1AAB901E0B0FBF4F5ED
:10840000092DCCBF572230222A4404FB150003F863
:10841000012BB4FBF1F4002CF0D100221A7030BC17
:108420007047B0FBF4F5092DCCBF372230222A4427
:1084300004FB150003F8012BB4FBF1F4002CF0D180
:1084400000221A7030BC70470546002AEBD1D7E7EE
:1084500003685A1C02601970704700BF2DE9F0478D
:10846000089C2578002B804689460CBF4FF0200AD7
:108470004FF0300A661C35B3002A29DD334601E08F
:10848000024698B113F8011B501E0029F8D1971E1F
:1084900060B13D46013D51464046C8476B1C002B2C
:1084A000F8DC257827EAE770013055B1041B29462E
:1084B0004046C847301916F8015B002DF7D1BDE8DA
:1084C000F087BDE8F087002A04DC2846BDE8F08785
:1084D0000020EBE7571EDCE783684268D0ED037AA3
:1084E00000EB83010133934281ED040A836004BFF2
:1084F0000023836000EB830393ED047A036870EE3E
:10850000277A9A42C0ED037A77EEC77AC0ED037AF4
:108510000CDA013307EE103AF8EEC76AB7EE007ACC
:1085200087EEA60A036030EE070A704707EE102AAE
:10853000B8EEC77A87EE870A704700BF90ED057ADC
:1085400090ED004AD0ED066AD0ED014AD0ED047AF4
:1085500090ED035AD0ED025AA4EE007AB0EE406AD4
:10856000B0EE470AB0EE667AA6EE247A67EEC07ADD
:10857000A0EE457AE6EE257A80ED057AC0ED067A22
:10858000704700BFD0ED057A90ED013AD0ED003A8A
:10859000D0ED064A90ED024A90ED077A90ED035A2D
:1085A00090ED086AD0ED045AC0ED067AF0EE406A0C
:1085B00027EE830AC0ED056AA3EEA60A80ED087ACD
:1085C000A4EE240AA5EE470AA5EEC60A80ED070A26
:1085D000704700BFD0ED007A90ED017A30EE670A67
:1085E000E7EE007AB0EE670AC0ED007A704700BF90
:1085F000704700BF0A44914214D030B40139551E6F
:1086000041F2210211F8014F082380EA04200404FA
:108610004CBF82EA40004000013B80B2F7D18D425E
:10862000F0D130BC704700BF704700BF704700BF3B
:108630002DE9F04FDFF8F8C1DFF8F8E1BCF80A7077
:10864000DEF80060BCF80C30BCF808A03C028BB02F
:10865000361B4FF00004CDE90034009CBCF8063016
:108660004FEA17654FF0000767EB0507B946B046BC
:10867000A4FB06670024CDE90634009C002304FB1C
:1086800009770024CDE90034AAFB0823CDE90223B1
:10869000039AF30D00930AFB09230393009B43EA1B
:1086A00047230093029B4FEAD31AFB150193039BC8
:1086B0004AEA436ADDE9002344464D46CDE90845D0
:1086C000069C12F5FA62A4FB086743F1000304FB61
:1086D0000977CDE90623BCF80440039BBCF80220CF
:1086E0004FEAE31B230C059323040493340A44EA62
:1086F00007643D12DDE904674FEAC23816EB0A064B
:1087000047EB0B0718EB0408DDE906344FEA524942
:1087100049EB0509B3F5FA6F74F10004B246BB46A4
:108720003CDADDE90067BC00B20044EA9673B41895
:1087300047EB030522463C462B4602FB04F406FBAE
:108740000344A2FB06232344940844EA83749D1047
:108750005B104FEA3202B8EB040869EB0509BAEB8B
:10876000020A6BEB030BDDE90623304C4FF0FF35BB
:10877000A242AB412CDBDDE90856A5FB052305FB36
:1087800006F403EB4403D40F44EA4304DD17DDE9A8
:108790000623121B63EB0503CDE90623DEF8044034
:1087A000A4FB082304FB0933540D44EAC3245D15DC
:1087B000B4EB0A0A65EB0B0B4FEADA3343EA4B439F
:1087C00000B1036009B1069B0B600BB0BDE8F08FF0
:1087D00040F6AC52B4184FF0000347EB03052246B5
:1087E000A2FB022304FB05F403EB4403941843EBC0
:1087F0000305A4185D414FEA850CA6004CEA947C61
:10880000B41A6CEB0305DF00D6006D104FEA340498
:1088100047EA5277921B63EB0703B8EB040869EB56
:1088200005091AEB020A4BEB030BA4E724FAFFFF3E
:1088300078500020642600202DE9F04FDFF81CB2AC
:10884000DFF81CE2BBF80020DEF80860BBF904305A
:10885000BBF90250BBF90A80C2EB261404FB04F4F6
:1088600024135200C2EBE60203FB04F305FB02F201
:108870009B1303EBE223B3F5FA364FEAE37589B0B5
:1088800045F1FF373246A6FB0645CDE9024502FB1E
:1088900007F205EB4202CDE90467029EBBF90840EE
:1088A000039208FB02FC4FEAE87906FB09CC3A4642
:1088B000A8FB0689049ECBF81830E51704FB02F2EA
:1088C00006FB0522A4FB0667E14417444FEA182281
:1088D00042EA096200924FEA292201923D03DDE952
:1088E0000078340345EA16553F19BBF80660069038
:1088F00048EB05083C1C48F5004503EB8302A4FB4C
:10890000068906FB0599803213124FEA69064FEA81
:10891000E977079356EA07038A4600F09280DDE97B
:108920000489BBF90E20DEF80C40BBF91000494663
:10893000C4F5801ED317DDE9024502FB01F108FBF7
:108940000311A2FB08230B444FEA43492B46C117EE
:1089500000FB03F304FB0133A0FB0401BBF90C4053
:108960001944E30001937346DC170023009349EA9E
:10897000D2394FEA4248DDE9002310EB080041EB11
:108980000901E50712184FEACE744B4145EA5E052E
:10899000A41A65EB0305221945EB050312196B4177
:1089A00099019001801841EA926159418B0082003F
:1089B00043EA9073101943EB05018B00820043EAF0
:1089C000907310460019194632463B46694137F00C
:1089D0007BFDBBF916204C13450B45EAC14502FB54
:1089E00004F6D31705FB0366A2FB05233344BBF94A
:1089F000146002FB04F405FB034406FB01FEA2FB2A
:108A00000523F717234400FB07EE540EA6FB00676F
:108A1000774444EAC3144FEAD64800194FEA636525
:108A200048EA473869414FEAE74918EB0008BBF9C3
:108A3000124049EB01094FEA182646EA096620016F
:108A40003618069B0BB1360A1E60BAF1000F02D031
:108A5000079BCAF8003009B0BDE8F08F88500020AD
:108A600064260020704700BF4FF400638382704784
:108A70004FF400638382704750F8043C012280F871
:108A80004520103803B11847704700BFBFF34F8F20
:108A90000549064BCA6802F4E0621343CB60BFF39A
:108AA0004F8F00BFFDE700BF00ED00E00400FA05B6
:108AB000F8B5057B466903681F2D29D9A5F1200467
:108AC0005F682021A1400F422A4613D01022A24005
:108AD000D960DA605A68E240D10703D5012202FA70
:108AE00004F4DC6004463046FFF78AFA227B2368F0
:108AF0001F2A20D9A2F1200008215A688140114282
:108B000000D0D9600422596882400A4221D1F8BDC0
:108B100020211C68A9400C422A460CD01022AA40F1
:108B200099609A601A68EA40D207DBD5012202FAFE
:108B300005F59D60D6E7082118689140014200D0F4
:108B400099600421186801FA02F2024203D09A6087
:108B5000F8BDDA60F8BDF8BD70B4037B04681F2B64
:108B600008D9203B2021626801FA03F31A421CD184
:108B700070BC70472021226801FA03F31A42F7D033
:108B800042691449582000FB021251685689CD6889
:108B90000868296821F001012960828992B222EADD
:108BA00006028281A36070BC70474269094958205F
:108BB00000FB021251685689CD680868296821F0C7
:108BC00001012960828992B222EA06028281E36071
:108BD00070BC70474493002030B4094B1C786CB1D2
:108BE000084A002502EBC404116893884D62888905
:108BF000083203439BB2A2428B81F5D130BC70474F
:108C0000049600200896002010B4037B01681F2BF7
:108C100009D9203B20224C6802FA03F31C4214D1EC
:108C20005DF8044B704720220C6802FA03F31C42E3
:108C3000F6D00C4A40680024147002685DF8044BBA
:108C400022F0010202608B607047064A40680024EF
:108C5000147002685DF8044B22F001020260CB60E0
:108C6000704700BF4F660020F0B5C4002218920084
:108C7000AE498B585B689D8AADB2EEB2F7070A44E5
:108C80005CD4B70732D5BFF35F8F167EF6B2012EE4
:108C900000F0C780A64D1A8BBFF35F8F221801EB3F
:108CA0008202167E022E00F0D580221801EB82028D
:108CB000167E032E00F088809A8895F9106092B293
:108CC00042F480629A80221801EB8202127E013205
:108CD00096425BD1AA7C00266E74002A40F09580F3
:108CE000204401EB800000234375F0BD77074ED48C
:108CF00016F0400600F0C9808D4D1E8A95F910E0EF
:108D0000176AF6B207F80E605FFA8EFE0EF1010CDC
:108D10004FFA8CFC177E85F810C00CF103029742C5
:108D2000664600F01C81221801EB8202127E9445F7
:108D3000C9D10EF1020676B22E74C4E71E887C4DAE
:108D400026F400663604360C1E801E88B6B246F441
:108D500080661E80967E00272F74002E48D06E7C81
:108D6000002E42D0221801EB82020126127E6E7480
:108D7000022A00F0B980221801EB8202927D42F0B3
:108D800001021A82204401EB8000037EF0BD684D91
:108D9000967E0127AF74002E73D06E7C002E7BD19F
:108DA000221801EB8202527E002A00F0A3801A886A
:108DB0002E7C92B2013642F4007276B21A802E7482
:108DC0001A88D205FCD47EE7927E002A3FF474AF65
:108DD0006A7C002A3FF470AF9A8895F9106022F4FB
:108DE00080621204120C9A806DE7D27DFF2AB9D0FE
:108DF000221801EB8202967D06F0FE061E82D37DCC
:108E0000FF2BBFD0FF232B74BCE79A8822F440725B
:108E100012042044120C01EB80009A800023437559
:108E2000F0BD927E424D002A3FF435AF6A7C002AA5
:108E30003FF431AF1A8822F480621204120C1A80B7
:108E4000BFF35F8F1A8B1A88AE7492B242F400722D
:108E50001A8031E7927E002A3FF427AF6A7C002A0D
:108E60003FF423AF1A8895F9106022F4806212044F
:108E7000120C1A809A8822F480621204120C9A80D2
:108E800021E76A7C002A8BD091E715F0800F284DEE
:108E90003AD195F9106016E7167ED2F820E01F88C7
:108EA000022E95F9106045D927F480673F043F0CE6
:108EB0001F801F8AFFB20EF806701F88D2F820E0CC
:108EC000BFB247F400771F80F2B21F8A561C76B2F9
:108ED000FFB20EF806709F88961CBAB276B242F4C2
:108EE00080622E749A806BE71A8892B242F4006214
:108EF0001A8040E71A8895F9106092B242F48072A5
:108F000001271A806F745BE795F91070B7F1FF3F86
:108F10002CD0D669F65D1E8292F818E001377AB23D
:108F2000964516462A747FF4CEAEA3E7B8450020D6
:108F300064260020BFB247F400771F801F8AFFB26B
:108F40000EF80670F6B21F8AD2F820E0721C52B2F8
:108F50000336FFB276B20EF802702E7430E79A88AC
:108F600022F480621204120C9A80DCE6D77D1F8204
:108F70002E74957E1DB9127E002A7FF403AF9A8865
:108F800022F480621204120C9A80FBE670B504464B
:108F900082B01430E56D06236A464321A847B0B17C
:108FA0009DF804009DF800609DF801109DF80250A6
:108FB0009DF803209DF8053041EA062143EA00238D
:108FC00042EA0522A187E287A4F84030012002B0DE
:108FD00070BD00BF70B5044682B00830656A0623D4
:108FE0006A463B21A847A8B19DF804009DF800609F
:108FF0009DF801109DF802509DF803209DF8053062
:1090000041EA062143EA002342EA0522E182228363
:109010006383012002B070BD002328220360027028
:109020002922C270012243608360827143727047BB
:10903000F8B50468C4F30D0405460E4604B32F6862
:1090400033F01CFA092840F08880454C236923F44A
:1090500040732361236943F400732361236943F060
:10906000010323613E6033F009FA2369092823F0E4
:109070000103236171D12B6804332B600020F8BDFC
:10908000384B394A93422BD902F58042934226D974
:1090900002F5804293422AD902F58042934228D9B0
:1090A00002F58032934226D902F50032934224D948
:1090B00002F50032934222D902F50032934220D9C0
:1090C00002F5003293421ED902F5802293421CD948
:1090D000B3F1016F1BD3052005F076FAFBE70824F6
:1090E00033F0CCF9092814D04FF0FF30F8BD10242C
:1090F000F6E71824F4E72024F2E72824F0E73024E8
:10910000EEE73824ECE74024EAE74824E8E758246F
:10911000E6E7134F3B6923F440733B613B6943F43B
:1091200000733B613B6923F0F8033B613B6943F00B
:1091300002031C433C613B6943F480333B6133F0E1
:109140009DF93B6923F002033B613B69092823F049
:10915000F8033B613FF473AFC6E76FF00100F8BD61
:10916000003C024000400008FF3F0008F8B50446FC
:109170000D468E180027B54201D12069F8BDE3687D
:10918000591CE160234415F8012B1A720429F2D10D
:10919000206918B9A1682046FFF74AFF2061E760FF
:1091A000E9E700BF70B582B004466946143029F083
:1091B0003DFEB0B19DF805009DF801609DF80210DC
:1091C0009DF803509DF804209DF8063041EA0621E1
:1091D00043EA002342EA0522A187E287A4F840304F
:1091E000012002B070BD00BF38B5254B9C68236BD1
:1091F00073B1636D626BCAB1998A1A88C90592B25C
:1092000001D5D20700D438BD4FF6F7721A8038BDA9
:10921000636D99891A88890692B2EBD59206E9D5D1
:10922000E26ACAB1988880B29047E2E799891A88C1
:109230000D0692B2E0D51006DED5A26A616A8A42B6
:1092400019D0A1692569885C98800132B2FBF5F1DB
:1092500005FB1122A262CFE79B88E2696169DBB25C
:109260008B54E269E068636D0132B2FBF0F100FB00
:109270001122E261BEE7DA6822F08002DA60BBE721
:109280009045002038B5254B5C68236B73B1636D46
:10929000626BCAB1998A1A88C90592B201D5D20700
:1092A00000D438BD4FF6F7721A8038BD636D9989C6
:1092B0001A88890692B2EBD59206E9D5E26ACAB15C
:1092C000988880B29047E2E799891A880D0692B291
:1092D000E0D51006DED5A26A616A8A4219D0A1697A
:1092E0002569885C98800132B2FBF5F105FB1122FB
:1092F000A262CFE79B88E2696169DBB28B54E269C5
:10930000E068636D0132B2FBF0F100FB1122E26113
:10931000BEE7DA6822F08002DA60BBE79045002001
:1093200038B5254B1C68236B73B1636D626BCAB192
:10933000998A1A88C90592B201D5D20700D438BDDE
:109340004FF6F7721A8038BD636D99891A888906BD
:1093500092B2EBD59206E9D5E26ACAB1988880B29A
:109360009047E2E799891A880D0692B2E0D5100677
:10937000DED5A26A616A8A4219D0A1692569885C32
:1093800098800132B2FBF5F105FB1122A262CFE712
:109390009B88E2696169DBB28B54E269E068636DC6
:1093A0000132B2FBF0F100FB1122E261BEE7DA68A4
:1093B00022F08002DA60BBE79045002003685B6A18
:1093C00003B11847704700BF03681B6A03B1184711
:1093D000704700BF03682DE9F041DF691FB13B46CC
:1093E000BDE8F0411847002A164611DD04460D4637
:1093F0000E4400E023689B68204698470028F9D077
:10940000236815F8011B1B6820469847AE42F1D12E
:10941000BDE8F08103689B69184700BF03685B697A
:10942000184700BF03681B69184700BF0368DB6863
:10943000184700BF03689B68184700BF03685B6854
:10944000184700BF03681B68184700BF014B186826
:10945000F8E700BF4CC4002038B50C46097849B184
:10946000054601342B6828461B68984714F8011BF1
:109470000029F7D138BD00BF064B53F820302BB17F
:109480001A689B8851690B4201D11383704753833B
:10949000704700BF80D0002003682DE9F04F03F132
:1094A0003F4404F57E04604EA40A0125345D04F0B7
:1094B0001F066409032C05FA06F500F0AF80042CA2
:1094C00000F0A780022C54D08588B5FA85F0C0F151
:1094D0001F0080B2C40803EB840400F00700266A72
:1094E00080000F27874026EA07062662276A01F0D8
:1094F000030602FA00F0721E3843012AC1F3810C00
:10950000C1F300182062C1F3411137D9002422466B
:1095100001274FF0030E03E0102A04F1020426D0C5
:1095200007FA02F0A84302F10102F5D1D3F800C016
:109530000EFA04F0C04300EA0C0CC3F800C0D3F8E4
:10954000008006FA04FC4CEA080CC3F800C0D3F80B
:109550000CC000EA0C00D860D3F80CC001FA04F08B
:1095600040EA0C00102AD86004F10204D8D1BDE80A
:10957000F08F2E4C666C35436564A5E700200246EB
:109580004FF0010E4FF0030904E00132102A00F100
:1095900002003CD00EFA02F737EA0504F5D1D3F801
:1095A00000A009FA00F4E4430AEA040AC3F800A0A0
:1095B000D3F800B006FA00FA4AEA0B0AC3F800A092
:1095C000D3F808A004EA0A0AC3F808A0D3F808B040
:1095D0000CFA00FA4AEA0B0AC3F808A0D3F804A070
:1095E0002AEA07075F60D3F804A008FA02F747EAFF
:1095F0000A075F60DF683C40DC60DF6801FA00F466
:1096000001323C43102ADC6000F10200C2D1BDE807
:10961000F08F064C266B3543256355E7034C266CCB
:109620003543256450E700BF105C04080038024051
:10963000026802F13F4303F57E032DE9F04F9B0AD8
:10964000544DEB5C03F01F055B090124032B04FA66
:1096500005F400F09980042B00F09180022B3ED09D
:1096600001F00306731E012BC1F3810CC1F3001836
:109670008588C1F3411137D90024234601274FF0D3
:10968000030E03E0102B04F1020426D007FA03F0C6
:10969000A84303F10103F5D1D2F800C00EFA04F09B
:1096A000C04300EA0C0CC2F800C0D2F8008006FAF1
:1096B00004FC4CEA080CC2F800C0D2F80CC000EA66
:1096C0000C00D060D2F80CC001FA04F040EA0C00A3
:1096D000102BD06004F10204D8D1BDE8F08F2E4BDE
:1096E0005D6C2C435C64BBE7002003464FF0010E29
:1096F0004FF0030904E00133102B00F102003CD0CD
:109700000EFA03F737EA0504F5D1D2F800A009FAFA
:1097100000F4E4430AEA040AC2F800A0D2F800B058
:1097200006FA00FA4AEA0B0AC2F800A0D2F808A02A
:1097300004EA0A0AC2F808A0D2F808B00CFA00FA43
:109740004AEA0B0AC2F808A0D2F804A02AEA0707DE
:109750005760D2F804A008FA03F747EA0A075760EF
:10976000D7683C40D460D76801FA00F401333C4329
:10977000102BD46000F10200C2D1BDE8F08F064B7F
:109780001D6B2C431C636BE7034B1D6C2C431C644B
:1097900066E700BF105C04080038024010B50409F9
:1097A000013C032C17D80D4B33F8142000F00F00A8
:1097B00042FA00F313F001030DD0012303FA00F085
:1097C0000138104036F0D0FE054A064B125D1044B9
:1097D00003EBC00010BD002010BD00BFE46604080C
:1097E000E0660408F4CE00202DE9F04F4A484B49CA
:1097F0004B4B4C4C4FF0010A4FF002094FF004085C
:109800004FF0080C4FF0100E20274026802530F82E
:10981000022B12F0010F03D01960A3F804A0083343
:1098200012F0020F03D01960A3F80490083312F06D
:10983000040F03D01960A3F80480083312F0080F56
:1098400003D01960A3F804C0083312F0100F03D03E
:109850001960A3F804E0083312F0200F02D0196059
:109860009F80083312F0400F02D019609E800833A9
:1098700012F0800F02D019609D80083312F4807FAF
:1098800005D04FF4807B1960A3F804B0083312F4BC
:10989000007F05D04FF4007B1960A3F804B00833B3
:1098A00012F4806F05D04FF4806B1960A3F804B0F8
:1098B000083312F4006F05D04FF4006B1960A3F861
:1098C00004B0083312F4805F05D04FF4805B196058
:1098D000A3F804B0083312F4005F05D04FF4005B26
:1098E0001960A3F804B0083312F4804F05D04FF488
:1098F000804B1960A3F804B00833D20B04D04FF4A6
:10990000004219609A80083301F58061A1427FF41A
:109910007EAFBDE8F08F00BFE4660408000002409F
:10992000F4CE00200010024000286AD003682DE920
:10993000F04F03F13F4404F57E045F4EA40A012575
:10994000345D04F01F066409032C05FA06F559D0AE
:10995000042C00F0AC80022C59D08588B5FA85F033
:10996000C0F11F0080B2C40803EB840400F00700BC
:10997000266A80000F27874026EA07062662276AA4
:1099800001F003068240701E3A430128C1F3810CA6
:10999000C1F300182262C1F341113DD900242246CF
:1099A00001274FF0030E03E0102A04F1020426D031
:1099B00007FA02F0A84302F10102F5D1D3F800C082
:1099C0000EFA04F0C04300EA0C0CC3F800C0D3F850
:1099D000008006FA04FC4CEA080CC3F800C0D3F877
:1099E0000CC000EA0C00D860D3F80CC001FA04F0F7
:1099F00040EA0C00102AD86004F10204D8D1BDE876
:109A0000F08F70472D4C266C35432564A5E72B4C11
:109A1000666C35436564A0E7002002464FF0010EF6
:109A20004FF0030904E00132102A00F102003CD09B
:109A30000EFA02F737EA0504F5D1D3F800A009FAC7
:109A400000F4E4430AEA040AC3F800A0D3F800B023
:109A500006FA00FA4AEA0B0AC3F800A0D3F808A0F5
:109A600004EA0A0AC3F808A0D3F808B00CFA00FA0E
:109A70004AEA0B0AC3F808A0D3F804A02AEA0707A9
:109A80005F60D3F804A008FA02F747EA0A075F60AC
:109A9000DF683C40DC60DF6801FA00F401323C43DF
:109AA000102ADC6000F10200C2D1BDE8F08F034C47
:109AB000266B3543256350E7105C040800380240EC
:109AC000002855D0026802F13F4303F57E032DE9DB
:109AD000F04F9B0A544DEB5C03F01F055B0901241A
:109AE000032B04FA05F444D0042B00F09780022BDA
:109AF00044D001F00306731E012BC1F3810CC1F3A6
:109B000000188588C1F341113DD90024234601275F
:109B10004FF0030E03E0102B04F1020426D007FAE5
:109B200003F0A84303F10103F5D1D2F800C00EFA07
:109B300004F0C04300EA0C0CC2F800C0D2F8008068
:109B400006FA04FC4CEA080CC2F800C0D2F80CC0BB
:109B500000EA0C00D060D2F80CC001FA04F040EA30
:109B60000C00102BD06004F10204D8D1BDE8F08FB6
:109B700070472E4B1D6C2C431C64BAE72B4B5D6C5D
:109B80002C435C64B5E7002003464FF0010E4FF014
:109B9000030904E00133102B00F102003CD00EFA5F
:109BA00003F737EA0504F5D1D2F800A009FA00F46A
:109BB000E4430AEA040AC2F800A0D2F800B006FAA8
:109BC00000FA4AEA0B0AC2F800A0D2F808A004EA98
:109BD0000A0AC2F808A0D2F808B00CFA00FA4AEA59
:109BE0000B0AC2F808A0D2F804A02AEA07075760B7
:109BF000D2F804A008FA03F747EA0A075760D768C3
:109C00003C40D460D76801FA00F401333C43102B88
:109C1000D46000F10200C2D1BDE8F08F034B1D6B90
:109C20002C431C6365E700BF105C04080038024049
:109C300010B1036882885A83704700BF10B103686F
:109C400082881A83704700BF18B10368828809B9F7
:109C50005A8370471A83704710B40A4B0A4A1C781B
:109C600001238340234052F8200029B9B3FA83F13D
:109C700049095DF8044BE7E7191C18BF01215DF89D
:109C8000044BE1E77CD0002080D0002030B1036895
:109C900082881B691A4214BF01200020704700BF50
:109CA00038B5044690F8590000285AD104F114053B
:109CB000236E80226B2128469847642005F02EF9F8
:109CC000236E0722682128469847642005F026F96C
:109CD000236E00226B2128469847642005F01EF968
:109CE000236E01226B21284698470F2005F016F9B4
:109CF00094F85320236E032A8CBF1A2218221B21AA
:109D0000284698470F2005F009F9236E18221C21D8
:109D1000284698470F2005F001F9236E94F8522049
:109D20001A21284698470F2005F0F8F8236E94F87A
:109D30005420192128469847642005F0EFF8236E37
:109D400010223721284698470F2005F0E7F82846CB
:109D5000236E0122382198470F20BDE8384005F0D6
:109D6000DDB8FFF71BFD0546FFF790FF00289DD1EA
:109D700015B12023E871AB7128460021FFF7A0FE42
:109D80002146054B41F8103F284635F087FA284612
:109D900035F072FA8AE700BF798A00082DE9F041B0
:109DA0000B4E346873691C400FD0DFF82880012700
:109DB000B4FA84F3C3F11F0307FA03F558F823003C
:109DC00003689847AC437561F2D1BDE8F08100BFEC
:109DD000003C0140BCD000202DE9F0410B4E34681E
:109DE00073691C400FD0DFF828800127B4FA84F390
:109DF000C3F11F0307FA03F558F8230003689847D7
:109E0000AC437561F2D1BDE8F08100BF003C014078
:109E1000BCD000202DE9F0410B4E346873691C4022
:109E20000FD0DFF828800127B4FA84F3C3F11F03B1
:109E300007FA03F558F8230003689847AC437561A7
:109E4000F2D1BDE8F08100BF003C0140BCD0002051
:109E50002DE9F0410B4E346873691C400FD0DFF8D8
:109E600028800127B4FA84F3C3F11F0307FA03F52E
:109E700058F8230003689847AC437561F2D1BDE8F8
:109E8000F08100BF003C0140BCD000202DE9F04132
:109E90000B4E346873691C400FD0DFF8288001270F
:109EA000B4FA84F3C3F11F0307FA03F558F823004B
:109EB00003689847AC437561F2D1BDE8F08100BFFB
:109EC000003C0140BCD000202DE9F0410B4E34682D
:109ED00073691C400FD0DFF828800127B4FA84F39F
:109EE000C3F11F0307FA03F558F8230003689847E6
:109EF000AC437561F2D1BDE8F08100BF003C014088
:109F0000BCD000202DE9F0410B4E346873691C4031
:109F10000FD0DFF828800127B4FA84F3C3F11F03C0
:109F200007FA03F558F8230003689847AC437561B6
:109F3000F2D1BDE8F08100BF003C0140BCD0002060
:109F4000084A094808B5536C43F480435364002120
:109F5000402239F08EF8054B4FF0FF321A60C3F8FB
:109F6000032008BD00380240BCD00020FCD00020F7
:109F70002DE9F041044618460D461646984635F040
:109F8000D9FD2768E6722844A07229467D694346B8
:109F900032462046AC46BDE8F0416047036810B544
:109FA00004461B689847236820469B689847A37B14
:109FB0000133A37310BD00BF10B5036804469B684E
:109FC0009847FF2301226373227310BD08B5FFF782
:109FD000E5FB38B12C2282710022C2712021BDE83C
:109FE00008406DE508BD00BF40F2E93300E0A3B1D1
:109FF0000289013B12F0020F9BB2F8D089B2818135
:10A0000040F2E93300E043B10289013B12F0010F55
:10A010009BB2F8D08089C0B270470C4A904209D0F8
:10A020000B4B984210D003F58063984201D0FF207B
:10A0300070470223074A02EB03135A89013292B296
:10A040005A815889C0B270470123F3E700300140BC
:10A0500000380040DCC6002038B500231C4620FA3A
:10A0600003F2C3F11F0102F0010201338A40202BE9
:10A0700044EA0204F3D1104D2868FFF7D9FD210E00
:10A080000E48FFF7B1FFC4F307410C48FFF7ACFFE0
:10A09000C4F307210948FFF7A7FFE1B20748FFF71C
:10A0A000A3FF022004F0E0FE2868FFF7C7FD0220AE
:10A0B000BDE8384004F0D8BE30460020003C0040E7
:10A0C000144B984224D003F58063984220D0028834
:10A0D00022F040021204120C0280028822F038039F
:10A0E0001B041B0C59B141F48071002991FAA1F2B3
:10A0F000B2FA82F108BF4FF0FF310139C9000B43BA
:10A100009BB2038003889BB243F0400303807047F7
:10A110004908DCE70038004010B58021044680691A
:10A12000FFF7CEFF012004F09FFE2046FFF7B8FDA9
:10A1300010226A2104F11400FEF784F8642004F070
:10A14000EDFEA0690421FFF7BBFF0120BDE8104030
:10A1500004F08ABEF0B484894FF6FF764FF47A7427
:10A1600063B300293CD00F78013101E0B4421AD02A
:10A170000589013C15F00205A4B2F7D0BCB2848178
:10A180004FF47A7402E0BCB2B4420CD0058915F0E9
:10A19000010504F1FF37F6D08589ADB20AB115701B
:10A1A0000132013BDCE7104B98420BD0A3F578431A
:10A1B000984217D003F58063984202D00120F0BC8A
:10A1C00070470225094B03EB05156B8901339BB2E0
:10A1D0006B81688980B2003018BF0120F0BC7047E5
:10A1E000FF27C5E70125EDE700300140DCC6002070
:10A1F00070B50546806810B104688088608341F0BE
:10A200008001686840F2E93400E0E4B10689013C6D
:10A2100016F0020FA4B2F8D089B2818140F2E93180
:10A2200000E029B30489013914F0010F89B2F8D094
:10A2300081890021FFF78EFFAB6813B11A689B88F4
:10A240001383012070BD1649884208D0A1F57841DA
:10A25000884221D001F580618842EAD10224114967
:10A2600001EB04146189013189B261816189E0E700
:10A270000B4CA04207D00C4988420FD001F58061F9
:10A280008842D6D10221074C04EB01114C890134DC
:10A29000A4B24C814989CCE70124E0E70121F2E72F
:10A2A00000300140DCC6002000380040F8B5050150
:10A2B000684C694B625961199A4204EB050704BF67
:10A2C00001230B730646387A34F000FC3B7A03F026
:10A2D0001F015B090122032B02FA01F26DD0042B4E
:10A2E00066D0022B5CD0631901361879FFF756FA55
:10A2F000F6B2074610B11223C671837163195879FB
:10A30000FFF74CFA10B11323C67183716319987962
:10A31000FFF744FA10B11423C671837166190A213C
:10A32000F2793846FFF700FB7079FFF737FAF279D8
:10A330000A21FFF7F9FAB079FFF730FAF2790A212A
:10A34000FFF7F2FA6359454A934247D0424A934293
:10A3500050D0434A934259D0424A934262D0424A33
:10A3600093426BD0414A93422CD02C44227BE2B9D9
:10A3700001200222198801F4415141F445710A4338
:10A3800002431A809A8B22F400621204120C0721F5
:10A390009A8319821A8892B242F040021A80F8BD5C
:10A3A000334B596A0A435A629DE700200246E1E7AF
:10A3B0002F4B19690A431A6195E72D4B196A0A4315
:10A3C0001A6290E702F564424FF40010536A43F4B6
:10A3D0000013536231F04CFF6359C6E702F5843233
:10A3E0004FF48050536A43F48053536231F040FF7E
:10A3F0006359BAE702F500324FF48040136A43F420
:10A400008043136231F03CFF6359AEE702F5FE3240
:10A410004FF40040136A43F40043136231F030FFFD
:10A420006359A2E702F582324FF40050536A43F4B5
:10A430000053536231F01CFF635996E702F56842FE
:10A440004FF48010536A43F48013536231F010FFCD
:10A4500063598AE7DCC60020003800400030014024
:10A46000003C0040003401400050014000540140D5
:10A4700000380240427A02B9704710B504460368BA
:10A48000406804F10A0198470023637210BD00BFC1
:10A49000437A5A1C0344D2B242729972037A9342AD
:10A4A00000D802B9704710B504460368406804F14B
:10A4B0000A0198470023637210BD00BF302828D0DE
:10A4C000312828D0322828D0332828D0342828D042
:10A4D000352828D0202828D0212828D0102828D076
:10A4E000112828D0122828D0132828D0142828D0A2
:10A4F000152828D0162805D0172808BF0F2202D00B
:10A50000002070470E22114B03EB420393F8210009
:10A5100070470022F7E70122F5E70222F3E7032262
:10A52000F1E70422EFE70522EDE70622EBE7072239
:10A53000E9E70822E7E70922E5E70A22E3E70B2239
:10A54000E1E70C22DFE70D22DDE700BFDC31040884
:10A5500070B5448806460D46C4F30B04224600211C
:10A56000284638F086FD3369094A934209D3094ADF
:10A57000934206D2224628461946BDE8704036F07E
:10A5800061BA23B121462846BDE87040184770BD26
:10A590004006000842070008064B07498B4202D3D9
:10A5A0000023184670471A88C2F30B029042F8D075
:10A5B0001433F3E79001000840060008024A1368CC
:10A5C00023EA000010607047786C0020F8B5174D42
:10A5D0002B78A32B28D16B78BE2B25D102222946BC
:10A5E0004FF6FF70FEF706F8114FAC1C22884AB1F7
:10A5F000A618BE4218D2052A16D92146FDF7FAFF41
:10A600003446F3E721460222FDF7F4FF0222A118A7
:10A61000FDF7F0FF0634074B641B1C8041F60F5317
:10A62000C31A58425841F8BD0020F8BD0040000848
:10A6300000800008A64700202DE9F04FDFF84C917C
:10A640004D4F8BB00326A7EB09071822002104A861
:10A6500038F00FFD494BCDF8109005971A69002A84
:10A6600004DA474A5A6002F188325A6001228DF8B2
:10A670002420F322DA60434B434C1B88ADF80030B2
:10A680000222694604A8FEF771FD022269464FF6D0
:10A69000FF70FDF7AFFFDFF8F8A080464FF0000B2A
:10A6A000544539D30AAC002524F8245D0222214602
:10A6B00004A8FEF75BFD022221464046FDF79AFF03
:10A6C00040BAC043ADF80800022202A904A8FEF770
:10A6D0004DFD079878B106ABC0F104022946184435
:10A6E00038F0C7FC089818B9069904A8FEF7A0FC32
:10A6F0000023089007939DF82430089A23B11F493E
:10A700000B6943F000430B61013E2DD0002A9CD120
:10A71000FFF75CFF50B32CE065888DF80DB0C5F3F2
:10A720000B05AB1DADF808302388C3F30B02ADF861
:10A730000A201B0B062202A904A88DF80C30FEF794
:10A7400015FD062202A94046FDF754FF61688046C8
:10A750002A4604A8FEF70AFD616840462A46FDF72E
:10A7600049FF143480469BE7002AD1D0052003F02E
:10A770002BFF0BB0BDE8F08F00800008003C0240CA
:10A78000230167451C3204089001000800400008BE
:10A79000400600080378202B024600F10100F9D0A2
:10A7A000092BF7D02D2B2CD02B2B03BF5378B7EED2
:10A7B000000A0246B7EE000AA3F13001C8B2092828
:10A7C0009FED467A10D8F2EE046A07EE901AF8EE82
:10A7D000E77A12F8013FE7EE267AA3F13001C8B21A
:10A7E0000928B0EE677AF0D92E2B4CD003F0DF03A6
:10A7F000452B0BD0F7EE007A67EE276A20EE260A8B
:10A8000070475378BFEE000A0246D5E710B451787E
:10A810002D2959D02B290ABF9178501C901C002457
:10A82000A1F13003092B53D8002303EB830301EB81
:10A83000430310F8011FA1F13002092AA3F13003EC
:10A84000F3D9B3F59A7F28BF4FF49A73072B42D9F7
:10A85000DFED236A1A46F7EE007A083A072A67EE18
:10A86000A67AFAD803F007032BB1F2EE046A013B93
:10A8700067EEA67AFBD124B3C7EE276A5DF8044BD6
:10A8800020EE260A70475378A3F13001C8B2092898
:10A8900002F10102AAD8F2EE046AF0EE665A07EE5F
:10A8A000901AF8EEE77A12F8013F87EEA66AA3F154
:10A8B0003001C8B2092866EEA56A37EE067AEED9ED
:10A8C00094E767EE276AD9E7901C91780124A7E7FF
:10A8D000F7EE007ACFE7F7EE007AC5E70000000058
:10A8E00020BCBE4CB5EEC00ADFED317AF1EE10FAB5
:10A8F000CCBF30EE270A30EE670ADFED2E7A20EE6D
:10A90000270A30B5FDEEC07A87B017EE904A0546AB
:10A9100084EAE470002303A9A0EBE47001930093A0
:10A9200002932AF051FE002CACBF20232D2303A854
:10A930008DF8003035F0FEF8012803A924D0022854
:10A940002DD0032805BF3023684668468DF80130B6
:10A9500038F0B5FB684635F0EDF80338C4B222464E
:10A960006946284638F009FC00232B55284635F067
:10A97000E1F82E22431C2A540DEB0401E81838F0AC
:10A98000BBFB284607B030BD302368468DF8013048
:10A990008DF802308DF8033038F091FBDAE7302380
:10A9A00068468DF801308DF8023038F088FBD1E729
:10A9B0006F12033A00007A442DE9F041064615462D
:10A9C0000846B6FBF2F43CB905FB1464124B1B5D60
:10A9D00000F8013BBDE8F081B4FBF2F767B90E4B1C
:10A9E00005FB174705FB1464DA5D00F8012B1B5DBE
:10A9F00000F8013BBDE8F081B7FBF2F8B8F1000FB9
:10AA000002D04046FFF7D8FF05FB1878024B13F839
:10AA1000082000F8012BE3E7EC66040830B4026874
:10AA20001146531C036011F8024B0160D31C51788E
:10AA300003609378151D05601B0443EA0123D07859
:10AA4000234343EA006030BC704700BF0368591CD1
:10AA50001A46016012F8021B0260587841EA002091
:10AA6000704700BF03685A1C02601878704700BF27
:10AA700038B504460068154635F0E4FF22682A44DC
:10AA8000226038BD036810B40A0E5C1C04601A70A2
:10AA900003680A0C5C1C04601A7003680A0A5C1CD8
:10AAA00004601A7003685A1C026019705DF8044B48
:10AAB000704700BF036810B40A0A5C1C04601A7077
:10AAC00003685A1C026019705DF8044B704700BFA0
:10AAD00003685A1C026010B4197003680A0A5C1CEF
:10AAE00004601A7003680A0C5C1C04601A70036826
:10AAF000090E5A1C026019705DF8044B704700BFC4
:10AB000003685A1C026019700368090A5A1C026023
:10AB1000197070472DE9F047002488B080460F4631
:10AB20001E46A14605AD531C0393117839B3252960
:10AB300033D1931CCDF810900393507830284ED029
:10AB40004FF0000AA0F13003DBB2092B42D96C2888
:10AB500019D0642800F0938024D825281CD063D90C
:10AB6000582876D063281BD131784046B847039ADD
:10AB7000531C03931178043601340029D7D12046A1
:10AB800008B0BDE8F087039B5A1C03921B78642B26
:10AB90007CD02AD8252B54D1252140460134B847F2
:10ABA000039AC0E7732833D044D975284FD106F1F2
:10ABB000040E30682B4600220A217646FDF710FC71
:10ABC000049A0095534639464046FDF747FC039AE0
:10ABD0000444A8E704AA03A928F0EEFEB7E7D31CB3
:10ABE000039390784FF0010AACE7732B10D05BD938
:10ABF000752B3AD0782B96D1A3F15802B2FA82F293
:10AC0000306852092B4610210436FDF7E9FBD7E7DF
:10AC10003368049A0093394600234046FDF71EFC32
:10AC200004360444039A7EE70028B9D1204608B0D0
:10AC3000BDE8F0876E28B3D1039A336804361C60F0
:10AC400071E72AD9582BD7D0632B8DD06BE77828A2
:10AC5000A6D1A0F15802B2FA82F2306852092B460E
:10AC60001021FDF7BDFB0436AAE706F1040E30689B
:10AC70002B4600220A217646FDF7B2FBA0E7331DE2
:10AC8000306829461E46FDF77DFB99E7331D306885
:10AC900029461E46FDF776FB92E7002B7FF443AF73
:10ACA000204608B0BDE8F0876E2BC6D03BE700BF5A
:10ACB0000EB400B584B005AB019053F8042B0649DF
:10ACC000039301A8FFF726FF019B00221A7004B02E
:10ACD0005DF804EB03B07047518400080FB430B541
:10ACE00083B006AB0A490B4853F8042B0968006887
:10ACF0000193FFF70FFF084C05462068FEF78EFB17
:10AD00000028FAD0284603B0BDE8304004B07047B0
:10AD100084450020884500204CC40020DFED2B7ABC
:10AD2000B4EEE70AF1EE10FA4ADDDFED296A9FED95
:10AD3000297A01E0B0EE670AB4EEC70AF1EE10FA24
:10AD400070EE667AF6DC9FED247AF4EEC77AF1EEC7
:10AD500010FA38D5DFED1E6A9FED207A01E0F0EEA3
:10AD6000407AF4EEC77AF1EE10FA37EEA60AF6D47E
:10AD7000DFED1B7AB4EEE70AF1EE10FA14DDDFED39
:10AD8000137A37EEC00A60EE006A9FED166A9FEDF7
:10AD9000167ADFED167AA6EE867A20EE266AE6EEC1
:10ADA000877AA6EE270A7047DFED117AB4EEE70A3C
:10ADB000F1EE10FA44BFDFED087A37EEC00AE2E7A1
:10ADC000F0EE407ABFE7B0EE670AD1E7DB0F49400B
:10ADD000DB0FC940E4CB1641DB0F49C0E4CB16C101
:10ADE000DB0FC93F92E741B99730083C15A82ABE4E
:10ADF000DB0FC9BF80EAE073A3EBE0738B4205DB96
:10AE0000002801DD401A704702D1704700207047CA
:10AE10000844704709B909E0194690FBF1F301FBBA
:10AE200013030846002BF7D1084670470146FBE79D
:10AE3000F0EEC07AB0EEE07AB4EEE77AF1EE10FA16
:10AE4000B4BFB0EE676AB0EE476AB5EE406AF1EEA5
:10AE500010FA46D0B4EEE77AF1EE10FA8CBFF0EEBD
:10AE6000675AF0EE475AC5EE866A9FED1F3A9FED8E
:10AE70001F6A9FED1F4A9FED1F5ADFED1F3ADFED5E
:10AE80001F4ADFED1F5AA6EEC36AE6EEA34AA6EEFE
:10AE9000864AB7EE006AA6EE845AA6EEA46AE6EEEB
:10AEA000855AC5EE866AB4EEE77AF1EE10FA48BF2D
:10AEB000DFED147AF5EEC00A48BF77EEE66AF1EEF0
:10AEC00010FA48BFDFED107AB5EEC00A48BF77EE42
:10AED000E66AF1EE10FA48BFF1EE666AB0EE660A75
:10AEE0007047DFED076ADEE739094E3DE3B59E3E68
:10AEF00088FA163E45FE7F3F99FB243F69A2163E25
:10AF0000A7DFA834DB0FC93FDB0F4940DFED317A03
:10AF100030EE277AFDEEC76A16EE903A2033402BCA
:10AF200002D99FED2D0A7047B4EEE70AF1EE10FA50
:10AF30004DDD9FED2A6ADFED2A6A01E0B0EE677A07
:10AF4000B4EEE67AF1EE10FA77EE467AF6DC9FED93
:10AF5000257AF4EEC77AF1EE10FA35D5DFED1F6AE7
:10AF60009FED217A01E0F0EE407AF4EEC77AF1EE3F
:10AF700010FA37EEA60AF6D4DFED167AB4EEE70A39
:10AF8000F1EE10FA1BDCDFED197AB4EEE70AF1EE10
:10AF900010FA44BFDFED137A37EEC00A60EE006AA4
:10AFA0009FED136A9FED137ADFED137AA6EE867A92
:10AFB00020EE266AE6EE877AA6EE270A7047DFEDD6
:10AFC0000F7A37EEC00AE9E7B0EE670AD4E7F0EE91
:10AFD000477ABCE7DB0FC93F00000000DB0FC94028
:10AFE000E4CB1641DB0F49C0E4CB16C1DB0FC9BF70
:10AFF00092E741B99730083C15A82ABEDB0F4940BB
:10B00000FDEEC07A17EE903A2033402B51D8DFED99
:10B010002D7AB4EEE70AF1EE10FA50DDDFED2A6A80
:10B020009FED2A7A01E0B0EE670AB4EEC70AF1EEAE
:10B0300010FA70EE667AF6DC9FED257AF4EEC77AA8
:10B04000F1EE10FA38D5DFED206A9FED227A01E0AB
:10B05000F0EE407AF4EEC77AF1EE10FA37EEA60A77
:10B06000F6D4DFED1D7AB4EEE70AF1EE10FA1BDC40
:10B07000DFED1A7AB4EEE70AF1EE10FA44BFDFED25
:10B08000147A37EEC00A60EE006A9FED156A9FEDF4
:10B09000157ADFED157AA6EE867A20EE266AE6EEC0
:10B0A000877AA6EE270A7047DFED067A37EEC00AE8
:10B0B000E9E79FED0E0A7047B0EE670AD1E7F0EEC0
:10B0C000407AB9E7DB0F4940DB0FC940E4CB1641BA
:10B0D000DB0F49C0E4CB16C1DB0FC93FDB0FC9BF93
:10B0E00092E741B99730083C15A82ABE000000003D
:10B0F00010B507EE901A2DED028BB8EE678ADFEDE2
:10B10000217A28EE008A044628EE278AB0EE480A03
:10B1100035F0EEFEF0EE408AB0EE480A35F04AFE19
:10B12000F7EE007A9FED187AF0EE675AE8EE875A4C
:10B130000023A361B0EE676AC7EEA56A636123626C
:10B14000E361A8EEC76ABDEC028B77EEC07AB6EE7B
:10B15000007AF8EE005A27EE877A20EE250A27EECD
:10B16000267A26EE266A67EEA67A20EE260A84ED77
:10B17000046AC4ED017A84ED007A84ED027A84EDEC
:10B18000030A10BD27D4D236F304353F10B44C095E
:10B19000012250F8243001F01F0102FA01F10B43A3
:10B1A00040F824305DF8044B704700BF4B0901F0B4
:10B1B0001F0150F82320012303FA01F1114214BFAB
:10B1C00018460020704700BF70B40749074E084D6D
:10B1D000084A01230020202488714B7170716B7222
:10B1E0001485138170BC7047106F002080B9002057
:10B1F000909800205891002010B5802104460848FE
:10B20000FEF75EFF44F6BD7344F27D00002C18BFCC
:10B210001846400140F01700BDE81040FEF71CBF83
:10B22000003C004038B504460D460C488021FEF72E
:10B2300047FF43F21020FEF70FFF042CA8BF0424A1
:10B24000E100074C072DD4BF4919073104EB8101F8
:10B25000BDE83840486CFEF7FFBE00BF003C004030
:10B26000DC3104080C4B984213D0A3F5806398425C
:10B270000FD003F5804398420BD003F580639842CA
:10B2800007D003F58063984203D0044B1868400848
:10B290007047024B1868704700040140D0980020A6
:10B2A000F0B5774B774A87B01968914200AF00F04C
:10B2B000DB800023744A3B607B60136843F4803377
:10B2C000136003E03B68B3F5A04F09D0136803F4A3
:10B2D00000337B603B6801333B607B68002BF1D01F
:10B2E000694B1B6813F4003318BF01237B607B6834
:10B2F000012B7BD0654D644B654AEA606549586F08
:10B30000654A0860AA605E6B644C654A654826F031
:10B3100080065E635E6F46F080765E67196B0C4355
:10B320001C63596B5963996B9963196C41F05B51BC
:10B3300041F47B1141F41F6141F00F011964596C14
:10B3400007F118040A4348F2FF715A6444F8101DCB
:10B35000002621460123FB733E737E73BE7330F0DB
:10B3600065FE21464FF6FF734F48BB6030F05EFE2E
:10B370004FF6FF7321464D48BB6030F057FE214623
:10B380004B4830F053FE21464A4830F04FFE2146EC
:10B39000494830F04BFE2146484830F047FE2146F0
:10B3A000474830F043FE2146464830F03FFE2046F5
:10B3B00031F01CF8444B454C1B68BA684448454979
:10B3C000A4FB03439B09A0FB0202013B920CB3F1D7
:10B3D000807F0A6007D2404AF0200721536085F839
:10B3E0002300966011601C37BD46F0BD264B3B4DD7
:10B3F0001A6C3B4842F080521A642C68426881689B
:10B4000044F440442C609C689C609C6844F4004474
:10B410009C609C6844F4A0549C600068120642EA58
:10B42000801242F48002490842F00802013942EADF
:10B4300001425A601A6842F080721A601A689201DA
:10B44000FCD52849104A40F205700860996821F03F
:10B4500003019960996841F002019960936803F0D3
:10B460000C03082BFAD145E700221A6062B61E4B86
:10B470001B6883F308881D4B1B689847FEE700BFD5
:10B48000FCFF0120EFBEADDE0038024000ED00E021
:10B490000005FA05BC98002000000008FF91670035
:10B4A000335F070000000240000402400008024031
:10B4B000000C02400010024000140240001802403C
:10B4C000001C024000200240D0980020D34D6210A2
:10B4D00083DE1B43B8D0002010E000E00070004085
:10B4E00000000020003C02400000FF1F0400FF1F7E
:10B4F00008B5054B1B6803B19847044B044A1A6012
:10B5000072B6FDF7C3FA00BF204C0020FCFF0120FB
:10B51000EFBEADDE08B5034B1B6803B1984772B6AA
:10B52000FDF7B4FA204C0020084B10B507281B6823
:10B53000C8BF143818440C46007DFEF72FF920B11F
:10B540002146BDE81040FEF77FBB10BDD07F002034
:10B5500030B50446406D61718389A26823F40053BD
:10B560001B041B0C838185B0A379009213F00402A5
:10B5700030D04FF4805213F00203ADF8042063D1B1
:10B58000ADF806304FF480630022ADF8083011F0BA
:10B590000103ADF80C2028D1ADF80A3008238D073F
:10B5A000694648BFADF80A3023F0F8FDA279636D13
:10B5B000D10724D412F0080F9A8A1BD122F0080276
:10B5C0001204120C9A829A8992B242F400529A8121
:10B5D00005B030BD13F00203ADF8042031D04FF4B4
:10B5E00000551346ADF80650CEE70423ADF80A30F7
:10B5F0000C23D4E792B242F008029A82E3E714499E
:10B600008B421CD0A1F54C418B4216D001F58061D4
:10B610008B4210D001F580618B420AD001F5806128
:10B620008B42C7D104200121FFF77EFFA279636D11
:10B63000C0E70320F7E70220F5E70120F3E7002049
:10B64000F1E7ADF806309FE74FF4005398E700BFED
:10B650000010014010B50446406DA160838923F4B9
:10B6600000531B041B0C8381A37984B013F00402E4
:10B67000009135D04FF4805213F00203ADF804204E
:10B6800063D1ADF806304FF480636279ADF80830CD
:10B69000D1074FF00003ADF80A30ADF80C3045BFCC
:10B6A0000423ADF80A3008230C236946920748BFEB
:10B6B000ADF80A3023F072FDA279636DD1071FD473
:10B6C00012F0080F9A8A16D122F008021204120C06
:10B6D0009A829A8992B242F400529A8104B010BDC3
:10B6E00013F00203ADF804202CD04FF400511346A0
:10B6F000ADF80610C9E792B242F008029A82E8E774
:10B7000013498B421CD0A1F54C418B4216D001F558
:10B7100080618B4210D001F580618B420AD001F527
:10B7200080618B42CCD104200121FFF7FDFEA2797C
:10B73000636DC5E70320F7E70220F5E70120F3E793
:10B740000020F1E7ADF806309FE74FF4005398E78B
:10B750000010014038B50D4B07281B68CCBFA0F185
:10B760001404044623440546187DFEF717F858B123
:10B7700001342722C47182710121FEF7A1F9284604
:10B780000021BDE83840CFE638BD00BFD07F0020A3
:10B79000064A00235168814202F11C0204D00133A1
:10B7A000102BF7D100207047D8B27047200100203D
:10B7B00070B50F4C0F4DC0EBC00004EB8004286B3C
:10B7C00026693043286382B09209667BA160002518
:10B7D000012101A863618DF804608DF805208DF8C2
:10B7E00006508DF8071023F0A1FC02B070BD00BF19
:10B7F0002001002000380240074BC0EBC00030B4ED
:10B8000003EB8000054C0569236B2B432363017612
:10B81000427630BC704700BF200100200038024053
:10B820002DE9F04F534C54F8204083B0002C00F029
:10B830009C80E56D002D00F09A8017464E4A984690
:10B84000064604F162032869226004F26222636101
:10B85000A2614FF400736A68A160E36023616265CE
:10B86000A24668B1FFF794FF721CD2B20C21FFF719
:10B87000C3FF636DA9682A6922630433A16323654A
:10B88000E868A0B1FFF784FF721C8146D2B20B2199
:10B89000FFF7B2FF2346EA7F38494846FFF788FFA3
:10B8A000636DA968EA6862630433E163E36494F852
:10B8B0006100FDF773FF814694F86000FDF76EFFAD
:10B8C0008346287F00284DD118F0080F36D1BA07DB
:10B8D0000DD5B9F1000F0AD00B22731C89F8062090
:10B8E00089F8073048466A7F2221FEF71DF8FB07DA
:10B8F00015D4A36B7BB995F82020A97F8DF806306D
:10B9000001A8930901228DF805308DF804108DF8F7
:10B91000072023F00BFC504603B0BDE8F08FBBF1CD
:10B92000000FE6D001360C238BF807608BF8063049
:10B9300058466A7F2221FDF7F7FFDAE70136F6B2B3
:10B94000B9F1000F04D00B2389F8076089F806309D
:10B9500018F0100F484614BF022112216A7FFDF72C
:10B96000E3FFC6E733F0B2F8AEE7A246D3E7AA4654
:10B97000D1E700BF90450020C0320408B18A00081A
:10B980000348D0F8AC3113B100F5D27018477047B6
:10B99000200100200348D0F8903113B100F5C470A5
:10B9A00018477047200100200348D0F8743113B1C4
:10B9B00000F5B67018477047200100200348D0F802
:10B9C000583113B100F5A8701847704720010020C6
:10B9D0000348D0F83C3113B100F59A70184770470E
:10B9E000200100200348D0F8203113B100F58C70FD
:10B9F00018477047200100200348D0F804310BB1EC
:10BA0000FC301847704700BF200100200348D0F8E1
:10BA1000E8300BB1E0301847704700BF200100202C
:10BA20000348D0F8CC300BB1C4301847704700BF82
:10BA3000200100200348D0F8B0300BB1A8301847DF
:10BA4000704700BF200100200348D0F894300BB1AC
:10BA50008C301847704700BF200100200248836FD8
:10BA60000BB1703018477047200100200248C36DA9
:10BA70000BB1543018477047200100200248036C76
:10BA80000BB1383018477047200100200248436A44
:10BA90000BB11C3018477047200100200248836812
:10BAA00003B11847704700BF20010020431C00F07D
:10BAB00014812DE9F04F4FEAC00808EB00039B000A
:10BAC000DFF8F4A25AF803B087B00AEB0304BBF125
:10BAD000000F00F0FF8014330AEB03010022DBF8B3
:10BAE00004704AF803204A608A60CA600346A56869
:10BAF00001900133D4F80C90DBB2002D00F0EE8001
:10BB00001522EB71AA71B9F1000F00F00081162225
:10BB100089F8062089F807309BF80E0032F0D6FF2E
:10BB2000BB8823F440731B041B0CBB802846FEF724
:10BB300085F84846FEF782F811212846FDF778FD82
:10BB400011214846FDF774FD0826642404E00A200C
:10BB50003CB103F089F9013C2846FEF797F800282C
:10BB6000F5D02846FEF764F80A2003F07DF9284650
:10BB7000FEF764F80A2003F077F9013EECD148465D
:10BB8000FEF756F80A2003F06FF92846FEF750F842
:10BB90000A2003F069F92846FEF750F80A2003F05E
:10BBA00063F94846FEF74AF8019B08EB03040AEBE9
:10BBB00084042846637C002B0CBF1221322104220E
:10BBC000FDF7B2FE637C002B0CBF122132214846E8
:10BBD0000422FDF7A9FE704B9F4200F0B7806F4B27
:10BBE0009F4200F0BD806E4B9F4200F0A580BB8855
:10BBF00001996C4A6C4C23F440731B041B0CBB80F2
:10BC00003B8888440AEB880A9BB243F001039AF808
:10BC100010103B80BD8802A8002918BF144630F0E0
:10BC2000E5FB049A6148B2FBF4F325F03F05A0FB65
:10BC300002122D04900C2D0C0543BD805C4C3988FC
:10BC40004FF4967202FB00F284FB02409BB2D217C3
:10BC5000002BC2EBA01221F0010108BF012309044F
:10BC6000013243F40043090C92B239803A84BB8319
:10BC70003B889BB243F001033B803B8823F4816304
:10BC800023F002031B041B0C43F480634FF4804237
:10BC90003B803A813B8823F080031B041B0C3B80D4
:10BCA0009BF810308DF808300024012302A88DF88D
:10BCB0000B308DF809408DF80A4023F037FA9BF8D5
:10BCC0000F308DF8083002A88DF809408DF80A4031
:10BCD00023F052FA07B0BDE8F08F7047B9F1000FBA
:10BCE00048D0162289F8073089F806209BF80E0004
:10BCF00032F0ECFEBB8823F440731B041B0C284677
:10BD0000BB80FDF79BFF4846FDF798FF18E79BF8BF
:10BD10000E0032F0DBFEBB8823F440731B041B0CC7
:10BD2000BB802846FDF78AFF4846FDF787FF1121B3
:10BD30002846FDF77DFC07E71E4A136A43F400031B
:10BD400013624FF4000030F09BFA50E7194A136A6F
:10BD500043F4001313624FF4001030F091FA46E7F9
:10BD6000144A136A43F4800313624FF4800030F0E6
:10BD700087FA3CE79BF80E0032F0A8FEBB8823F45C
:10BD800040731B041B0C4846BB80FDF757FF484619
:10BD9000FDF754FFD8E600BF0054004000580040B3
:10BDA000005C0040009F2400804F120083DE1B4394
:10BDB000D34D621000380240B8450020F8B54FEA74
:10BDC000C00E274F069C0EEB000507EB85056E683D
:10BDD000002E42D04900C9B2A9754FF0000C0121D4
:10BDE000EA7585F819C0A9762B76697585F814C0AF
:10BDF000B3882C629905EC6114D43388DA050CD42D
:10BE00004FF4805401E0013C1ED033889B05FAD4E6
:10BE100033889BB243F480733380B3889BB243F47E
:10BE20004073B3800EEB000107EB81024FF48054A6
:10BE300001E0013C08D0537D002BFAD107EB8107CC
:10BE40003C7D84F00100F8BD064A138801339BB2A3
:10BE50001380FFF72BFE2046F8BD3046F8BD00BF2B
:10BE6000B8450020A447002070B590F904506C1C20
:10BE700082B00AD0032D08DC16460A4641790096A6
:10BE80002846FFF79BFF02B070BD002002B070BDD6
:10BE900000B50378012B83B004D1032301AA00214C
:10BEA000FFF7E2FF9DF805309DF804209DF806009D
:10BEB0001B0243EA0243184303B05DF804FB00BFD2
:10BEC00008B5FFF7E5FF014B586008BD6426002068
:10BED00008B5FFF7DDFF014B186008BD64260020A0
:10BEE00070B50378012B82B004D106236A46F7218E
:10BEF000FFF7BAFF9DF801209DF804309DF800601F
:10BF00009DF803509DF802409DF805000749120175
:10BF10001B0142EA063243EA053342EA141243EABD
:10BF20001013CA608B6002B070BD00BF6426002091
:10BF3000F0B585B002AB04460093032206231E2110
:10BF40000020FFF73BFF00283CD09DF808509DF8EB
:10BF500009109DF80A709DF80B209DF80C609DF863
:10BF60000D3041EA052142EA072243EA062309B2DD
:10BF700012B21BB2144D06EE901A07EE102A07EE0D
:10BF8000903AF8EEE66A95ED035AD5ED055A95ED2F
:10BF9000046AB8EEC77AF8EEE77A66EE856A27EEAD
:10BFA000257A67EE867AFDEEE66ABDEEC77AFDEE8B
:10BFB000E77A16EE901A17EE102A17EE903A2180C3
:10BFC000A280638005B0F0BD0000002000B583B002
:10BFD000002000920A466821FFF7F0FE03B05DF8EA
:10BFE00004FB00BFF0B5C60033189B00254DEA588E
:10BFF0005468A28A83B092B20192019A2B4412F43F
:10C00000706F1CBF01221A75019B13F4E06F074685
:10C010000CD1A38A3E4423F4706305EB86051B0410
:10C020001B0C0022A3826A7503B0F0BD238BA3888A
:10C0300023F480631B041B0CA380019B9B05E8D4A5
:10C0400023889805E5D42388D9050ED52388DA05F9
:10C05000FCD423889BB243F40073238023889B0580
:10C06000FCD43846FFF722FDD3E723889BB243F484
:10C0700000732380A38823F440731B041B0CA3804C
:10C08000C7E700BFB8450020F0B583B0441C8DF869
:10C09000073001D0032802DD002003B0F0BDC70047
:10C0A000244E3B1806EB83035D68002DF4D0490055
:10C0B000C9B2997501240021DA755C7699761C76EF
:10C0C0005C751975A9880DF107028905DA611A6294
:10C0D00014D42B88DA050CD44FF4805401E0013CD1
:10C0E0001ED02B889B05FAD42B889BB243F4807317
:10C0F0002B80AB889BB243F44073AB80074406EBC4
:10C1000087024FF4805401E0013C09D0537D002B9D
:10C11000FAD106EB87073C7D84F0010003B0F0BD47
:10C12000054A138801339BB21380FFF7BFFC2046FA
:10C13000B3E700BFB8450020A447002010B4044670
:10C14000134690F904000A4661795DF8044B9BE7B9
:10C150000278012A00D070474821EFE70278012ACF
:10C1600000D070475821E9E70378012B00D07047D1
:10C170003122F421E2E700BF2DE9F043322083B001
:10C1800002F0CCFE0022104611231E21FFF77CFF97
:10C19000602301221E210020FFF776FF642002F0B9
:10C1A000BDFE6846FFF7C4FE0024DFF88C812546FB
:10C1B00026460A27012302221E210020FFF764FFE2
:10C1C000322002F0ABFE6846FFF7B2FEBDF902E096
:10C1D000BDF90410BDF900208E457346A8BF0B467B
:10C1E0009342A8BF134643454FF0010075440C44E9
:10C1F0001644C0F29180FDF73FF9013FDAD14FF0CC
:10C2000001090022104612231E21FFF73DFFDFF82F
:10C2100028810A27012302221E210020FFF734FF74
:10C22000322002F07BFE6846FFF782FEBDF902E095
:10C23000BDF90410BDF900208E457346A8BF0B461A
:10C240009342A8BF134643454FF00100A5EB0E05EE
:10C25000A4EB0104A6EB02065BDBFDF70DF9013F41
:10C26000D8D107EE906AF8EEE76A07EE905AB8EE7A
:10C27000E77A07EE904ADFED2A5A9FED2A5A2A4EB6
:10C28000F8EEE77A85EEA66A0022104670231E219A
:10C29000C5EE876A85EE277AB0EEC66AF0EEE66AEA
:10C2A000F0EEC77A86ED036AC6ED046AC6ED057A3C
:10C2B000FFF7EAFE202301221E210020FFF7E4FE03
:10C2C0000023184602221E21FFF7DEFE642002F042
:10C2D00025FEB9F1000F04D14FF07E53F3603361B6
:10C2E0007361124C206810B1FDF7D0FC18B9012021
:10C2F00003B0BDE8F0830E490E4B41F8143F2068AF
:10C3000032F0CCFF206832F0B7FF012003B0BDE867
:10C31000F0834FF00009A4E74FF0000971E700BF78
:10C3200000406F4601C05E460000002074500020AF
:10C33000642600202D86000801F0FFFFF0B587B0CD
:10C340000DF10F0305460093022201230C2100206A
:10C35000FFF734FD18B19DF80F30DB0703D400243C
:10C36000204607B0F0BD04AB0093032206230C2146
:10C370000020FFF723FD0DF10F0300930922012395
:10C380000C210020FFF71AFD04460028E7D09DF895
:10C390000F0010F00C00E2D19DF811E09DF8101094
:10C3A0009DF813709DF812209DF815609DF81430CB
:10C3B00041EA0E2142EA072243EA0623C1EB81311A
:10C3C000C2EB8232C3EB8333890092009B00298049
:10C3D0006A80AB800A2201230C21FFF755FEBFE7DC
:10C3E00010B5002384B018460A220C21FFF74CFE3A
:10C3F000142002F093FD0F230A220C210020FFF7E6
:10C4000043FE0A2002F08AFD03AB009310220323AF
:10C410000C210020FFF7D2FC0A2002F07FFD002350
:10C4200018460A220C21FFF72FFE0DF10B040A20FB
:10C4300002F074FD0094012302220C210020FFF77A
:10C44000BDFC0094012309220C210020FFF7B6FC5B
:10C4500001230A220C210020FFF716FE012004B060
:10C4600010BD00BF134600200A4668210CE600BF3D
:10C470000220FCF7F9BB00BF0220B3E50120FCF766
:10C48000F3BB00BF0120ADE50020FCF7EDBB00BF12
:10C490000020A7E51549164B16480A6810B48C68A9
:10C4A0001549B2FBF4F203FB02F30360D1F88820D4
:10C4B000124B134C42F47002C1F888201A68002015
:10C4C00042F001021A6098601A6822F0847222F425
:10C4D00080321A605C601A684FF0006422F4802297
:10C4E0001A60D8608C605DF8044B70470000002033
:10C4F00040420F00D098002000ED00E000380240DC
:10C5000010300024044B4FF4F0700A21022283E81B
:10C510000700FFF7BFBF00BF0000002038B50B4C7D
:10C5200023688BB15A68821A002A054604DA0CE0A7
:10C530005A68AA1A002A07DB9A68226018461A6805
:10C5400090472368002BF3D138BD38BD544A0020F2
:10C550000B4B002210B4027203F5B474032102E005
:10C56000072A09DC9979890702D5197981540132A2
:10C570009C4203F11803F3D15DF8044B704700BFF0
:10C58000905A040813230370704700BF012310B4AE
:10C5900032213124302244704171C2700370037122
:10C5A00083705DF8044B70472DE9F0410B78047BF4
:10C5B000DB43DEB200F1100200F1380342F8044F11
:10C5C0009342FBD1DFF89CC000F16001002243F8E8
:10C5D000042F8B42FBD14FF0140E0521002546FAA3
:10C5E00001F303F00103002B1D4414BF4FF01908A1
:10C5F0004FF00A0811F0010FEDB214BF27460027D3
:10C6000000220EEB02039BB200EB83030132424592
:10C610005F61F6D1013A92B2013201390EEB0203A9
:10C620004A1C9BB201D09E46D9E715F0010F14BFFA
:10C6300019250A2500215A1892B200EB8202013115
:10C64000A9425461F7D10B449BB21A1D00EB820240
:10C65000013300219BB25160ACF800300361BDE8AA
:10C66000F08100BF84260020254B5B880B332DE929
:10C67000F04F8A4601F1060B1FFA83F94FF00108CB
:10C68000002100271AF801EB3E464C460122A4F196
:10C690000B039BB207E001339BB2B0F80CC0C5F8A6
:10C6A00014C09C420AD000EB8305002AF3D100EBB2
:10C6B000830501339BB29C426A61F4D1231D00EBD8
:10C6C00083030136092FF6B259600CD0092E14D01D
:10C6D00008FA07F313EA0E0F14BF012200220C34EC
:10C6E000A4B20137D3E709F17809DA451FFA89F9CD
:10C6F000C7D1034B5980BDE8F08F0022EFE700BFA0
:10C70000842600202DE9F047DFF85C80B8F804307B
:10C7100004338A461FFA83FC01F109094FF0010E28
:10C720001AF8017B64460026231F0EFA06F29BB21C
:10C730003A40BAB1818900EB830501339BB29C4238
:10C740006961F6D101360434082EA4B2ECD10CF1A3
:10C75000200CCA451FFA8CFCE2D10023A8F8043053
:10C76000BDE8F0871146E6E78426002010B4037B7D
:10C7700001681F2B09D9203B20224C6802FA03F3E1
:10C780001C4214D15DF8044B704720220C6802FA59
:10C7900003F31C42F6D00C4A40680024147002686F
:10C7A0005DF8044B22F0010202608B607047064A7C
:10C7B00040680024147002685DF8044B22F0010206
:10C7C0000260CB60704700BFE885002008B520F00C
:10C7D0001BF8FEF79FFE00BF024A034B1278197840
:10C7E0001BF0B6BC6029002061290020038A2DE9D6
:10C7F000F0478589ADB21D4029D00F4606464FF05F
:10C8000000484FF00009B5FA85F328FA03F2D24345
:10C8100091B21B3B15403182042B16D8DFE803F0A0
:10C820003129211903007B6A002B32D003F1FF3A32
:10C830001FFA8AFAC7F824903C6A34B1236820466C
:10C84000514698476468002CF8D1002DDBD1BDE833
:10C85000F0873868716B036889B29847002DD2D190
:10C86000F5E77868B16B036889B29847002DCAD1A3
:10C87000EDE7B868F16B036889B29847002DC2D123
:10C88000E5E7F868316C036889B29847002DBAD1A2
:10C89000DDE7F36A1FFA83FACEE700BF2DE9F04F18
:10C8A0002DED028BA0F10A0389B00C46E72B00F2B4
:10C8B0002C87DFE813F01C012A072A072A072A071A
:10C8C0002A072A072A072A072A072A072A072A07E0
:10C8D0002A072A072A072A072A072A072A072A07D0
:10C8E0002A072A072A0780012A072A072A0771012F
:10C8F0002A072A072A0764012A076F022A072C023F
:10C900002A0721022A0719022A07F4012A07E0014F
:10C910002A072A072A07DA01D3012A07CB052A07A3
:10C920002A07C3052A07D3052A072A072A074B0324
:10C930002A072A072A072A07E4022A07FC002A07EF
:10C94000260303032A072A072A072A072A072A0792
:10C950002A07D3062A0786062A0751062A07FC0556
:10C960002A0715072A072A072A072A07A0056505A7
:10C970003105B302E800F404E0041905D4042A07E1
:10C980009D0481042A072A072A072A0776042A0712
:10C990002A0755042A072A072A0746042F041B04DE
:10C9A000D9032A072A072A07A4038D037E035E03FF
:10C9B0002A072A072A072A072A072A072A072A07EF
:10C9C0002A072A072A072A072A072A072A07A0056B
:10C9D0002A072A072A072A072A072A072A072A07CF
:10C9E0002A072A072A072A072A072D012A072A07C2
:10C9F0002A072A072A072A072A072A072A072A07AF
:10CA00002A072A072A072A072A072A072A072A079E
:10CA10002A072A072A072A072A072A072A072A078E
:10CA20002A072A072A072A072A072A072A072A077E
:10CA30002A072A072A072A072A072A072A072A076E
:10CA40002A072A072A072A072A072A072A072A075E
:10CA50002A072A072A072A072A072A072A072A074E
:10CA60002A072A072A072A072A072A072A072A073E
:10CA70002A072A072A072A072A072A072A072A072E
:10CA80002A079E01A901AE4E337853B1AD4F002560
:10CA900037F8021F2046FEF733F833780135AB42F2
:10CAA000F6DC012009B0BDEC028BBDE8F08FA44E8E
:10CAB0003378002BF5D0A44F0025B846236817F82B
:10CAC0001520591C21601A7098F8011001EB8101A2
:10CAD00001EB810101F2EE2189B22046FEF710F848
:10CAE00033780135AB4208F10208E7DCD9E7974D0E
:10CAF000284633F01FF80028D3DD2B460544226872
:10CB000013F8011B501C9D4220601170F7D1C8E73B
:10CB10000B68DFF87CC2591C9CF8002021601A7059
:10CB20009CF80030002BBCD0894E8A4D8A488B4936
:10CB30000023226816F8017F02F1010EC4F800E01C
:10CB40001770226815F8017F02F1010EC4F800E0A9
:10CB50001770226810F8017F02F1010EC4F800E09E
:10CB60001770226811F8017F02F1010EC4F800E08D
:10CB700017709CF8002001339A42DADC91E70B68C9
:10CB8000774A581C11782060197023685278591C14
:10CB9000216001201A7085E7724D08462988FDF74B
:10CBA000AFFFA9882046FDF7ABFF20462989FDF796
:10CBB000A7FF012076E76C4D05F15006287831F08B
:10CBC000D9F82368027A591C21601A7023686A78A0
:10CBD000591C21601A702368AA78591C21601A70A8
:10CBE0002368EA780435591CAE4221601A70E5D1F9
:10CBF00057E75E4D0846E989FDF782FF2046A9897F
:10CC0000FDF77EFF01204DE7594B03F170052268C7
:10CC10001978501C2060117022685978501C2060CF
:10CC2000117022689978501C206011702268D978A0
:10CC3000501C2060117022681979501C20601170FE
:10CC400022685979501C2060117022689979073345
:10CC5000501C9D4220601170D9D122E70B6801223F
:10CC60009918216010461A701CE708460021FDF74C
:10CC70002FFF012016E73F4D3F4E05F1300795F994
:10CC800002103E4B93F906208A4203F1080300F09C
:10CC90003F859E42F6D10835BD42F0D101E7384BC1
:10CCA00003F15A0522685979501C206011702268DE
:10CCB0001978501C2060117022685978501C20602F
:10CCC000117022689978501C206011702268D97800
:10CCD000501C20601170226819790633501C9D4247
:10CCE00020601170DED1DCE60B68264A591C527DAB
:10CCF000216001201A70D5E6234D05F1800655F814
:10CD0000041F2046FDF7E4FEAE42F8D1C9E61F4DF0
:10CD100005F14006B5F880102046FDF7F1FE2368C6
:10CD200095F88220591C21601A70236895F8832099
:10CD30000435591CB54221601A70EBD1B1E600BF31
:10CD4000085800202EB50020F84B0020B0660020C7
:10CD5000175300202753002047530020375300204B
:10CD6000FC4F00203446002000500020544F00208B
:10CD7000CCBA0020589100208C9800205C980020AC
:10CD80007868002090980020486500204C650020BD
:10CD900015530020A14D0B682A7A591C21601A7086
:10CDA000A98B2046FDF7ACFE298B2046FDF7A8FE97
:10CDB000698B2046FDF7A4FE2368EA7C591C21609C
:10CDC0001A70A98C2046FDF79BFEE98C2046FDF7E2
:10CDD00097FE2368AA7F591C21601A70236895F872
:10CDE0002020591C21601A70698C2046FDF788FEAE
:10CDF0002368EA7A591C21601A70E9682046FDF719
:10CE000067FE23682A7C591C21601A70236895F8F4
:10CE10002120591C216001201A7043E6804D814E6B
:10CE20009FED818ADFF83C82DFED808A05F12007E3
:10CE30000EE0FCEEE77ACDED017ABDF80410204655
:10CE40000435FDF75DFEBD4206F118063FF429AE3C
:10CE5000717C0029F3D0764BD5ED007A1B78012B3D
:10CE6000E7D1744B1B68DB0440F11085F5EE407A86
:10CE7000F1EE10FA40F0428540F2DC51DFE70B683A
:10CE80006D4D591C2A7921601A7023686A79591CE2
:10CE900021601A7029882046FDF732FE2368AA799E
:10CEA000591C21601A7069882046FDF729FE236805
:10CEB000EA79591C216001201A70F3E50B685F4E76
:10CEC00001255A1C0A601D700B68B278591921603F
:10CED0001A7031F06DFA2368594A5A495F19276070
:10CEE0001870B1F90010B2F90000FDF793FF236844
:10CEF0005A192260187031882046FDF701FE284635
:10CF0000D0E50B68504D01269A190A601E702AF070
:10CF1000C5FC002840F0D1844C4B2268511C216094
:10CF20001070226841F2B410511C185C216041F26B
:10CF30007811107059582046890AFDF7C9FDA96A71
:10CF400020464908FDF7C4FD0120ABE50B6800252C
:10CF50005A1C0A6020461D702946FDF7B9FD294676
:10CF60002046FDF7B5FD20462946FDF7B1FD01201D
:10CF700098E50B68364F591C3A7821601A703B7857
:10CF8000002B3FF48EAD0025EEB2304622F0CCFEF1
:10CF900023684278591C216030461A7022F0C4FE82
:10CFA00001892046FDF7ACFD3B780135AB42EBDC57
:10CFB00077E5284B2849B3F9003081FB0321DB17C3
:10CFC000C3EBA101204689B2FDF79AFD012069E576
:10CFD0000A68224B501C1978206011702268597819
:10CFE000501C2060117022689978501C20601170CC
:10CFF0002268DB78511C21600120137052E5184D26
:10D000000846298AFDF77CFD698A2046FDF778FDF0
:10D010002046A98AFDF774FD012043E59098002081
:10D02000D44F00205C9200200000404200E0824487
:10D0300040930020709600206C6A00208CB700207E
:10D040003CC500203EC5002084B3002038A100204C
:10D05000056E0020644F002067666666FC52002063
:10D060001C930020DB9B9141DFF810E30027FEB208
:10D07000714600232268501C206016702268501CE4
:10D0800020601370226811F8010F0133551C062B24
:10D0900025601070EED10137062F0EF1060EE6D195
:10D0A000A14900232268501C206017702268501C80
:10D0B00020601370226811F8010F0133551C0B2BEF
:10D0C00025601070EED12368984A581C0721206013
:10D0D000197023680021581C20601970236892F889
:10D0E000F020591C216001201A70DBE40B68904A83
:10D0F00090491078904A5D1C2560187023688978E3
:10D10000581C2060197023689278591C21600120F6
:10D110001A70C7E40A68894B89491878551C25603C
:10D12000107022685878551C2560107022689B7812
:10D13000501C206013702046C988FDF7E1FC0120D7
:10D14000B0E47F4D08462988FDF7DAFC698820465F
:10D15000FDF7D6FC2046A988FDF7D2FC0120A1E40A
:10D16000784D05F16006A9882046FDF7C9FCE988DD
:10D170002046FDF7C5FC29892046FDF7C1FC236840
:10D18000AA7A591C21601A702368EA7A591C216016
:10D190001A7055F80C1B2046FDF79AFCAE42E2D1FE
:10D1A0007FE4694952232268501C2060137011F8F3
:10D1B000013F002BF7D174E464480023226805681E
:10D1C00003EB4301561C6D5C2660157002682568F0
:10D1D0000A446E1C527826602A70026825680A4448
:10D1E00001339278691C0A2B21602A70E6D158E439
:10D1F000574D0B682A68591C127821601A702B68E9
:10D2000022689978531C2360002311702A682168D2
:10D210001A4401335279481C032B20600A70F5D15F
:10D2200023682A68591C127A21601A7023682A68B8
:10D23000591CD27821601A7023682A68591C127907
:10D2400021601A702B6820465989FDF759FC2A681D
:10D250002368527A591C21601A702A6895E43D4B64
:10D2600008461968FDF734FC3B4B20461988FDF74A
:10D2700047FC012016E4394B08461988FDF740FCAD
:10D28000374B20461988FDF73BFC364B22681B784C
:10D29000511C03F0010321600120137002E4324BA2
:10D2A0000A681B78314D511C03F002032160137092
:10D2B00023682A7D591C21601A7029682046FDF7D1
:10D2C00007FC69682046FDF703FC29892046FDF725
:10D2D00017FCE9892046FDF713FC2046298AFDF753
:10D2E0000FFC0120FFF7DEBB214D08462988FDF722
:10D2F00007FC69882046FDF703FCB5F904301D4A98
:10D30000D91782FB0323C1EBA301204689B2FDF7A5
:10D31000F7FB0120FFF7C6BB084610221649FDF7B0
:10D32000A7FB0120FFF7BEBB2F6600204C65002045
:10D330004C960020544F0020644F00204C4F00209A
:10D34000506A0020F4C00020E8320408C8660020BB
:10D35000807F0020F8C30020ECC30020B0B700207D
:10D36000AE660020E45100201CC4002020C4002030
:10D37000FCC3002067666666C44F00200B66002071
:10D38000A74B9B8AB3F5006F00F29582B3F5806FCF
:10D3900000F2B282B3F5007F34BF01270227A14D0E
:10D3A00005F10C0655F8041B91FBF7F1204689B2F4
:10D3B000FDF7A6FBAE42F5D19B4D9C4F05F10C0647
:10D3C000B5EC010AD7ED087A80EE270A33F044FD68
:10D3D00081B22046FDF794FBAE42F1D1944D05F1A8
:10D3E0000C0655F8041B204689B2FDF789FBB542AF
:10D3F000F7D1FFF756BB00258146DFF85882DFF8EA
:10D4000058B2059504950695079501214FF6FF7AC8
:10D4100005E001350B2D00F0998118F9011F4F1C13
:10D420004AFA05F3F5D0DE07F3D5BBF800302B41FF
:10D43000D807EED506A8FDF7A9FEEAE708460822B8
:10D440007C49FDF715FB0120FFF72CBB0B687A4ADE
:10D45000581C917820601970FFF797BB0B68774ACA
:10D46000774D1178774A581C206019701168204652
:10D47000FDF72EFB23686F4A591C127A21601A703F
:10D4800029882046FDF73CFBA9882046FDF738FB9C
:10D4900029892046FDF734FB00212046FDF730FBAB
:10D4A00020460021FDF72CFB0120FFF7FBBA0021ED
:10D4B0002046FDF725FB00212046FDF721FB00213A
:10D4C0002046FDF71DFB23685F4D00265A1C226095
:10D4D0001E7023682A68591C92F82C2021601A704B
:10D4E00023682A68591C92F8362021601A70236834
:10D4F0002A68591C92F8372021601A7023685A1C38
:10D5000022601E7023685A1C22601E7023685A1CF9
:10D5100022601E702B682046598FFDF7F1FA2B68A8
:10D520002046198FFDF7ECFA23682A68591C92F8F7
:10D530002E2021601A7023685A1C22601E702B68EE
:10D540002046598EFDF7DCFA2B682046998EFDF7B0
:10D55000D7FA0120FFF7A6BA3C4E0B6872793A4D14
:10D56000591C21601A702B682046198CFDF7C8FAE7
:10D570002B682046D98BFDF7C3FA71892046FDF749
:10D58000BFFAB1892046FDF7BBFA2B682046598CBB
:10D59000FDF7B6FA2B682046998CFDF7B1FAF189B0
:10D5A0002046FDF7ADFA318A2046FDF7A9FA2A6830
:10D5B000236892F82620591C216001201A70FFF779
:10D5C00071BA224EF378002B00F069810B680822B3
:10D5D000591C21601A7023680122991821601A7061
:10D5E00023681B4D591C2A7921601A702368AA7878
:10D5F000591C21601A7029882046FDF781FAE989B3
:10D600002046FDF77DFA2368F279591C21601A70D3
:10D610002368EA78591C216001201A70FFF742BA8A
:10D62000A4C30020DCC30020649600200CC70020A7
:10D630006C57002090980020704F0020FC4F002075
:10D6400034460020786C0020C86600204C960020EC
:10D650001C93002018330408786600201AF06CFD33
:10D66000FF28064600F0318108A9002501F8125D67
:10D670000DF10D008DF80D501AF03EFD08A800F8D0
:10D68000115D1AF02DFD08A800F8105D1AF01CFDC0
:10D6900008A820F8085D1AF00BFD23685A1C2260C8
:10D6A0001E7023689DF80D20591C21601A70236894
:10D6B0009DF80E20591C21601A7023689DF80F20D8
:10D6C000591C21601A7023689DF81020591C216094
:10D6D0001A702046BDF81810FDF712FAFFF7E1B9ED
:10D6E0000B68AD4AAD49D078AD4A5D1C2560187015
:10D6F00023684979581C206019702368D278591C16
:10D70000216001201A70FFF7CDB90020FFF7CAB9D8
:10D7100023685A1C2260197029882046FDF7F0F909
:10D720002368EA78591C21601A7023682A79591CE9
:10D7300021601A702368AA79591C21601A70236825
:10D740006A79591C21601A70FFF7A5BADFF87CA22C
:10D7500000254FF008080135C5F1200208FA02F251
:10D76000A5F120032AFA05F6164328FA03F31E430F
:10D77000252D06F001024FF000030BD01343EAD031
:10D78000E8B224F0D3FF0028E5D0294606A8FDF72B
:10D79000FDFCE0E7834B1B78DA0700F19D80002554
:10D7A000814E2F4602E00135252D0DD02946304609
:10D7B000FDF7FCFC0028F6D0294606A8FDF7F6FC8C
:10D7C00000285ED10137EEE7784B794DB3F8501061
:10D7D0002046FDF795F9774B1988204689B2FDF769
:10D7E0008FF9754B19684B0103F02002C1F3400318
:10D7F0001343C1F3800243EA4203C1F3C00243EA88
:10D800008203C1F3401243EAC20301F0100119433D
:10D810002046FDF775F904A904222046FDF728F9F2
:10D8200023682978654A581C20601970118864297A
:10D83000A8BF64212046FDF763F9B9F1960F50D0D7
:10D8400000212046FDF75CF92168B7F1190348BFB4
:10D85000A7F11203A3F3C4034A1C226020461A4610
:10D860000B7005A9FDF704F92368554A581C1021CF
:10D870002060197020461188FDF72AF90120FFF772
:10D8800011B9394604A8FDF781FC9BE7F4EEC87A8C
:10D89000F1EE10FA58DA4FF47A71FFF7D0BA0B684C
:10D8A000B178484A581C2060197023681278591CB6
:10D8B00021601A7094E6082771E595F82420424B00
:10D8C000002A38D13046FFF728BB23685A1C226053
:10D8D00001201E70FFF7E6B8069B43F00103069394
:10D8E0005DE723680322591C21601A7023686A7857
:10D8F000591C21601A70A7E7042750E5F4EEC87A96
:10D90000F1EE10FA3FF5B8AAF4EEE87AFDEEE77A08
:10D91000F1EE10FA17EE901A2FD86FF4F973303930
:10D9200003FB01F140F2E73391FBF3F101F2DB512C
:10D9300089B2FFF784BA5978022918D003290CBF9D
:10D9400004203046FFF7E9BAFDEEE77A40F2E7320D
:10D9500017EE903A303B02FB03F388FB0312D91712
:10D96000C1EB622101F2E93189B2FFF768BA042AFA
:10D9700034BF02200320FFF7D0BA40F2F313A1F521
:10D98000836103FB01F140F2E73391FBF3F101F214
:10D99000DD5189B2FFF753BA544F002080B90020FF
:10D9A000644F0020946E0020C4C40020681F002033
:10D9B000CC660020A447002018C40020A8470020FF
:10D9C000D0B70020484F002038A1002090E33FF45A
:10D9D0001C4C08B501210220FCF73EF9237803F026
:10D9E0000502052A29D003F00903092B08D00021DC
:10D9F0000120FCF731F900210846FCF72DF9FEE77C
:10DA0000114A124B11681A680B68114C23F001037C
:10DA10000B601388206823F001031B041B0C138088
:10DA200018B1292200238271C37103224A21FBF716
:10DA30007BFF2068FCF7FCF8D9E71EF077FF23781E
:10DA4000D1E700BF8C450020002F0020F82E0020D9
:10DA5000FC2E0020022828BF022010B4084C094BDD
:10DA6000207000EB8002C0EBC20207495DF8044B56
:10DA7000013003EB4203C0B20B602BF045B900BF8D
:10DA8000CC6600204A6B0020C866002008B515F05F
:10DA9000DBFBFCF7D1FDBDE8084015F0BDBB00BFC6
:10DAA00038B5484B5A899989914224BF00225A813E
:10DAB000198ADA89914224BF0022DA81DA78CAB160
:10DAC000072A41496AD091F85700404D01240021AE
:10DAD0000A282C709C70D9715DD00C2807D0002AC0
:10DAE0006CD0DFED3B7A072A0ED00A2862D0DFED3A
:10DAF000397A09E0344A92F857000A2856D00C289F
:10DB00005BD1D979DFED347A344C9FED350AA278B8
:10DB1000002918BFF0EE407A062A04D8314901EBFB
:10DB2000820191ED0F0A217979B1013A032A0BD8CC
:10DB3000F7EE007A87EE800A33F08EF92388984258
:10DB400028BF1846208038BD38BD9B781F4A07EE95
:10DB5000103A1178B8EEC77A67EE277A07EE101AF6
:10DB6000B8EEC77A27EE277AB4EEC70AF1EE10FABC
:10DB7000EADD80EE277AFDEEC77A17EE903A102B99
:10DB8000A8BF1023012BB8BF0123DBB28B4238BFE3
:10DB90000B46137038BDDFED147AA4E791F85700F7
:10DBA0000A2803D00C28ACD0D9799AE7D979DFEDCF
:10DBB0000E7AA9E7DFED0D7AA6E7D979DFED047AD1
:10DBC000A2E700BF4C9600200CC70020484F002061
:10DBD0006F1203396F12833A0AD7A3391C930020BE
:10DBE0006F120338E83204085304E9380F506E3AD4
:10DBF00038B50D4C0D4DAC4206D261682046143448
:10DC0000FCF7A6FCAC42F8D3FDF7DEFA084A094B54
:10DC1000094C1460002209491A705A7008480860BB
:10DC2000BDE8384019F060BB9001000840060008CC
:10DC3000C8660020CC6600204A6B0020807F002050
:10DC4000F664002008B5FFF7D3FF15F0FDFAFCF7E6
:10DC5000F3FCBDE8084015F0DFBA00BFF0B50C29B1
:10DC600034D8DFE801F0893333335E333333343370
:10DC700033330700048C9689B2F802E01788734D9D
:10DC800024F480542404240C0484038C8488818B21
:10DC900023F4005321F4E6411B0409041B0C46EA5B
:10DCA0000E06090C43EA063341EA0721A8429BB25B
:10DCB000A4B289B200F09E8005F58065A84200F00C
:10DCC000998092688480818302640384F0BD048C0F
:10DCD0009589B2F802C0B2F800E05C4F24F4807479
:10DCE0002404240C0484038C8688818B23F4007321
:10DCF0001B0421F073011B0C45EA0C04090443EAE0
:10DD00000423090CB8429BB2B6B241EA0E015CD0C2
:10DD10004F4CA04259D0926886808183C2630384AD
:10DD2000F0BD048C9589B2F802C0B2F800E0474E0D
:10DD300024F010042404240C0484038C8788018BB1
:10DD400023F0200321F4E6411B0409041B0C45EADF
:10DD50000C04090C43EA041341EA0E21B0429BB2C1
:10DD6000BFB289B25DD03A4CA0425AD09268878047
:10DD7000018382630384F0BD048C9789B2F802E0CA
:10DD80001688324D24F001042404240C0484038CEE
:10DD90008488018B23F002031B0421F073011B0C08
:10DDA00047EA0E0709043B43090CA8429BB2A4B200
:10DDB00041EA060125D005F58065A84221D0926888
:10DDC0008480018342630384F0BDD589148A578A15
:10DDD00023F4006343EA05254FF6FF332B40958873
:10DDE00026F440563C4343EA052346EA04169BB218
:10DDF000B6B290E7158A24F4804444EA8514A4B2AC
:10DE00005FE7D689158A578A23F00803334324F441
:10DE1000407496883D4323F004032C433343A4B25B
:10DE2000CDE7D489158A568A23F0800343EA041388
:10DE30004FF6BF741C40938827F44067354344EA8B
:10DE4000031347EA85079BB2BFB28FE7000001408A
:10DE5000000401402DE9F84F4FF4A07200218A48D8
:10DE60008A4C8B4D8B4E8C4FDFF84882DFF84892FE
:10DE700035F0FFF889488A49DFF840E2DFF840C210
:10DE8000002213588B4200F0C280B3F1804F00F0A3
:10DE9000D180AB4200F0D580B34200F0D580BB42C8
:10DEA00000F0D580734500F0D580634500F0D58043
:10DEB000434500F0D5804B4500F0D480DFF804A244
:10DEC000534500F0D2800AF5806A534500F0D080B7
:10DED000AAF5983A534500F0CE800AF5806A53457A
:10DEE00000F0CC800AF5806A534500F0CA801832F1
:10DEF000B2F5C07FC5D1694E6A4F06F5C0784FF0C4
:10DF0000030A4FF0020902E01836B0457DD0B3791C
:10DF1000002BF9D033791C09013C032C03F00F03CB
:10DF2000F2D8614A32F8140040FA03F2D207EBD576
:10DF3000012505FA03F3013B184032F015FB5B4B5A
:10DF40001B5D184417EBC002DED057F83030584C38
:10DF5000317A03F13F4000F57E00800A205C00F03A
:10DF60001F044009032805FA04F55DD0042855D0A4
:10DF7000022804D14548406C054344484564B2F842
:10DF800004E0BEFA8EF2C2F11F0292B2D00803EB97
:10DF9000800002F00702046A92000F25954024EAEF
:10DFA00005040462046A01FA02F2224300250262B7
:10DFB0004FF0010C2A4603E0102A05F10205A3D018
:10DFC0000CFA02F030EA0E0102F10102F4D11C68F1
:10DFD0000AFA05F1C9430C401C60D3F800B009FAF5
:10DFE00005F444EA0B041C609C680C409C609C682F
:10DFF0009C605C6824EA0000586058685860D868E3
:10E000000140D960D968D960D6E7BDE8F88F01230F
:10E01000D4F844A043EA0A03636468E71B48006B32
:10E0200005431A480563AAE71848006C05431748DA
:10E030000564A4E74FF0010A236C43EA0A03236452
:10E0400055E74FF0020AF7E74FF0040AF4E74FF004
:10E05000080AF1E74FF0100AEEE74FF0200AEBE76D
:10E060000223D5E74FF48033D2E74FF40033CFE7F4
:10E070004FF48023CCE74FF0400ADDE74FF0800AF1
:10E08000DAE74FF4807AD7E7CC2C00200038024042
:10E090000004004000080040000C0040905A0408B2
:10E0A00000000140F4CE0020E4660408E0660408A5
:10E0B000105C0408000401400040014000100040D2
:10E0C000001400400044014001490248FEF78EBBA5
:10E0D000E42D00200048014001490248FEF786BBBC
:10E0E000942D00200040014001490248FEF77EBB0C
:10E0F0006C2D00200004014001490248FEF776BB68
:10E100006C2D00200004014001490248FEF76EBB5F
:10E11000442D00200008004001490248FEF766BB7C
:10E120001C2D00200004004002494FF08040FEF703
:10E130005DBB00BFF42C002010B5064C06482146FC
:10E14000FEF754FB04F1F0010448BDE81040FEF76F
:10E150004DBB00BFCC2C002000000140004401401A
:10E1600001490248FEF742BBCC2C002000000140D0
:10E17000F0B50468544DA30AAB4200F082805AD92E
:10E18000524DAB4269D075D9514DAB4261D001358A
:10E19000AB4240F096804FF49C7E07264779B00052
:10E1A0004FEA970C002978D063460227A5899F4043
:10E1B00083190CEB43032F4303F1040C454DBFB20D
:10E1C00045F8231045F82C20A781EFF31181502248
:10E1D00082F31288821905EBC2021369002B40D02A
:10E1E00013620433821905EBC202576917B11F602D
:10E1F00053690433821905EBC202976917B11F6096
:10E2000093690433821905EBC202D76917B11F6005
:10E21000D36904330027CAB21F6082F311883044E7
:10E2200005EBC000036AFBB9A38923F001031B04BB
:10E230001B0CA381F0BD3F3DAB422AD00135AB4260
:10E2400003D0B3F5801F20D0F0BD4FF0980E032609
:10E25000A4E74FF4887E0626A0E74FF0E80E0526D7
:10E260009CE705EB0E03BDE7A3899BB243F00103D6
:10E27000A381F0BD0F3DAB4224D14FF0C00E042668
:10E280008CE74FF0200E002688E74FF0480E01265D
:10E2900084E74FF0700E022680E70223BF0803FADE
:10E2A00007F7A3890B4D9BB223EA070387190CEBF1
:10E2B000470CA3810CF1040345F82C1045F82320EA
:10E2C00083E7F0BDF0BD00BF40001000500010001B
:10E2D00051001000CC2C002010B503688348013990
:10E2E000834282B089B200F0CB80A0F58060834287
:10E2F00000F0C68000F58040834200F0B88000F551
:10E300008060834200F0B38000F58060834200F0BB
:10E31000AE80774C188824686408B4FBF2F4013CA2
:10E32000A4B282B2B3F1804F0AD07248834207D0C0
:10E3300000F58060834203D000F58060834202D103
:10E3400022F0700292B26C48834200F0A28000F585
:10E350008060834200F0A78022F4407200F56C4098
:10E3600092B283421A80D9621C854FD05F4A934291
:10E370004CD001229A821A8892B242F001021A808D
:10E38000B3F1804F00F099805A4A934200F0978091
:10E3900002F58062934200F0948002F5806293421D
:10E3A00000F0918002F58062934200F08E8002F5C9
:10E3B0008062934200F08B8002F57042934200F03D
:10E3C000888002F57052934200F0858002F58062E9
:10E3D000934200F0828002F5806293427FD0A2F5E2
:10E3E000983293427DD002F5806293427BD002F551
:10E3F0008062934208BF0D2215D002A84FF001237E
:10E4000040F8043D20F092FE02B010BD0122002130
:10E4100019869A821A88394892B242F001028342E0
:10E420001A80ADD10A46364B03EBC20301A893F81C
:10E430005D408DF80440012300228DF805308DF8F1
:10E4400007308DF8062020F071FE1B2C08D02E2CF2
:10E45000DAD12C4B019301A820F068FE02B010BD68
:10E46000294B019301A820F061FE02B010BD204CA1
:10E4700018882468B4FBF2F4013CA4B282B251E7DC
:10E480001B4C18882468B4FBF2F4013CA4B282B29D
:10E4900056E701201A80D9621C8598821A8892B2A8
:10E4A00002431A8070E701201A80D9621C85988285
:10E4B0001A8892B202431A8062E70122B3E702226D
:10E4C000B1E70322AFE70422ADE70522ABE706225E
:10E4D000A9E70722A7E70822A5E70922A3E70A225E
:10E4E000A1E70B229FE70C229DE700BF000401403B
:10E4F000D0980020000400400010004000000140BF
:10E50000E83204082C010001190100012C4B98424B
:10E510003DD0B0F1804F3CD0A3F57C4398423AD037
:10E5200003F58063984238D003F58063984236D073
:10E5300003F58063984234D003F58063984232D06B
:10E5400003F57043984230D003F5705398422ED0B3
:10E5500003F5806398422CD003F5806398422AD05B
:10E56000A3F59833984228D003F58063984207D0EA
:10E5700003F58063984208BF0D2202D00020704747
:10E580000C22104B03EBC20393F85C00704700228F
:10E59000F7E70122F5E70222F3E70322F1E704227D
:10E5A000EFE70522EDE70622EBE70722E9E708227D
:10E5B000E7E70922E5E70A22E3E70B22E1E700BFEC
:10E5C00000000140E83204082DE98048013085B0A0
:10E5D000C3B203938A4D8B4F8B4C8C4E0A2302930C
:10E5E000DFF82C9230F0B0FC4FF4FA7A4FF0100CB8
:10E5F0004FF47A70D9F80430C3F30803002B40F0CD
:10E60000C180EFF31183002B40F0BC802968A26821
:10E6100000BF2B689942F9D1D7F800E000FB0EF358
:10E620009B1AB3FBFEF300FB01314FF0010E019189
:10E63000D9F80430C3F30803002B40F08780EFF3D0
:10E640001183002B40F082802B68A16800BF2A68EC
:10E650009342F9D1D7F800B000FB0BF2521AB2FB8B
:10E66000FBF200FB0323019A9B1AB3F57A7FDFD3F9
:10E67000BAF1010ABED1039B002B40F0BD804FF4DC
:10E680007A7ADFF88C9150464FF0100CD9F80430AC
:10E69000C3F30803002B40F09280EFF31183002BAB
:10E6A00040F08D802968A26800BF2B689942F9D19B
:10E6B000D7F800E000FB0EF39B1AB3FBFEF300FB60
:10E6C00001314FF0010E0191D9F80430C3F3080372
:10E6D00003BBEFF31183EBB92B68A16800BF2A6875
:10E6E0009342F9D1D7F800B000FB0BF2521AB2FBFB
:10E6F000FBF200FB0323019A9B1AB3F57A7FE3D365
:10E70000BAF1010AC2D1029B013B02937FF468AFC8
:10E71000FCF7EEFEEFF311888CF31288A1682368F2
:10E72000DB0344BFC6F800E0A1682B6832685FFADB
:10E7300088F888F31188D7F800801A4400FB08F3A2
:10E740005B1AB3FBF8F300FB0233D4E7EFF3118855
:10E750008CF31288A1682368DB0344BFC6F800E08D
:10E76000A1682B6832685FFA88F888F31188D7F8B7
:10E7700000801A4400FB08F35B1AB3FBF8F300FBBC
:10E78000023370E7EFF311828CF31288D4F808E0BB
:10E790002368D90303D501233360D4F808E02B683C
:10E7A0003168D2B282F311883A68194400FB02F34F
:10E7B000A3EB0E03B3FBF2F300FB013135E7EFF3FC
:10E7C00011828CF31288D4F808E02368D90303D5AA
:10E7D00001233360D4F808E02B683168D2B282F3A9
:10E7E00011883A68194400FB02F3A3EB0E03B3FB54
:10E7F000F2F300FB013164E7184630F007FA3EE718
:10E80000B4D00020B8D0002010E000E0B0D000204C
:10E8100000ED00E02DE9F047AB4FAC4E14F014FDD5
:10E82000BE421ED2DFF83083DFF83093444625889D
:10E8300062197DB14A450DD2052D0BD93388618807
:10E84000C3F30B03994200F0ED801446258862194A
:10E85000002DEFD1716830461436FBF779FEBE42C9
:10E86000E4D39B4A1378A3F1170102290FD99949E0
:10E8700011F83300002840F01A81D800014449788B
:10E8800029B1954911F833300BB918231370934C03
:10E890006378022B84BF002363702378022B84BF2C
:10E8A000002323708E4B9A78042A00F0F78032B947
:10E8B0001A88B2F5F07F84BF4FF4F0721A80894D48
:10E8C000894A2B681A40002A00F0FA80D80700F124
:10E8D000E080590400F1D8801A0700F1D0809B0431
:10E8E00000F1C680814D2B685A8C998C914224BFCF
:10E8F00000225A84FFF7D4F826F0F6F9002800F039
:10E90000B3804020FBF75AFE4FF40070FBF756FE31
:10E910004FF00070FBF752FE4FF08060FBF74EFEA9
:10E920006378022B06D8724A724903EB430302EB69
:10E9300083030B602378022B07D803EB83016E4A15
:10E94000C3EBC10302EB43032B6023F067FF0021FD
:10E9500030226A4834F08DFB28682CF025FC684B87
:10E960002D6803F1500102E0043399427AD01A78FD
:10E97000002AF9D19C78D8788442F5D26149624B5B
:10E980000A7028461D6019F02BFB604B604A1E7907
:10E9900060496148614B1160C825642212FB065230
:10E9A0005F4C406B31F8061C5A60002221809A604F
:10E9B000DA601A615A619A61DA6183F8202083F87B
:10E9C000212008B116F0A8FF564B9FED575A1B881F
:10E9D000564A9FED576A557B564C57495748086031
:10E9E00006EE903AF8EEE66A1389C5EE265A07EE6F
:10E9F000103A5389127BC4ED005A07EE903AB8EEF4
:10EA0000C77A4F4BF8EEE77A1D725A7227EE067AF4
:10EA100067EE867ABDE8F04783ED017AC3ED007AB0
:10EA200014F0FABB63799B077FF40FAF716894F819
:10EA300004A03046FBF78CFD3388BAEB133F04D0BB
:10EA40001436BE42FFF4F2AE0BE773887068AA1F5B
:10EA5000C3F30B039A4204F10601A8BF1A4631F032
:10EA6000F1FFEDE7012289E7364829F009F848E788
:10EA70003548FBF7A3FD4020FBF7A0FD32E7334804
:10EA8000FBF79CFD2B682AE73148FBF797FD2B68C5
:10EA900022E73048FBF792FD2B681AE79A8AB2F515
:10EAA0007A7FBFF40CAF4FF47A729A8207E7D800EE
:10EAB0000C186468002C7FF4E1AE17241470DDE6B6
:10EAC00043F008032B6001E74006000890010008AE
:10EAD000FC4F0020445C040858630408CC66002006
:10EAE0001C930020786C002009600002C86600209A
:10EAF000F6640020807F00204A6B0020142A00204A
:10EB000000500020B41E0020482A00206C6A00201B
:10EB10009CC400205A4F0020A4C30020806600201F
:10EB2000CC500020502C0020C0C9FB488426002077
:10EB300017B7D138542C0020446800203661023DBC
:10EB40002068002058910020094000020160000266
:10EB5000092000020860000202400008008000084E
:10EB600008B514F071FBFBF767FD14F055FBFFF7D8
:10EB700051FE0120BDE808402AF0C6B82DE9F04F4B
:10EB8000013085B0C3B203930B4602918B4C8C4E7F
:10EB9000002B00F099808B4D8B4FDFF8309230F0D6
:10EBA000D3F94FF4FA7A4FF0100C4FF47A70D9F889
:10EBB0000430C3F30803002B40F0DE80EFF3118331
:10EBC000002B40F0D9802968A26800BF2B689942C9
:10EBD000F9D1D7F800E000FB0EF39B1AB3FBFEF36C
:10EBE00000FB01314FF0010E0191D9F80430C3F35D
:10EBF0000803002B40F08780EFF31183002B40F0D7
:10EC000082802B68A16800BF2A689342F9D1D7F8A7
:10EC100000B000FB0BF2521AB2FBFBF200FB032325
:10EC2000019A9B1AB3F57A7FDFD3BAF1010ABED1FC
:10EC3000039B002B40F0BD804FF47A7ADFF88C9173
:10EC400050464FF0100CD9F80430C3F30803002BE2
:10EC500075D1EFF31183002B71D12968A26800BF31
:10EC60002B689942F9D1D7F800E000FB0EF39B1A0C
:10EC7000B3FBFEF300FB01314FF0010E0191D9F817
:10EC80000430C3F3080313BBEFF31183FBB92B6804
:10EC9000A16800BF2A689342F9D1D7F800B000FB01
:10ECA0000BF2521AB2FBFBF200FB0323019A9B1AF0
:10ECB000B3F57A7FE3D3BAF1010AC4D1029B013BD9
:10ECC0000293002B7FF467AF05B0BDE8F08FEFF340
:10ECD00011888CF31288A1682368DB0344BFC6F84F
:10ECE00000E0A1682B6832685FFA88F888F3118821
:10ECF000D7F800801A4400FB08F35B1AB3FBF8F363
:10ED000000FB0233D2E7EFF311888CF31288A1687D
:10ED10002368DB0344BFC6F800E0A1682B683268B3
:10ED20005FFA88F888F31188D7F800801A4400FB4E
:10ED300008F35B1AB3FBF8F300FB023370E7EFF361
:10ED400011828CF31288D4F808E02368D90303D524
:10ED500001233360D4F808E02B683168D2B282F323
:10ED600011883A68194400FB02F3A3EB0E03B3FBCE
:10ED7000F2F300FB01317FE7EFF311828CF312888D
:10ED8000D4F808E02368D90303D501233360D4F80D
:10ED900008E02B683168D2B282F311883A681944CE
:10EDA00000FB02F3A3EB0E03B3FBF2F300FB013114
:10EDB00018E718462FF02AFF3EE700BF10E000E0FA
:10EDC000B0D00020B4D00020B8D0002000ED00E08A
:10EDD000204B5B68C3F3080330B4BBB9EFF3118376
:10EDE000A3B91D4B1D4C1868A16800BF1A6890425A
:10EDF000F9D11B4B1C684FF47A7202FB04F3591AC9
:10EE0000B1FBF4F130BC02FB00107047EFF311824C
:10EE1000102383F3128811498C680B6813F4803F28
:10EE2000104B02D0012018608C680B49D2B20D68DB
:10EE3000186882F311880A4B19684FF47A722844D3
:10EE400002FB01F31B1B30BCB3FBF1F302FB0030F0
:10EE5000704700BF00ED00E0B4D0002010E000E0FB
:10EE6000B8D00020B0D000202DE9F84F8046FFF741
:10EE7000AFFF254E2549DFF8A0E0254A254D844601
:10EE800010274FF47A740120DEF80430C3F308032E
:10EE9000D3B9EFF31183BBB90B68D2F808A000BF58
:10EEA000D1F800904B45F7D1D6F800B004FB0BF930
:10EEB000A9EB0A09B9FBFBF904FB0393A3EB0C03D1
:10EEC0004345E1D3BDE8F88FEFF3118A87F3128849
:10EED000D2F808B01368DB0344BF2860D2F808B04A
:10EEE0000B68D5F800905FFA8AFA8AF31188D6F891
:10EEF00000A0994404FB0AF3A3EB0B03B3FBFAF362
:10EF000004FB0933DAE700BFB8D00020B4D00020FA
:10EF100010E000E0B0D0002000ED00E02DE9F04F5F
:10EF2000DFF830C1474A4849484E494D80461027CE
:10EF300018F1FF38C0F08480DCF80430C3F3080314
:10EF4000002B5CD1EFF31183002B58D10B68946830
:10EF500000BF08688342F9D1D6F800904FF47A7068
:10EF600000FB09FEAEEB040EBEFBF9FE00FB03EE58
:10EF7000DCF80430C3F308034FF47A740120FBB9C2
:10EF8000EFF31183E3B90B68D2F808A000BFD1F802
:10EF900000904B45F7D1D6F800B004FB0BF9A9EB74
:10EFA0000A09B9FBFBF904FB0393A3EB0E03B3F5CA
:10EFB0007A7FBDD2DCF80430C3F30803002BDFD026
:10EFC000EFF3118A87F31288D2F808B01368DB03D5
:10EFD00044BF2860D2F808B00B68D5F800905FFAFB
:10EFE0008AFA8AF31188D6F800A0994404FB0AF340
:10EFF000A3EB0B03B3FBFAF304FB0933D5E7EFF301
:10F00000118487F31288D2F808901368D80303D5C7
:10F0100001232B60D2F808900B682868E4B284F3CF
:10F020001188D6F800A04FF47A7400EB030E04FBAD
:10F030000AF3A3EB0903B3FBFAF304FB0E3E97E7D5
:10F04000BDE8F08F10E000E0B4D00020B8D0002080
:10F05000B0D0002000ED00E030B4EFF311831022B7
:10F0600082F312880649074C0A68074801320025D6
:10F070000A602560DBB2026883F3118830BC7047F8
:10F08000B4D00020B0D0002010E000E00F4B1B886F
:10F09000014643B90E4B0F4A1B7810680BB981F03B
:10F0A0000101FAF7D1BD0C4B5A691AB118B91A68A7
:10F0B000106058747047094A18681188084A92FB12
:10F0C000F1F2012102605974704700BF8CD000201A
:10F0D0008ED0002090D0002094D00020ACD0002012
:10F0E00020A1070038B5254B1C69236B73B1636DF4
:10F0F000626BCAB1998A1A88C90592B201D5D20742
:10F1000000D438BD4FF6F7721A8038BD636D998907
:10F110001A88890692B2EBD59206E9D5E26ACAB19D
:10F12000988880B29047E2E799891A880D0692B2D2
:10F13000E0D51006DED5A26A616A8A4219D0A169BB
:10F140002569885C98800132B2FBF5F105FB11223C
:10F15000A262CFE79B88E2696169DBB28B54E26906
:10F16000E068636D0132B2FBF0F100FB1122E26155
:10F17000BEE7DA6822F08002DA60BBE79045002043
:10F1800038B5254BDC68236B73B1636D626BCAB114
:10F19000998A1A88C90592B201D5D20700D438BD20
:10F1A0004FF6F7721A8038BD636D99891A888906FF
:10F1B00092B2EBD59206E9D5E26ACAB1988880B2DC
:10F1C0009047E2E799891A880D0692B2E0D51006B9
:10F1D000DED5A26A616A8A4219D0A1692569885C74
:10F1E00098800132B2FBF5F105FB1122A262CFE754
:10F1F0009B88E2696169DBB28B54E269E068636D08
:10F200000132B2FBF0F100FB1122E261BEE7DA68E5
:10F2100022F08002DA60BBE7904500202DE9F04F34
:10F220002DED028B95B080462AF0A2FC8E4B1D7806
:10F2300025B115B0BDEC028BBDE8F08F8B4B1B6880
:10F240005905F6D58A4BDFF880B21B686BB1894A45
:10F25000DBF800101368CB1A7C2B06D986481160A6
:10F260000378013303702DF0EBFC844B1B78002BEB
:10F270006DD0834C834AD4F81031A8EB030393423A
:10F2800001F2278394F81891B9F1000F32D17E4F23
:10F290003868FAF7D3F8C0B201280FD902287B4E9C
:10F2A00042F013803378002B42F00881D4F81C31EF
:10F2B000A8EB0303B3F57A6F82F0CE82D4F8203145
:10F2C000002B44D094F81831BBB9714B1B689B7864
:10F2D00001211E3B00228B4284F8181184F82C2156
:10F2E00042F26C823868022104302DF05BFC94F805
:10F2F000243110E0D4F820314BB3D4F8283140F653
:10F30000B732A8EB0303934221D994F82431002BA0
:10F3100001F0D9865C4F013BDBB284F82431002B2D
:10F3200001F00A84D4F8206194F82C2116F8011B0E
:10F3300094F82D313868C4F820610A44013384F808
:10F340002C2184F82D31FAF77DF8C4F82881514B2F
:10F35000DBF800601B7843B14F4F386828B14F4B42
:10F360001B78013B012B41F2F6834D4B1B786BB1AF
:10F370004C4F3B6853B1DBF80030414C03931A46C5
:10F38000D4F84431D31A632B01F29381464F3B7872
:10F39000022B01F078863D4E96F87430032B01F075
:10F3A000B683424B1B7873B1414D2B685BB1344C33
:10F3B000FFF70EFDD4F85031039044F61F62C31AD4
:10F3C000934200F231813B4B1B78002B7ED13A4BAC
:10F3D0001B7843B12A4CD4F8A03203F5C333A033D1
:10F3E000984581F03782354B1B78002B3FF421AFD5
:10F3F000234E334C334D06F2C1272068FAF71EF82E
:10F4000000283FF416AF2068FAF710F82B788046F2
:10F410005A1E33B120682A70FAF710F80028F2D18A
:10F4200007E703223946781E33F009FE96F8C0320A
:10F4300096F8C12286F8C38283F47F4383F0FF03EA
:10F440009B1A1FFA88F89BB2B8EB132FD5D196F808
:10F45000C222DBB29A42D0D1781E20F0E1FC2B7898
:10F4600018442870C9E700BF50570020709600204C
:10F47000D4C10020F4C30020F0C3002062B80020F3
:10F480009C2600203F0D03009CC300202800002084
:10F49000A0C3002064B80020D8C100206CB80020B0
:10F4A00074B8002094C300201E4B00207CB80020BC
:10F4B00080B80020ECB80020FDB8002086B80020FD
:10F4C0008CB8002090B80020B4D00020484C22789E
:10F4D000A2B1484B9B7A53B1FFF77AFC464B1B68AD
:10F4E000C31AA3F57A73B3F5FA6F07D82278434BA2
:10F4F00043491868F9F76EFF00232370414CD4F894
:10F50000983203F5C333A0339845FFF460AF3E4D06
:10F51000C4F898822B78002B41F010873B4D2B7854
:10F52000002B41F06B8694F89C2239498D5CEA07E8
:10F5300002F10780AF0701F1C787680701F18887EB
:10F540002A0748D5334B344E0D9314AA1146A3F124
:10F550003D0241F8202D0020A3F140020D4603F8A2
:10F56000400C059102231121517093702846316897
:10F57000FBF788FA28467168FBF784FAF389274974
:10F5800003EBC3039B00053381FB0321DB17C3EBB4
:10F59000A101284689B2FBF78DFA338A03EB830376
:10F5A000590089B22846FBF785FA1D4B059D1B784B
:10F5B0009B0743BF318901F57A7189B24FF47A71A3
:10F5C0002846FBF777FA0C9B327D591C0C91284694
:10F5D0001A702AF05DFA134A94F89C3211780133BC
:10F5E00093FBF1F201FB123384F89C32EFE600BF8B
:10F5F00054B80020909800208C4A0020F0B80020D9
:10F6000014B800209C260020F4B80020F5B8002093
:10F61000F8B8002014B8002020C400206766666691
:10F620001CC40020FCB8002094F85631002B41F097
:10F63000CB85D34B1A6802F00803002B48F6034130
:10F640004AF60B404BF60F4349F6074604BF034604
:10F650000E4612F0040F4FF0190118BF1E46970610
:10F6600084F8561103D546F4804646F02006C54B73
:10F670005F79C6F30909002F42F013819B79002BB3
:10F6800042F01E821F4664204FF0FF3A4FF0000EFA
:10F690000C960D96ADF83E70ADF83CE0CDF842E02A
:10F6A000CDF846E0CDF84AE0CDF83890ADF840A06E
:10F6B0008DF84E000CAE0FCEB34F84F805E00FC7A7
:10F6C00096E80F0007C727F8023B39464FF0010EB6
:10F6D0001B0CFE261F20C82201F81E39A670A2713D
:10F6E00084F807E0E07094F86601207180F0F1037F
:10F6F00083EA0313DAB2130983F0E70343EA022330
:10F7000083EAC2031BB283EA0312D2B2C3F3072314
:10F7100083EA121343EA022383EAC2031BB283F093
:10F72000C80282EA0212D2B2C3F3072383EA121399
:10F7300043EA022383EAC2031BB283EA0E0686EA87
:10F740000616F6B2C3F3072282EA161242EA06222E
:10F7500000EB0E0382EAC60607EB0E0084F8663162
:10F76000268011F8013B734083EA0313DBB21A09C8
:10F7700082EA162242EA032282EAC3031BB29EB245
:10F7800081422680EDD183F07C0383EA0313DBB250
:10F790004FEA131E8EEA162E8EEA032E8EEAC30E51
:10F7A0000FFA8EFE1FFA8EFC784FA4F800C05FFAA5
:10F7B0008EFE4FEA1C2C84F828C084F827E007F559
:10F7C000C77904F1220A38687968BA68FB684E463E
:10F7D0000FC610375745B146F5D1386830606C4ECA
:10F7E0003B7989F8043006F1270784F8B5E184F8FD
:10F7F000B6C116F8011F2868F9F724FEB742F8D100
:10F8000094F85731002B41F0E4846249DBF8002082
:10F8100009780A2084F85701002901F000865E4E1D
:10F8200001293088079042F25181708806900229A0
:10F8300002F04F80B0880590032902F05E81F088C5
:10F840000490042902F054810529308902F04C818A
:10F850000629B6F80A9002F044810729B6F80CC0D0
:10F8600000D0F38994F866110C920F4687F03002AD
:10F8700082EA0212D2B216094849089786F07A063F
:10F8800046EA02260988277186EAC202444EC1EB85
:10F89000012186FB017A079E4FF0000E66F30F0EE2
:10F8A000069E12B266F31F4E8A44059ECDF834E0E0
:10F8B000C917C1EB6A2A002782EA0211C9B266F3AE
:10F8C0000F07C2F30722002682EA111260F30F0627
:10F8D000002007926CF30F00049A8DF845A063F3A3
:10F8E0001F40079B109062F31F4769F31F464FF0BC
:10F8F00000090E970F968DF8449043EA01220DF10E
:10F90000300E82EAC106BEE80F0036B286F0C80C9F
:10F910008CEA0C1C1C4F84F805905FFA8CFCC6F333
:10F9200007260FC786EA1C1646EA0C239EE803004A
:10F9300083EACC031BB283F0230247F8040B82EA6C
:10F940000212D2B2C3F30723089E83EA1213384689
:10F9500043EA022383EAC20206F1010E20F81419D9
:10F960004FF0230C1621FE26C82384F866E10237E7
:10F970002280E17084F807C0A670A371114611E0DF
:10F9800018C4002004C40020A42600209E260020C5
:10F990002B2800200858002030B50020ACB70020EC
:10F9A0000308208010F8013B4B4083EA0313DBB2CD
:10F9B0001A0982EA112242EA032282EAC3031BB235
:10F9C00099B2B8422180EDD183F0F40383EA0313A6
:10F9D000DBB24FEA131E8EEA112E8EEA032E8EEA58
:10F9E000C30E0FFA8EFE1FFA8EF7C84E27804FEA1D
:10F9F000172C5FFA8EFE84F81EE084F81FC0716831
:10FA0000B2683068F36806F5C7770FC73069716967
:10FA1000B26904F28F1607C704F2AD1784F8ADC1BE
:10FA200084F8ACE116F8011F2868F9F70BFDB7421E
:10FA3000F8D194F85A31002B41F0DB83B44B069394
:10FA40001B681922980684F85A2140F1EA82B14BCA
:10FA5000B14E1B78990741F12187337D042B8CBF70
:10FA600003270227FFF7B4F9338A32890C9003EB9E
:10FA700083035B00ADF84A304FF47A7033688DF839
:10FA80004C700E93F18996F814E073688DF84DE090
:10FA900000FB02F24FF0000C0CAF4FF0FF30CDF83E
:10FAA00034C010920F93ADF848101190BE46BEE8D6
:10FAB0000F000597994F0FC79EE80F0007C73A46FA
:10FAC000182122F81C39E17194F8661184F805C0F8
:10FAD00081F0780383EA0313D8B2030983F0F603B5
:10FAE00043EA002383EAC0031BB283EA0310C0B2D7
:10FAF000C3F3072383EA101343EA002383EAC00316
:10FB00001BB283F0C80080EA001E5FFA8EFEC3F3CA
:10FB1000072080EA1E1040EA0E2080EACE0000B2E4
:10FB200080F0180383EA0313DBB2C0F3072080EAF6
:10FB3000131040EA032080EAC30301F1010EFE2006
:10FB40004FF01E0C4FF0C809A0700237217184F8E5
:10FB500066E1238084F803C084F80690184612F802
:10FB6000011B414081EA0111C9B20B0983EA10234C
:10FB700043EA012383EAC10109B288B2BA42208074
:10FB8000EDD181F0180181EA0111C9B20A0982EAB6
:10FB9000102383EA012383EAC1031BB29AB25B49B3
:10FBA0000491DBB24FEA122C2280079384F827C01D
:10FBB00084F826300F4601F5C77A04F12209386827
:10FBC0007968BA68FB68D646AEE80F0010374F4533
:10FBD000F246F4D13868CEF80000DFF84C919DF879
:10FBE0001C3084F8B43109F1260784F8B5C1CA463F
:10FBF0001AF8011F2868F9F725FC5745F8D1FFF7D7
:10FC0000E7F8069B71681B683289069113F0140FA0
:10FC10004FF47A71D6F800E001FB02F141F00B8657
:10FC20000E4694F866A10C908AF06A003C4B3D4F5A
:10FC3000B3F90420CDF834E080EA0010C0B2030923
:10FC400083F0D50343EA002383EAC0031BB283EAAF
:10FC50000310C0B2C3F3072383EA101343EA00235F
:10FC600083EAC0031BB287FB0207D2174FF0000CD8
:10FC7000C2EBA7020698DDF814E0109683F0C807DF
:10FC80000E900F91ADF84A20ADF844C0ADF846C0D3
:10FC9000ADF848C087EA0717FFB2C3F30726BEE8EE
:10FCA0000F0086EA171646EA072686EAC7071B4EA4
:10FCB00084F804A03FB20FC687F021039EE8070036
:10FCC00083EA0313DBB2C7F3072787EA13170AF1A6
:10FCD000010E47EA032786E8070087EAC30384F892
:10FCE00066E14FF0210A4FF0FE0E1C27C8220C36A9
:10FCF00084F805C084F807A084F802E0A6F11C018E
:10FD0000E7701846A271238010E000BF9E260020F5
:10FD100018C400201CC4002020C40020A4260020F9
:10FD2000FCC30020676666662B28002011F8012BB3
:10FD3000424082EA0212D2B2130983EA102343EA54
:10FD4000022383EAC20212B290B2B1422080EDD106
:10FD500082F0680282EA0212D2B24FEA121A8AEAEA
:10FD6000102383EA022A8AEAC20A0FFA8AFA1FFAE1
:10FD70008AF3D74E23804FEA132C5FFA8AFA04F1F4
:10FD8000220384F825C084F824A006F5C77E0693D4
:10FD9000F36830687168B26877460FC7069B103603
:10FDA0009E42BE46F4D13388CA4E3B804F4684F80B
:10FDB000B2A184F8B3C117F8011F2868F9F742FB14
:10FDC000BE42F8D194F866E1C34AC44E84F804E018
:10FDD0008EF0EB0383EA0313D9B20B0983F0C5035A
:10FDE00043EA012383EAC1031BB283EA0310C0B2D2
:10FDF000C3F3072181EA101141EA002181EAC00121
:10FE00000CCA09B281F0C80787EA0717FFB24FF0A2
:10FE1000000C0C92C1F30721059A0D93CDF838C060
:10FE200081EA171343EA072307CA83EAC7031BB211
:10FE300083F0310786E8070087EA0717FFB2C3F3AC
:10FE4000072383EA171343EA072383EAC703277AC2
:10FE5000607AA17AE27A267B84F805C01BB25F4003
:10FE600087EA0717FFB2C3F3072383EA171343EAAE
:10FE7000072383EAC7031BB2584080EA0010C0B2D0
:10FE8000C3F3072383EA101343EA002383EAC00382
:10FE90001BB2594081EA0110C0B2C3F3072181EAC5
:10FEA000101141EA002181EAC00109B24A4082EA08
:10FEB0000212D2B2C1F3072383EA121343EA0223E8
:10FEC00083EAC2031BB25E4086EA0616F6B2C3F3AB
:10FED000072383EA161343EA0623607BA17BE27BB8
:10FEE000277C94F811C083EAC6031BB2584080EA0D
:10FEF0000010C0B2C3F3072383EA101343EA0023C0
:10FF000083EAC0031BB2594081EA0111C9B2C3F3AD
:10FF1000072383EA111343EA012383EAC1031BB2D7
:10FF20005A4082EA0212D2B2C3F3072383EA1213C1
:10FF300043EA022383EAC2031BB25F4087EA071742
:10FF4000FFB2C3F3072383EA171343EA072383EAC5
:10FF5000C7031BB28CEA030C8CEA0C1C5FFA8CFC06
:10FF6000C3F3072383EA1C1343EA0C2383EACC037D
:10FF7000A17CE27C5A4F1BB2594081EA0111C9B2FF
:10FF8000C3F3072383EA111343EA012383EAC1037E
:10FF90001BB25A4082EA0212D2B2C3F3072383EAA9
:10FFA000121343EA022383EAC2031BB283F027063B
:10FFB00086EA0612D2B2C3F3072686EA121646EA8A
:10FFC000022686EAC20636B20EF10103B2B2312031
:10FFD0004FF0FE0C0C2184F86631C8234FEA122E34
:10FFE0005FFA86FA2280E07184F802C0E170A371A2
:10FFF000049E84F814A084F815E07168B268F36870
:020000040801F1
:100000003068B6F810C00FC727F803CB84F8A3E117
:1000100084F8A2A119F8011F2868F9F713FA4F45CF
:10002000F8D194F85E71002F41F0DE802D4B94F8EA
:1000300066E1B3F90010B3F90220B3F904309FED83
:100040002A6A677107EE103ADBF800300C938EF0E5
:100050006A0383EA031306EE901AD9B20B0983F000
:10006000D50343EA012383EAC1031BB283EA0311E8
:100070005242C9B207EE902AC3F3072383EA111351
:1000800043EA0123F8EEE77AF8EEE66AB8EEC77ABB
:1000900083EAC1031BB267EE867A66EE866A27EEB4
:1000A000067A002083F0C80CCDED0E7ACDED0D6AF6
:1000B0008DED0F7A1090119012908CEA0C160DF1C4
:1000C0003009F6B2C3F3072CB9E80F000EE000BF09
:1000D0009E2600204F28002028520020A426002021
:1000E0002C280020FCC3002088C3E43A8CEA161CAC
:1000F0004CEA062C8CEAC60CD04E0FFA8CFC0FC6CC
:100100008CF01E0799E8070087EA0717FFB2CCF3C7
:10011000072383EA171343EA072386E8070083EAE5
:10012000C707C8214FF005094FF01E0CFE231C2005
:100130000EF10102A17184F85E9184F807C0A370EA
:10014000E070A6F1100184F804E00C36278084F8F2
:10015000662111F8013B7B4083EA0313DBB21A09E5
:1001600082EA172242EA032282EAC3031BB29FB249
:10017000B1422780EDD183F0270383EA0313DBB27A
:100180004FEA131E8EEA172E8EEA032E8EEAC30E56
:100190000FFA8EFE1FFA8EFCA94FA4F800C05FFA7A
:1001A0008EFE4FEA1C2C84F825C084F824E007F565
:1001B000C77904F1220A38687968BA68FB684E4644
:1001C0000FC610375745B146F5D19E4E3B88A9F86A
:1001D000003006F1240784F8B2E184F8B3C116F8C0
:1001E000011F2868F9F72EF9B742F8D194F85F910A
:1001F000B9F1000F40F0F287934B1B68052284F899
:100200005F219A0641F11581904ADFED917AD189FB
:1002100007EE101AB8EEC77A13F0140F27EE277AFC
:1002200001F071838B4BDFED8A6AD3ED007AF8EE33
:10023000E77A67EEA67A94F866C1874B874AB3F9E6
:100240000410B2F90620864E86488DED0D7A8CF0AA
:10025000220383EA0313DFB23B0983F0590343EA25
:10026000072383EAC703B2F5FA6F1BB2A8BF4FF4A6
:10027000FA6283EA0317FFB2B2F57A7FC3F307236A
:1002800083EA1713B8BF4FF47A724FF0640E43EA53
:100290000723A2F57A720EFB02F283EAC70786FBF8
:1002A00002E680FB01E03FB2C917D217C2EBA612EB
:1002B000C1EBA0034FF0000A0CA987F0C806CDEDF2
:1002C0000E7AADF84220ADF84030CDF830A0CDF830
:1002D0003CA08E4686EA0616F6B20591C7F30727BC
:1002E000BEE80F0087EA161747EA062787EAC60620
:1002F000524FDEF800E084F804C00FC736B286F033
:100300004A0383EA0313DBB2C6F3072181EA131120
:100310003A4641EA03210CF1010C81EAC30314209F
:1003200042F810E9FE264FF04A0E002184F866C11B
:100330004FF0C80CE0702380043784F807E0A67003
:10034000617184F806C0184612F8011B414081EA29
:100350000111C9B20B0983EA102343EA012383EA9E
:10036000C10109B288B2BA422080EDD181F01401F6
:1003700081EA0111C9B24FEA111E8EEA102E8EEAEF
:10038000012E8EEAC10E2E4B0FFA8EFE1FFA8EF64C
:100390001F464FEA162C5FFA8EFE84F81CE084F8A4
:1003A0001DC0386859689A68DB68B7F818A00497C8
:1003B00026803E4607F5C7770FC73069716903C7C6
:1003C00004F28F16A7F800A0374684F8ABC184F872
:1003D000AAE104F2AB1A17F8011F2868F9F732F8FE
:1003E000BA45F8D1204B214A1B781278013B12F014
:1003F0000100DBB214BFC0214021172B03D81C4AD7
:10040000134493F830901B4B1A8897071ABF0023A8
:1004100041F01001012312F4027F18BF022312F0F1
:10042000100F18BF062312F0200F18BF102300284A
:1004300041F008824FF0030C1EE000BFA42600200C
:100440009E2600202B28002018C4002020C4002055
:100450000AD7233CF8C30020FCC3002030B500209D
:10046000D34D621067666666FC4F0020946E0020D4
:10047000B03304087866002094F866E10C938EF09F
:10048000460383EA0313DAB2130983F0920343EAC3
:10049000022383EAC2031BB283EA0310C0B2C3F390
:1004A000072282EA101242EA002282EAC00212B255
:1004B00082F0C80787EA0717FFB2C2F3072282EA71
:1004C000171200238DF837C0032042EA072C059A43
:1004D0008DF834908DF835308DF836108DF8380061
:1004E00007CA8CEAC70C0FFA8CFCD04FE3718CEA78
:1004F0000C1903C75FFA89F9CCF3072C8CEA191C95
:100500004CEA092181EAC90994F808C03A700FFA47
:1005100089F98CEA090C8CEA0C1C5FFA8CFCC9F393
:10052000072282EA1C1242EA0C22607AA17A94F82D
:100530000B90637182EACC0212B2504080EA001C38
:100540005FFA8CFCC2F3072080EA1C1040EA0C2002
:1005500080EACC0000B2414081EA0111C9B2C0F387
:10056000072282EA111242EA012282EAC10212B291
:1005700089EA020989EA09195FFA89F9C2F30722AF
:1005800082EA191242EA092294F80CC0607BA17B2E
:1005900084F804E082EAC90212B28CEA020C8CEA06
:1005A0000C1C5FFA8CFCC2F3072282EA1C1242EA9E
:1005B0000C2282EACC0212B2504080EA0010C0B293
:1005C000C2F3072282EA101242EA002282EAC00243
:1005D00012B2514081EA0111C9B2C2F3072282EA84
:1005E000111242EA012282EAC102E17B94F81090E2
:1005F00013B281EA030282EA0212D2B2C3F30723E2
:1006000083EA121343EA022383EAC2031BB289EA94
:10061000030282EA0212D2B2C3F3072383EA12135F
:1006200043EA022383EAC2031BB283F0320282EA66
:100630000212D2B2C3F3072383EA121343EA02235E
:1006400083EAC2031BB29AB24FF0FE0C5FFA83FB3F
:100650000920C8210EF1010E84F802C04FEA122CC5
:10066000E070A17184F866E1228084F812C084F8F9
:1006700011B0049B186859689A68B3F80CA007F584
:10068000C07EAEE8070007F5C8778EF80290AEF896
:1006900000A084F8A0C184F89FB116F8011F286853
:1006A000F8F7D0FEB742F8D1039BC4F85031FEF7FB
:1006B0008ABEDFF898A15E4EDFF8949141202CF0BD
:1006C0001DFABAF9023086FB0320DB17C3EBA0004A
:1006D00080B22CF0F7F9BAF9003086FB0320DB1763
:1006E000C3EBA00080B22CF0EDF9BAF9043086FB20
:1006F0000320DB17C3EBA00080B22CF0E3F999F8DC
:1007000000103868F8F79EFE94F848A11AF0010628
:1007100000F0F784474B06931B689A0673D5464B47
:10072000464E1B789B0741F15180337D042B8CBFD3
:100730004FF0030A4FF0020A47202CF0DFF930682F
:100740002CF08CF970682CF089F93D4AF3893868EF
:10075000A2FB0323C3F3471319460493F8F772FE71
:10076000069B99F800101A68049B12F0140F83EA94
:10077000010389F8003040F067863389642000FB6C
:1007800003F02CF06BF9367D38684AEA8606F6B23B
:100790003146F8F757FE99F8003038685E40314628
:1007A00089F80060F8F74EFE94F848A1BAF1000FFE
:1007B00029D1244E4F202CF0A1F930682CF04EF9AD
:1007C00070682CF04BF950462CF048F9012138683C
:1007D000F8F738FE184A99F800301678386806F0AD
:1007E0000106314683F0010389F80030F8F72AFE4C
:1007F00099F8003038685E40314689F80060F8F7B3
:1008000021FE94F848A1039B0F4AC4F844310AF131
:100810000103DBB2A2FB0312D20802EB8202A3EBBC
:10082000420384F84831FEF7B1BD00BFA426002082
:100830006766666618C400201CC4002020C400201F
:100840001F85EB5128520020CDCCCCCCFCC300201E
:1008500098C3002094F8A432C24AC4F8A08202EBE4
:100860008302926C42B314AD04F2AB23BE4E45F842
:10087000203D002104F2BD2331800D9380211523FA
:10088000A52784F8AA32284684F8A91284F8A87209
:10089000904728463188FAF733F90C9DB34804F5A0
:1008A0002A716D1A152DA8BF15252A4630F0CAF8F1
:1008B000AF4A94F8A4321570AE4A013382FB03129A
:1008C000A2EBE37202EB42029B1A84F8A432FEF719
:1008D0008ABDA94AA94BD4F81411DBF800001B8883
:1008E000D77AA74A401A4FF47A71DEB201FB07F1BA
:1008F0001B0A9677167588424FF00006D37753751A
:100900009670167180F0D1849E4E9F4BD6F800C031
:100910001B689E4E9E48DFF8989201688068DFF859
:1009200094E286FB0376DB17C3EB661303F5FA73D9
:100930009BB293761B0AD37689FB0173C917C1EB6F
:10094000A30189FB00791177C0170912C0EBA90038
:1009500051778E4982F820000CF5EA43001281FBA2
:100960000C71303382F821004FEAEC701B12C0EB9F
:100970006110884E9EF800E082F823307830864B74
:1009800082F824000CF13001307D03901EF0020F3C
:1009900082F82210987600F08584D6F800E07F4A2D
:1009A000D6F804A07E48DFF810C282FB0E194FEA89
:1009B000EE7182FB0A72C1EBA9514FEAEA79C9EBE9
:1009C000A25200FB01E900FB02A009EB490900EB80
:1009D00040004FEA49094000049207468CFB092079
:1009E000801405908CFB072CF089049A36890797B0
:1009F00002EB820206F5FA7600EBC00002EB8202FF
:100A0000B6B204960892059E8200099201EB81011C
:100A10004FEAE972B01A01EB8101624E069102467B
:100A2000039906FB1292069E40B2052900EB860050
:100A30004FEAE7714FEAAC4C5A4E0590ACEB01001F
:100A4000014606FB1070089E504FDFF870C14FEA58
:100A5000DA7A49B201EB86014FEADE7E87FB006954
:100A600083F80EA087FB026A099F83F809E0DFF88C
:100A700050E13E468EFB066EBCF8006003969DF882
:100A800010605E75049EBDF814C083F80AC04FEA7A
:100A9000162689B204964FEAE2724FEAE777424E91
:100AA000D973C2EB6A12C7EBAE174FEA1C2A4FEAA2
:100AB000112E4FEAE0700399368883F80BA0C0EB43
:100AC000691083F810E04FEA22291A739DF810206C
:100AD0009A754FEA202CC7F3072A4FEA112134BF39
:100AE0004FF0320E4FF0330E9DF80C2083F80D902E
:100AF000587483F812C0DF7183F808A0DA7419758E
:100B000083F81BE01E77C4F81081FEF7BBBBDFF84B
:100B1000B490D9F80000F8F781FC00283EF441AC0D
:100B2000D9F800000121F8F775FC0222002386F8AD
:100B300074203B70FEF735BC94F82C1194F82D31DD
:100B400038684A1C013384F82C2184F82D31F8F7D9
:100B500079FCFEF7FABB154CDFF86C904FF0000AF9
:100B60003FE000BFB0330408D2B700207448002033
:100B70008948002056555555106F0020086F0020F9
:100B800094B80020ECC30020F8C300201F85EB516F
:100B9000E0C1002020C40020C0B800206BCA5F6BF9
:100BA000806967FF40420F00AE6600209C2600204F
:100BB000676666661CC4002083DE1B43B0B7002056
:100BC000D34D6210AC4B0020280000201B2B00F0FE
:100BD0006F820D2B00F04B814FF0010389F801303B
:100BE0003868F8F72BFC002839D03868F8F71EFC75
:100BF00083B27E2BDBF800202AD099F8011000295F
:100C0000EED194F82E21002AE0D07D2B00F0368220
:100C100094F83CE1BEF1000F04D080F02003DBB279
:100C200084F83C11511CC9B22244092984F82E11C0
:100C300082F8303100F016820829D1D8B4F83A2170
:100C4000134403EB132303F0FF03A4F83A31C7E77F
:100C500084F82EA184F82FA189F801A0C0E794F8A8
:100C60003D3133B194F8313184F83D01302B00F03F
:100C7000C18594F82F21C54BC549DFF850A3DFF893
:100C800050E391464A46002A3EF46FABDBF8002061
:100C9000921B012A24D894F83E21002A40F01E829B
:100CA00094F83FC133F81C00F8B94FF0010284F802
:100CB0003F210A689706E5D59AF800209007E1D50C
:100CC000B44EB549F2894FF4F36303FB02F381FBA1
:100CD0000321DB17C3EB61114FF403602BF048FFD6
:100CE000002384F82F31FEF740BB0CF1010C5FFAB2
:100CF0008CFCB0F5E06F84F83FC100F098801BD801
:100D0000B0F5047F00F0238135D8B0F5887F00F07E
:100D1000CD80B0F5007F00F0B380B0F5807FB1D119
:100D20000A685207AED59D4B19682BF021FF0023AE
:100D300084F82F31FEF719BBB0F5026F00F05A812D
:100D40006AD8B0F5E46F00F08180B0F5006F00F074
:100D5000D680B0F5E26F95D1914BDA6B998A642316
:100D600003FB02F393FBF1F12BF002FF002384F865
:100D70002F31FEF7FABAB0F5826F00F05181B0F56D
:100D8000C06F00F02781B0F5806F7FF47BAF94F8DF
:100D900040310133DBB2032B00F2AD8142F210711E
:100DA00084F8403101FB03F17E4B1B88002B40F09F
:100DB000A08101317C4B1B78DB077C4B1B8848BF33
:100DC0000431DF0748BF0A31980748BF14311A06BB
:100DD00048BF2831DF0548BF2831580748BF643174
:100DE0001A0748BFC8319F0548BF01F5C87198066A
:100DF00048BF01F57A71DA0648BF01F5FA615F066E
:100E000048BF01F57A614FF480602BF0B1FE0023FA
:100E100084F82F31FEF7A9BAB0F5046F1AD0B0F5F7
:100E2000116F52D0B0F5036F7FF42CAF41E75C4BEC
:100E300091469A6B998A642303FB02F393FBF1F1C9
:100E40002BF096FE84F82F91FEF78FBA544B914603
:100E50001A6CEFE7564BB3F9041001EB8101914690
:100E600049002BF085FE84F82F91FEF77EBA4FF0F3
:100E7000010184F82E1184F83031A4F83A21AFE64C
:100E80009EF80620002A3FF4FDAE4A4B4A491B68F3
:100E900081FB0321DB17C3EBA1014FF400702BF0A2
:100EA00067FE002384F82F31FEF75FBA0A68520705
:100EB0007FF5E8AE414B4FF4887019682BF058FE6F
:100EC000002384F82F31FEF750BA9EF80520002A3F
:100ED0003FF4D8AE3A4A107800283FF4D3AE394BED
:100EE0001B8803EB8303590091FBF0F14FF4116071
:100EF0002BF03EFE002384F82F31FEF736BA0A6845
:100F000097067FF5BFAE9AF8002090077FF5BAAE3E
:100F10001CF0010F1F4E204900F05C84726882EAC9
:100F2000E273A3EBE27303EB5303A1FB0331C908A4
:100F3000002AACBF41F0004141F040414FF4006055
:100F40002BF016FE002384F82F31FEF70EBA9EF820
:100F50000520002A3FF496AE194A107800283FF485
:100F600091AE194B5B7B002B00F09484154B1B88D2
:100F700093FBF0F000EB800041004FF404702BF085
:100F8000F7FD002384F82F31FEF7EFB9B0330408E2
:100F900018C4002020C400201F85EB51F8C3002096
:100FA000A4C30020D0B70020946E002078660020F3
:100FB000FCC30020E0C1002067666666ECC3002029
:100FC0001E6F0020086F0020106F00201CC400203E
:100FD00004C400209EF80620002A3FF453AEC34B01
:100FE0004FF4C06099682BF0C3FD002384F82F31C3
:100FF000FEF7BBB90F68BF067FF544AE9AF800C094
:101000001CF0020F3FF43EAEB94E33896421914685
:1010100001FB03F12BF0ACFD84F82F91FEF7A5B98D
:101020000A68900640F1F180B24BB14E1878317DDC
:1010300000F00203002B0CBF00234FF47A7340F63C
:10104000B83208BF4FF4FA6210F0010F18BF134610
:1010500019444FF482602BF08BFD002384F82F316C
:10106000FEF783B9B4F83A21C2F1FF0293427FF44C
:10107000B3AD4FF0010384F83D31ADE54FF001030E
:1010800084F83C31ACE5FDF7A3FE9B4B1B68C01A0E
:1010900040F6B833984200F21E81DFF89CA29AF81D
:1010A00004303A2B00F0BA8200233B70FEF779B986
:1010B0003868F8F7C3F900287FF48EAD4FF00103CC
:1010C00084F82F318CE5C4F8203184F818318B4F27
:1010D0002BF09CFD94F82431FEF71DB988490620B9
:1010E0001EF028FF002384F83E0184F82F31FEF71C
:1010F0003CB902315EE6012384F8403142F21071BE
:1011000052E6804B1B88D80513D4D90600F17A83A8
:101110009A0600F1F183580600F1F383190700F1F4
:10112000F983DA0700F1148413F0020F0CBF0426D0
:101130000C26754B754A1B78D27803F001030AB16F
:1011400043F00203532004932BF0D8FC704A12881A
:1011500002EB820202EB8202900080B22BF0B2FC22
:1011600000202BF0AFFC6B4A6B4912883868C2EB49
:10117000C212520081FB023111444FEAE27ACAEBFB
:10118000612A5FFA8AFA5146F8F75CF999F800206B
:10119000049B38681E438AEA020A002189F800A0ED
:1011A000F8F750F931463868F8F74CF999F80030FB
:1011B00038687340DBB2194689F80030F8F742F915
:1011C00094F848A1FFF7F2BA013B84F85631FEF7D4
:1011D00017BB013B84F85731FEF72BBC09F1FF39EF
:1011E00084F85F91FFF760BA013F84F85E71FEF703
:1011F000FDBF013B84F85A31FEF713BF47493A203F
:101200001EF098FE2870FEF7E2B8454A12681206F2
:1012100000F1FA82434A127B002A3FF433AD94F87E
:101220004111032900F28A83DFE801F03228190214
:101230003D4B1B6859799A79DB7901F1407101EBDB
:10124000022101EB0341002384F841314FF4826015
:101250002BF08EFC002384F82F31FEF786B8334B39
:101260001A68137A507992781B0403EB0023134415
:101270004A1C84F8412103EB0161E7E72B4B1A6814
:10128000D379107952781B0403EB00231344EFE762
:10129000264B1A689379D07812781B0403EB00234D
:1012A0001344E5E72D22DA762DE4214BDBF800101C
:1012B0001B78C4F81411013B012B3FF625AB10211C
:1012C000022391701371FFF71FBB2BF08FFC0123DA
:1012D0003370FDF7F3BF174AB2F84A3100210133EA
:1012E000A2F84A313970FEF75CB800BFE0C10020B7
:1012F00020C400201CC40020244B00209CC30020DC
:1013000069CB030878660020946E00208066002078
:10131000086F0020ACB7002003082080F19A030872
:1013200070960020106F0020807F0020C86600208B
:10133000C4B700209C2600200C4B0020A64EA74BD3
:1013400000930024A6F13F01A54BA64A0A9106F896
:10135000404CA5490B960CA8F9F7AAFC0A9E731CF1
:101360000A9334700A9B2922591C0A911A700A9B0D
:10137000EA22591C0A911A700A9BC822591C0A9128
:101380000CA81A702EF0D6FB471C0CA93A460A98F6
:101390002FF058FB0A9AD31901330A93D4550A9BAC
:1013A0005A1C0A921C700A9B5A1C0A921C700A9BB7
:1013B0005A1C0A921C700A9B5A1C0A921C700A9BA7
:1013C0005A1C0A921C700A9B5A1C0A921C700A9B97
:1013D0005A1C0A921C700A9B5A1C0A921C700A9B87
:1013E0005A1C0A921C700A9B5A1C0A921C700A9B77
:1013F0005A1C0A921C700A9BFF22591C0A911A70EF
:101400000A9B0122991814A80A911A7050F8283DD5
:101410009B1B337028F03CFB2C70FDF7D8BF8C462B
:101420008946084604910591069107910B46FEF7FF
:1014300019BA9FED6E7A13F0140F08BFF0EE477AD9
:101440007EF4F0AEFEF7F7BE694B1868FFF799B966
:10145000684A614B12680D93A3F14007002103F81D
:10146000401C2123D100BB7040F13A82624903261F
:10147000624B1B885A0500F12982D80700F13E8291
:1014800003F002035E4A002B1CBF03261146DFF85F
:101490008891324648462FF0D5FA06EB090314A886
:1014A0000133A9F1020140F8203D00225B1A06F841
:1014B00009207B7028F0ECFAFEF742B8C4F81C81D2
:1014C00086F80090FDF7FABE434A4E4B0D9214AEDB
:1014D000A2F13D0046F8200D19884B4FA2F14003C0
:1014E00000204FF00A0E02F8400C082283F801E0B9
:1014F00030469A70F9F7DEFA3B684449DA1781FB07
:101500000313C2EBA30399B23046F9F7D3FA0DF0F7
:10151000DDF9BF680C9B3A0C591C0C911A700C9B9E
:101520003A0A591C0C911A700C9B5A1C0C921F7091
:101530000C9B5A1C0C921870304628F0A9FAFDF743
:10154000FCBF334F9FED338AB7F9022022480D903C
:1015500007EE902AF8EEE77A14AE67EE887AA0F1EB
:101560003D01FDEEE77A46F8201D00F8403C0823D7
:10157000CDED037A00F83F3C1E23BDF80C1000F8B7
:101580003E3C3046F9F796FAB7F9003007EE903A4C
:10159000F8EEE77A304667EE887AFDEEE77ACDED31
:1015A000037ABDF80C10F9F785FAB7F9043007EEA5
:1015B000903AF8EEE77A304667EE887AFDEEE77A01
:1015C000CDED037ABDF80C10F9F774FA304628F027
:1015D0005FFAFDF7AFBF00BF14B80020D26600204D
:1015E00030670408386704084467040800000000F6
:1015F000F8C30020C8B700201C67040878660020E4
:101600002C670408086F0020E0C10020676666664A
:10161000FCC3002058A08B41D7B700209AF80240A5
:10162000C4B1013CE4B2013454445146002211F8E3
:10163000013B534083EA0313DBB2120ADE0042EAA5
:1016400003228C4286EA131382EA0302EFD1002AB6
:101650007FF42AADC04AC14EC14B1288C149C24C69
:10166000F261DFF838931A6809689B68F262B4F88F
:101670004A21F066F364D9F80000F163F265F6F7E9
:101680007BFD039000287DF487AE0221D9F800008D
:10169000F7F7C0FE94F84C319AF803200492642BBB
:1016A0004FF0040286F8742040F07C8194F84D31AC
:1016B000072B04BF9DF80C3084F84D3194F84D3160
:1016C000079306EB031ADAF80410039108462EF08C
:1016D00031FADAF8081006915FFA80FA08462EF01F
:1016E00029FAC0B205900AEB0002079B9F480399B4
:1016F00003900832C27123F00F0286468272059869
:1017000003F00F0300EBCA008EF80D3052468EF83E
:101710000E000EF10F002FF095F9954B059A0699E2
:101720000AF1090018442FF08DF90398C37903F1E9
:10173000010ACBB1013B5FFA83FC0CF1080CDFF826
:1017400060E284440023073010F8011B59408B00ED
:10175000CA0883EA410302F018024B404EFA02F233
:1017600053408445DBB2EFD1814A04980AF8023035
:1017700024F082FB94F84D310022013384F84D317E
:1017800084F84C21039BDDF80CA09B785BB11AF820
:101790000510D9F80000F7F755FE01359AF8023028
:1017A000EDB2AB42F3D894F84C310322013384F804
:1017B0004C3186F874203A70FFF7ABB902213868D3
:1017C000F7F728FE94F82431FDF7A5BD4FF0010A84
:1017D000FEF7B2BF326882EAE273A3EBE27303EB77
:1017E0005303A1FB0331C908002AB8BF41F080416F
:1017F000FFF7A4BB5F49881F2BF03CF884F83E013B
:10180000FFF737BA342694E4102300260422184642
:101810000CA98DF830308DF831208DF832608DF8BC
:1018200033608DF834608DF835602BF081F984F8E1
:101830002F61FDF79ABD4B4B1E6806EB86067600BE
:10184000FEF7EFB94C4AD278002A0CBF4FF0040CD7
:101850004FF0050CFEF710BE012338683370F7F720
:10186000E5FD06463868F7F7E1FD72067DF426AD22
:101870008A2851D08E287DF421AD94F81831002BA0
:101880007DF438AD3D4BC4F820312D2384F824314C
:10189000FDF71BBD304B1888FFF76CBB0127FEF727
:1018A000E1B82D499A790B8803EB830303EB83039B
:1018B0009F00BFB2002A00F01181294B1B680FFA6C
:1018C00083FA0DF003F840B2FDF7E0BE03262C4981
:1018D000DDE59C469946184604930593FDF7C2BF83
:1018E000284B294A1B68294903F48003002B16BFA3
:1018F000114604260326BBE524261AE424490426BF
:10190000C5E5102615E4138907EE903AF8EE677ADC
:10191000FEF791BC20260CE41E4B1B689B067DF550
:10192000CDAC94F81831002B7DF4E4AC1A4BC4F81C
:1019300020312D2384F82431FDF7C7BC4B1CDBB2CA
:10194000042B84F841314FEA01613FF47CAC7DE423
:101950000826FFF7EEBB00BF086F0020280000201C
:10196000E0C10020F8C300209C2600205CB30020CA
:1019700062B30020D42700208066002094B80020A5
:1019800020670408709600201C6704081467040888
:101990002467040818C40020C0B80020AC4B002005
:1019A0000007090E96F875A0574905951AF00F0F14
:1019B00004BF0AF1010A5FFA8AFABAF1070F28BFD9
:1019C0004FF0010A4FEA0A1C06EB0C03187C4F4B40
:1019D00003930A18002392F824104C4A93725FFA7A
:1019E0008CF31A464A4B964606EB0C024EEA000070
:1019F00001291870D26803F101000CD90239C9B26B
:101A00008D1C1D44034603F8012BAB424FEA122202
:101A1000F9D101310844B44422F060030AF1010A0B
:101A20009CF811205FFA8AFA1343BAF1080F037089
:101A300000F1010340D04FEA0A1C06EB0C01344AC6
:101A4000087C314901449A1A91F8241055180EF176
:101A5000100E132D5FFA8EFEC6DD059D0398DFF88C
:101A6000BCE0D2B2931DDBB243F04001C17103F17F
:101A7000010CCBB10532D3B20833C31805930EF174
:101A80000100002310F8011B59408B0083EA410339
:101A9000CA084B401F4902F0180241FA02F25340B3
:101AA000059A8242DBB2EDD104980CF80E3086F82C
:101AB00075A024F0E1F965E6154A059D9A1ACDE76F
:101AC000154B6420B3F900A0FDF7E0BD9C46994694
:101AD0001846049305930693FDF7C4BE4FF0FF33F9
:101AE000EDE69C46FDF7BEBE9C469946FDF7BABEA4
:101AF0009C4699461846FDF7B5BE9C469946184641
:101B00000493FDF7AFBE00BFB03304085CB3002000
:101B100069B300200007090EE0C1002062B3002075
:101B20002DE9F047B0F908500D81EDB2442D8AB08F
:101B30000C46164600F06682074642D9812D00F019
:101B4000A48200F29580542D00F0C88040F2F38109
:101B50006E2D00F02582802D40F01081934B93F87C
:101B6000009009F1020919F0FF0900F09480904BF0
:101B7000904F914EDFF870A2994403F101080A25B5
:101B800016E0322D01F0D183A5F13C00C0B213283C
:101B900041F2D28300232268511C21601570226813
:101BA000C84502F101012160137074D018F8015B7F
:101BB0000A2DE6D1BAF80030FF2BA8BFFF23DBB215
:101BC000E9E7052D00F00C821ED8022D7ED040F2F0
:101BD0009F81032D00F0DA81042D40F0CF807749FA
:101BE00020462A46F8F744FF00212046F8F788FFF0
:101BF00022680021531C0125236028462B461170C2
:101C000063810AB0BDE8F087242D5DD040F23681B3
:101C1000282D00F0FF81382D40F0B0800A68684B15
:101C20000125511C21601570226805215019206082
:101C3000117022680A215019206011702268002159
:101C400050192060117022681978501920601170A5
:101C500022685978501920601170226899785319B8
:101C600023602B461170284663810AB0BDE8F087D7
:101C7000A02D17D040F22181B82D00F00482FE2D56
:101C80007CD1504D05F1080635F8021B2046F8F7C7
:101C900037FFB542F8D101252B46284663810AB0AB
:101CA000BDE8F087484B08461968F8F711FF474B25
:101CB00020461968F8F70CFF454B196820460125A6
:101CC000F8F706FF2B46E8E7424BF6E704224249C5
:101CD00020460125F8F7CCFE2B46C4E70B683F4FA2
:101CE000591C012221601A70236800259A1822606D
:101CF0001D70236897F85B20591C21601A702368B7
:101D000097F85A20591C21601A70B7F856102046CF
:101D1000F8F7F6FE29462046F8F7F2FEB7F8581015
:101D20002046F8F7EDFEBD1E07F1480635F8021F04
:101D30002046F8F7E5FEB542F8D12268284B0C2181
:101D4000501C20605D181170226813F8011F501C90
:101D5000AB4220601170F7D123680222591C216028
:101D60001A70B7F85C102046F8F7CAFE0125B7F8DC
:101D70005E102046F8F7C4FE2B4674E7214628463D
:101D8000FAF78CFD002886D1742D00F0F280772DB3
:101D90002CD13B687A689A421BBF5A1C3A600146B4
:101DA0001978104A20462BF091FF74E7056E002049
:101DB00004340408676666664C2E0020D266002054
:101DC000356B0020286E0020107AFF1F147AFF1F49
:101DD000187AFF1F786C0020AC67040824B7002035
:101DE0006DB7002021D20308742E0020F52D01F0DC
:101DF000DA82762D00F0DC813E687968A5F1210356
:101E00008A1B3046362B00F2D382DFE813F08A02B9
:101E1000D102D102D102D102D102D102D102A90252
:101E2000D102D102D102D102D102D102D102D1021A
:101E3000D102D102D102D102D102D102D102780263
:101E4000D102D102D102D102D102D102D102D102FA
:101E5000D102D102D102D102D102D102D102D102EA
:101E6000D102D102D102D102D102D102D102D102DA
:101E7000D1024502D1022002D1021C02202D7FF4A2
:101E80007DAF0B68B64D591C6A7821601A702368C3
:101E90002A78591C21601A702368AA78591C21607D
:101EA0001A7029892046F8F72BFE23686A79591C95
:101EB00021601A702268A9799CE6822D7FF45EAFBA
:101EC0000B68A84AA84D1178A54A581C20601970C3
:101ED00011892046F8F714FEA44B22681B88FF2BBB
:101EE00002F10101A8BFFF2321601370A96881F3EB
:101EF000100189B22046F8F703FE296801F30F01AB
:101F000089B22046F8F7FCFD994B2268197871E6F2
:101F1000012D7FF433AF0B680022591C21601A7029
:101F200023685A1C22601D7022682421531C2360E0
:101F30002B46117097E6522D7FF420AF0A688D4E24
:101F4000531C0321236006F10C0711703346062051
:101F500001212268551C2560117022689F4202F100
:101F600001012160107000F0DC809979D879063386
:101F7000EFE73B687A689A421BBF5A1C3A600146F9
:101F800019787D4A20462BF0A1FE84E60B685A1C86
:101F90000A601D700B680222591C21601A7027E626
:101FA000724B0A681B88704DFF2BA8BFFF23511C82
:101FB00021601370A96881F3100189B22046F8F7F7
:101FC0009FFD6E4B20461988F8F79AFD296801F3AA
:101FD0000F0189B220460125F8F792FD2B4642E613
:101FE0000B2267492046F8F743FD08226549204641
:101FF000F8F73EFD0125072263492046F8F738FD32
:102000002B4630E6002A3FF446AE604B13600125B4
:102010002B4628E60B68DFF894815D4E591C02229E
:1020200021601A70236806275A1C22601F702368DB
:102030000A22591C21601A70236801255A1922604E
:102040001D70B8F800102046F8F75AFDB8F80210D5
:102050002046F8F755FD23685A1922601F7023683F
:102060005022591921601A702368002259192160E1
:102070001A7031882046F8F743FD71882046F8F73A
:102080003FFD2B46EFE5434B17E6434B1E780436E6
:1020900016F0FF063FF4FFAD404B414F1E4403F1E5
:1020A00001094FF00A0824E0B8F1500F01F03A811D
:1020B000B8F15A0F01F05681B8F1320F01F0568194
:1020C000A8F13C00C0B2132841F2548100252946F2
:1020D00023685A1C2260204683F80080F8F710FD20
:1020E00029462046F8F70CFDB1453FF4D4AD19F868
:1020F000018BB8F10A0FD7D12A4B9D68196805EBFF
:1021000085054FF6FF736D009D42A8BF1D4699429D
:10211000A8BF194625EAE57521EAE171ADB289B299
:10212000D6E7214B21681A78481C20600A70002AE3
:102130003FF4B1AD013AD2B202EB420206EB4202E9
:102140005278002A3FF4A7AD0132D5180133226836
:1021500013F8011F501C9D4220601170F7D19AE5C1
:1021600004C400201E6F0020E0C10020086F002082
:10217000C4B700208C6204086DDB0308ACB70020F4
:10218000B4670408C0670408CC670408CDC700081A
:10219000802F00206C680020056E00201434040895
:1021A000842F0020A42E0020EC850020444F002026
:1021B0003B685A1C3A601B78002B01F04E81102BB3
:1021C00007BF724A92E82200054629462268501C41
:1021D000206013702046F8F77BFC29462046F8F76C
:1021E00077FC6B4B20461968F8F772FC20460021FB
:1021F000F8F786FC00212046F8F782FCF8E4072374
:10220000B2FBF3F3C3EBC301521A1CD1DBB203F1EF
:10221000FF385FFA88F8002B3FF43DADDFF874918A
:1022200008F101089246431C3B6090F90010594B9D
:10223000002593F902208A4203F1080301F07B8113
:102240000135062DF5D14FF0FF352B460BE5731CFC
:102250003B6096F80080B8F1FF0F01F09881B8F16B
:10226000FE0F01F055813846F8F7F0FB97E80C00B7
:102270009B1A002B07DD531C3B6013781BB9B8F188
:102280000B0F41F27981B8F1240FDCD8424B0125C4
:1022900023F818002B46E6E4731C3B6030780328D3
:1022A000D1D8431E3D4D3E49DBB203EB430305EB62
:1022B000430308705D7800283FF4EDAC531EDBB299
:1022C000AB42C0D10022C1F80620C1F802208A72B8
:1022D0005BB1581C3B6808444A1C01333B6013F84F
:1022E000011C02F8011F8242F7D12E4B1B78002BF4
:1022F0003FF4D1AC012521F03DFB2B46B3E4731C28
:102300003B6033780A2B01F0F4803846F8F7AAFBDB
:102310003846F8F7A7FB01253846F8F7A3FB2B460C
:10232000A1E43346721C3A601F4D13F8022B6A7009
:102330003B6073782B70F31C3B60B378AB7038460E
:10234000F8F784FB3B682881591C1A46396012F85B
:10235000021B69713A605B78AB7101252B4682E400
:10236000731C3B6033780A2B01F07C80502B40F0CB
:1023700008863846F8F76AFB0C4E30803846F8F786
:1023800065FB012570802B466DE400BF4C2A0020C0
:10239000442C00205891002024B700208C620408AF
:1023A000EC850020042F002004C40020802F002092
:1023B0000B3DEF2D3FF647AF01A353F825F000BFCB
:1023C000752E01084722010847220108472201080B
:1023D0004722010847220108472201084722010835
:1023E0004722010847220108472201084722010825
:1023F0004722010847220108472201084722010815
:102400004722010847220108472201084722010804
:1024100047220108472201084722010847220108F4
:10242000252E010847220108C92D0108472201086D
:10243000A72D010847220108472201084722010869
:102440007F2D010847220108252D01084722010898
:10245000F32C010847220108CD2C0108472201086E
:102460000330010847220108AF2F01084722010865
:10247000FF210108472201084722010847220108DD
:1024800047220108971C010847220108932F0108E1
:102490004722010847220108F730010847220108B6
:1024A000392F010847220108472201084722010865
:1024B0004722010847220108472201084722010854
:1024C00047220108F92E010847220108AB2E010816
:1024D0004722010847220108E53201084722010886
:1024E0004722010847220108472201084722010824
:1024F0004722010847220108193201084722010832
:1025000083300108472201081530010847220108DD
:10251000853101084722010811310108AF2C01085B
:1025200047220108472201084722010847220108E3
:1025300047220108472201084722010847220108D3
:1025400047220108472201084722010847220108C3
:1025500047220108472201084722010847220108B3
:1025600047220108472201084722010847220108A3
:102570004722010847220108472201084722010893
:102580004722010847220108472201084722010883
:102590004722010847220108472201084722010873
:1025A0004722010847220108472201084722010863
:1025B0004722010847220108472201084722010853
:1025C0004722010847220108472201084722010843
:1025D0004722010847220108472201084722010833
:1025E0004722010847220108472201084722010823
:1025F0004722010847220108472201084722010813
:102600004722010847220108472201084722010802
:1026100047220108472201084722010847220108F2
:1026200047220108472201084722010847220108E2
:1026300047220108472201084722010847220108D2
:1026400047220108472201084722010847220108C2
:1026500047220108472201084722010847220108B2
:1026600047220108472201084722010847220108A2
:10267000852C0108472201086F2C01084722010818
:102680004722010847220108472201084722010882
:102690004722010847220108472201084722010872
:1026A0004722010847220108472201084722010862
:1026B00047220108152C0108C32B01088B2B0108A8
:1026C00047220108EF2A0108D52A0108672A0108D4
:1026D000472201084D2A0108E7290108BF290108FE
:1026E000AD2901084F2901084722010821290108C5
:1026F0004722010847220108FF280108D1280108C4
:10270000BD280108952801087528010853280108EB
:10271000272801080F28010847220108472201083D
:1027200047220108472201084722010847220108E1
:1027300047220108472201084722010847220108D1
:1027400047220108472201084722010847220108C1
:10275000F527010847220108472201089B270108A5
:1027600047220108472201084722010847220108A1
:102770004722010847220108472201088127010852
:10278000C04B1B78DB073FF55EAD0125FBF77EF9FB
:10279000FCF740F82B46FFF766BA731C3B603378B2
:1027A0000F2B3FF650ADB21C3A60C3EBC303B64AE1
:1027B0007178D154F11C39601344B2785A70321DCB
:1027C0003A60F2789A70721D3A603279DA70B21D0E
:1027D0003A6072791A71F21D3A60B2795A7106F153
:1027E00008023A60F2799A71012528F065FA2B46C1
:1027F000FFF739BA3846F8F729F9A44EF081384680
:10280000F8F724F90125B0812B46FFF72CBA38469A
:10281000F8F71CF99E4A00EB800043000125138065
:102820002B46FFF720BA3246731C3B60994B12F8D7
:10283000021B19703A6072785A70F21C3A60B278D2
:102840009A70321D3A60F278DA7001252B46FFF754
:102850000ABA3846F8F7FAF88F4E30823846F8F759
:10286000F5F870823846F8F7F1F80125B0822B466A
:10287000FFF7F9B93346721C3A6013F8020B3B605C
:10288000F31C71783B60B27818F072FB00287FF47B
:1028900002AAD8E43346721C3A60804A13F8021B3D
:1028A00011703B60794A73789370F31C3B60784BEE
:1028B000B2789A7001252B46FFF7D5B9784B794944
:1028C00018684E2201252EF0BDF82B46FFF7CBB934
:1028D0003246731C3B60744B12F8021B19703A604D
:1028E00072785A70F21C3A60B2789A703846F8F7EB
:1028F000ADF86E4B0125D8802B46FFF7B4B93846AA
:10290000F8F7A4F8694E30803846F8F79FF87080E1
:102910003846F8F79BF80125B0802B46FFF7A3B99E
:10292000DFF8A88198F80030002B3FF4B4A9604E7E
:1029300000253846F8F78AF819F0E4FE98F80030D8
:10294000A6EC010A01359D42F3DBFFF7A4B90D2A7D
:102950007FF479AC731C3B603578072D3FF673AC80
:10296000DFF86C8138460C26F8F770F806FB05F6A0
:1029700008EB0605A8803846F8F768F8E88038467E
:10298000F8F764F83B6828811A46591C396012F838
:10299000021BA9723A605B78EB723846F8F73EF892
:1029A000012548F806002B46FFF75DB93846F8F7D1
:1029B0004DF8404B012518802B46FFF754B9731C86
:1029C0003B603078060600F130862E4B1B78DD0721
:1029D0003FF561A9032828BF00200125FBF73AF83D
:1029E0002B46FFF740B9731C3B60384696F80090C1
:1029F000F8F714F880463846F8F710F805463846D8
:102A0000F8F70CF806463846F8F720F83846F8F795
:102A10001DF83846F8F726F8B9F1000F00F0F085F8
:102A2000B9F1100F7FF437A9234BC3F800805D6024
:102A30000EB1224B1E602249224B0222081F0125A3
:102A40001A7015F06BFA2B46FFF70DB90D4B1B787A
:102A5000D8073FF520A90125FBF7F4F8FBF7DAFECC
:102A60002B46FFF700B9074B1B78DA073FF513A990
:102A7000154A1378012543F0040313702B46FFF722
:102A8000F2B800BF946E0020CCBA0020544F002052
:102A9000644F0020FC5200201C9300204C96002024
:102AA000C8660020704F04084C4F0020506A002078
:102AB000A8690020F85200204C2A0020442C002055
:102AC000502A0020E65100201CC40020056E002082
:102AD000F4C00020C34B1B78D9073FF5DCA8C24BDC
:102AE0004FF4C87201251A802B46FFF7BCB8092A9B
:102AF0007FF7A9ABDFF828833346721CD8F8005063
:102B00003A6013F8022B2A703B607378AB70F31CA9
:102B10003B60B378642BA8BF6423321D6B713A60AD
:102B2000F378642BA8BF6423721DAB713A603379CC
:102B3000EB71B31D3B607379642BA8BF6423F21D56
:102B40002B723A60B379EB7006F108033B60F379BE
:102B50002B713846F7F77AFF7A683B686881D11A9B
:102B600000290CDD591CD8F800003960521A002ADF
:102B70001978417203DD9A1C3A605B784370012535
:102B80001FF04CFE2B46FFF76EB8984B1868F31CED
:102B900002462136991E396013F8031C1170591E24
:102BA000396013F8021C51703B6013F8011C9170DE
:102BB00003339E4202F10302ECD128F06BFCFFF7D5
:102BC0006AB8731C3B603378894A002B00F00D858E
:102BD000137843F00203B11C1370864D396073788B
:102BE0002B753846F7F71AFF28603846F7F716FFB7
:102BF00068603846F7F72AFF28813846F7F726FF3E
:102C00007D4AE8811378012543F0020313702B46B7
:102C1000FFF729B8C2F34705122D3FF614ABB5B143
:102C20000AAB0DF1020903EB4506C846263E3846BD
:102C3000F7F70CFF28F8020F4645F8D16F4B39F82B
:102C4000022F23F8022FC845F9D1112D09D86C4A5B
:102C50006B00023B13440021223223F8021F9A42E8
:102C6000FBD1684A01231D461370FEF7FCBF664E78
:102C7000002338463360F7F7D1FE012530602B463C
:102C8000FEF7F1BF3346721C3A6013F8025B3B60FB
:102C9000F31C70783B60B178002D00F0AB84012DFF
:102CA0007EF4F9AF0BF0E2FD2B46FEF7DCBF4D4B97
:102CB0001B7813F001017FF4C6AA731C3B603078C7
:102CC00001250BF03DFA2B46FEF7CDBF731C3B6090
:102CD00035781F2D3FF6B7AA052A7FF4B4AA3846E7
:102CE000F7F79CFE494B43F8250014F0FDFAFEF778
:102CF000D2BF464D05F140063846F7F7A7FE3B68C0
:102D0000A5F88000591C1A46396012F8021B85F894
:102D100082103A605B7885F883300435B542EBD198
:102D2000FEF7B9BF731C3A4D3B6033782B723846BF
:102D3000F7F78CFEA8833846F7F788FE28833846D5
:102D4000F7F784FE3B6868835A1C3A601B78EB7483
:102D50007B689A1A032A00F3E1843E689A1B052ACD
:102D600000F3CB849B1B002B7EF795AF731C3B605D
:102D7000337885F8213001252B46FEF774BF731C8C
:102D80003B60244A30781070C91A00297EF783AF5F
:102D9000B31C3B607378003318BF012301255370C7
:102DA0002B46FEF760BF3846F7F750FE1A4E3060EC
:102DB0003846F7F74BFE70603846F7F747FE0125B7
:102DC000B0602B46FEF74FBF144E002333603846E9
:102DD000F7F724FE33680125034333602B46FEF7E3
:102DE00042BF00BF946E0020A07F0020C866002074
:102DF0001CC4002020C40020E45100208E49002083
:102E000090490020B44900206C6800204C650020E7
:102E100090980020FC4F002034460020786C002061
:102E2000807F0020731C3B603578132D3FF60BAA82
:102E3000B31C3B6070782AF083FF00283FF403AA9C
:102E4000BD4B027803F82520F21C3A6003EB8503A2
:102E5000B2785A70321D3A60F2789A70721D3A60F8
:102E6000B6493279DA70086801251FF065FC2B46F7
:102E7000FEF7F9BEB24B102A4FF0000128BF102216
:102E8000196059609960D9601974002A3EF403AF43
:102E90003968013B0A440131396011F8010C03F82B
:102EA000010F9142F7D1FEF7F6BE731C3B6096F816
:102EB0000080B8F1110F3FF6C6A9B31C3B60A14DCD
:102EC000737805F818303846F7F7C0FD40F6CA03A6
:102ED0009842A8BF184640F2EE23984205EB4801FD
:102EE000B8BF18460125A0F2EE222B46192092FB0E
:102EF000F0F24A70FEF7B7BE3346721C924D3A604C
:102F000013F8022B2A713B6073786B713846F7F720
:102F10009DFD3B6828805A1C3A601B78AB7138468F
:102F2000F7F794FD3B6868805A1C3A601B78EB7198
:102F300001252B46FEF797BE731C3B60834B32780E
:102F4000DFF838821A700023C8F800303846F7F7E7
:102F500065FD3A68D8F800307D497E4D0343501C2A
:102F6000C8F80030386013780B723846F7F76EFDFA
:102F700028603846F7F76AFD68603846F7F766FD5F
:102F8000A8603846F7F762FD3846F7F75FFDFEF7B1
:102F900082BE3346721C3A606F4A13F8021B91706E
:102FA0003B607378537001252B46FEF75CBE731CA3
:102FB0003B6033780E2B3FF646A9B21C3A6070781E
:102FC00003283FF640A96549062202FB03F28B184D
:102FD000F51C58713D60B0788854321D3A60F27823
:102FE0005A70721D3A6032799A70B21D3A607279E5
:102FF000DA70F21D3A60B2791A7101252B46FEF79C
:1030000032BE731C3B60524B32785A7501252B46F9
:10301000FEF729BE731C3B60484DDFF864813378AE
:1030200088F8053038462E68F7F710FD30843846AA
:10303000D5F80090F7F70AFD7B683E68A9F81E00F6
:103040009A1B072A00F340839A1B032A00F32F835D
:103050009B1B002B05DD721C2B683A60327883F8CD
:103060002620FAF71DFD21F073FA3D4B1B68002B5B
:1030700000F0B0822868012527F0B2FE2B46FEF74B
:10308000F2BD3346721C3A60DFF8F48013F8022B6D
:1030900088F802203B60334A73781370F31C3B605E
:1030A000314DB3782B71331D3B60F378092BA8BFEA
:1030B00009233846AB70F7F7C9FC3E687B68288067
:1030C0009A1B012A05DD3846F7F7C0FC3E687B688D
:1030D000E881B34240F0C082FAF7E2FC3B687A68CC
:1030E0009A423EF4D8AD5A1C3A601B78EB70012529
:1030F0002B46FEF7B8BD1D4B03F10802711C396069
:10310000317803F8011F9A423EF4C5AD3E68F5E7F9
:103110003346721C3A60164A13F8021BD1703B60AA
:10312000144A73785371F31C3B60134BB278DA7016
:1031300001252B46FEF797BD00500020C8660020F1
:10314000B0660020F84B00206C6A0020FC4F002085
:103150009098002034460020704F002078680020AE
:10316000F84F0020484F00201C9300208F9800202B
:10317000544F002080B90020644F0020786C00205C
:103180004C9600203846F7F761FC3846F7F75EFCAE
:103190003846F7F75BFC3846F7F764FC3B68BC4DF4
:1031A0001946581C2A68386011F8020B82F82C0066
:1031B0003960597882F83610D91C39609B7882F8CA
:1031C00037303846F7F74EFC3846F7F74BFC3846B1
:1031D000F7F748FC38462E68F7F738FC7087384612
:1031E000D5F80080F7F732FC3E687B68A8F8380015
:1031F0009A1B012A0ADD721C2B683A60327883F828
:103200002E203846F7F72EFC3E687B689B1B032B6D
:1032100000F342822868D0E43846F7F717FC0546E9
:1032200014F08AFFFF283EF436AD3F2D00F21D82D8
:103230000DF12808002308F8243DEE0841460DF161
:1032400003008DF80330013614F056FF9DF803306B
:10325000F6B205F00705B34205F1010503D19DF86B
:103260000430AB4203D02946304614F051FF3B688E
:103270007A68D21A012A7EF70EAD5A1C0AA83A6063
:1032800000221D7800F8252D14F02AFF9DF8033048
:10329000AB420AD07F4B1B683BB19A79AA4204D358
:1032A0001B681B690BB1284698473B685A1C3A605B
:1032B000404600221D788DF8042014F005FF9DF88B
:1032C0000430AB423EF4E7AC724B1B68002B3EF47B
:1032D000E2AC1B685B69002B3EF4DDAC28469847E6
:1032E000FEF7D9BC6C4B1B78012B3EF6D4AC731C9B
:1032F00032463B60DFF8C48112F8023B88F80230A6
:103300003A60F31C70783B60CB1A012BB17840F324
:1033100097813846F7F79AFB0125A8F800002B465D
:10332000FEF7A1BC5D4BFEF7E8BE3388FF2BA8BFBC
:10333000FF23DBB2FEF72FBC1CF0F6FC00283EF4A6
:1033400029AC03780A2B2CD8B0F9023087FB031282
:10335000DB17C3EBA2039BB2FF2BA8BFFF23DBB29B
:10336000FEF719BC4E4B5D68FEF7C8BE97E8220019
:10337000FEF7C5BE1CF0D8FC00283EF4A7AE0378CB
:103380000A2B3EF6A3AEB0F90430B0F9061003EBF9
:10339000830383F3500521EAE171ADB289B2FEF7F0
:1033A00097BE0023DBE73B687A689A4260D13D4BC9
:1033B000FF221A704FF000093B4D0AF0D1F949463F
:1033C00020223A4885F800902FF053FE8DF80490A3
:1033D0009DF80430072B00F2FB80DFF8E480334FC8
:1033E0004A469DF8043003EB430308EBC3035B7CC0
:1033F000E3B19DF8043003EB430308EBC303202142
:103400005B699BB19DF8043003EB430308EBC303F6
:10341000586947F82200F6F753FB2B7857F823003A
:10342000F6F70CFC2A780132D2B22A709DF80430EB
:103430000133DBB28DF804309DF80430072BD0D96E
:103440002368591C21601A70002E3EF424AC184BDE
:10345000336001252B46FEF706BC164A92E822008F
:10346000FEF7B4BE3846F7F7F1FA134EFEF785BF04
:103470005A1C19463A600B4811F8022B0270396049
:103480005B784370042A1DD9FF2A7EF4B1AB91E723
:10349000C8660020C4660020636C0020D82E00207F
:1034A000E42E002060290020A9B90020284B00202C
:1034B000F9A5030828520020444F00208CB70020B3
:1034C0005C920020A5490978994205D8022A7EF429
:1034D0008FABFF2B7EF48CAB236801255A19226039
:1034E0001D70002E3EF4D7AB9D4B33602B46FEF78C
:1034F000BABBB31C3B609B4B72781A70F21C3A60EB
:10350000B2785A70321D3A60F2789A70FEF7C3BBF7
:10351000B31C3B607578022D3EF695AE3846F7F742
:1035200095FA914B03EB45034FF0FF35A3F85C0090
:103530002B46FEF798BB09EBC5063846B170F7F786
:1035400085FA3B6829F835001A46591C396012F88B
:10355000021BF1703A605A783271DA1C3A609A783C
:10356000B271181D38600AF1010ADB787371D04519
:103570007EF459AEFEF78FBB7B4B0030984418BFEA
:103580000120012588F84A002B46FEF76CBB38461F
:10359000F7F768FA3B68744E1A46591C396012F8FE
:1035A000021B86F85B103A605B7886F85A30384622
:1035B000F7F74CFAA6F856003846F7F747FA3846B8
:1035C000F7F744FA0125A6F858002B46FEF74BBB47
:1035D0004A4635E765486649664A674B03600125F8
:1035E0000B6013602B46FEF73EBB137803F0FD0320
:1035F000FFF7F1BA012527F0BBFD2B46FEF733BBE1
:103600005E4B1020C3F800805D6025F095FB5C4A9E
:10361000137843F001031370002E3EF43CAB594B7A
:1036200001251E602B46FEF71EBB00F07F0003281D
:1036300028BF002001250BF035F92B46FEF713BB00
:10364000514B1A88012512FB00F22B4692FBF1F236
:10365000A8F80020FEF707BB731C3B6033780033EB
:1036600018BF012388F8073036E50DF104084046FD
:1036700014F01EFDBDF80430AB423FF4F8AD434BEF
:103680001B68002B3FF4F3AD1B689B69002B3FF4D4
:10369000EEAD28469847EAE538462E68F7F7D6F9A2
:1036A000708638462E68F7F7D1F9B086B2E538460D
:1036B000F7F7CCF9A8F80E003846F7F7C7F93E68D7
:1036C0007B68A8F81000C3E43846F7F7BFF9A8F8FC
:1036D0000A003846F7F7BAF9A8F80C0038462E6801
:1036E000F7F7B4F970843846D5F80090F7F7AEF9DB
:1036F0003E687B68A9F82400A6E4731C3B6033781D
:10370000EB723846F7F78AF93B68E8605A1C3A6072
:103710001B782B743E687B68FFF724BB3846F7F7AD
:1037200095F9A8843846F7F791F93E687B68E884F4
:103730009A1B032A7FF712AB3346721C3A6013F8C8
:10374000022BAA773B60737885F820303846F7F76C
:103750007DF93E687B686884FFF700BB056E00203A
:10376000D9C70008356B002024B70020BCBB00205F
:1037700010BC002010C00020F18500082852002055
:103780001CC40020442C00203CC50020C46600203E
:103790002DE9F04F724B734A1C7893B000F59C41B1
:1037A0002031814607911160002C00F024856E4A7B
:1037B0001268904240F227826C4A6D491768DFF820
:1037C000E8B10492013C1C706A4C039107F48057E5
:1037D000002F40F02582039B5B7D002B40F09884F6
:1037E000049B1B681D0400F17387634B9945A37804
:1037F00000F26F83002B40F06F83604B0693049BB5
:103800001F6817F4805940F0F683039BBBF90660EC
:103810005B8B9E42B4BF00260126594B1B6813F0F8
:10382000805300F00782069A127812F0010200F02D
:10383000088203985349408C91ED037A07EE900A71
:10384000F8EEE77AB4EEE77AF1EE10FA81F206804C
:10385000002E40F0FD814C4D95F8A010002940F05D
:10386000F7814A484A49056895F82D5000200860BC
:10387000486088604749002D40F0EB810D70002AB8
:1038800040F0EC81444B1A78002A50D10399BBF9DF
:1038900000E04F8B898BBBF90200BE45CCBF802571
:1038A000002545F040038E45A8BF2B469B0843F0FA
:1038B0008005B842C8BF2B4643F040058842A8BFE8
:1038C0001D46BBF904E0BBF90600AD0845F08003D6
:1038D000BE45C8BF1D4645F040038E45A8BF2B46D8
:1038E0009B0843F0800E284DB842C8BF734643F092
:1038F000400E95F8A2708842B8BF73469F4201F00F
:103900003C81A5F8A42085F8A620244985F8A2309A
:103910000F78002F01F0AD805F2B01F014816F2B29
:1039200000F0F487069B1B78D90740F1B687049B0B
:103930001B4A1B68059203F00403002B40F04685E8
:103940000DF14008174D0023C8F8043005F1500967
:10395000109340F6330A192740F2833629E000BF5E
:103960005C4B00208C490020584B002070960020B2
:103970009098002080660020404B4C00946E002000
:10398000C8B70020206F002064290020C8660020EE
:10399000804F0020D02B00209C6C0020B41E002003
:1039A00018C400200050002030B5002004354D45DB
:1039B00020D0AA78EB789A4217FB0261F6D26A7897
:1039C000043217FB03633BF912205245A8BF52464D
:1039D000B2F5617FB8BF4FF461729142E6DA9A4264
:1039E000E4DC29782429E1D840460435F7F7CEFBFA
:1039F0004D45DED1B04B98E803001F78AF4B83E80C
:103A00000300002F00F039840121AC48F7F7CEFB0A
:103A1000002840F02382E378002B40F01F82A84C5E
:103A200023881DB225F00105AEB2B342268000F016
:103A3000AE86A44D02270E204FF014094FF0FF0868
:103A40002F7085F8019085F8028025F045F83946F9
:103A50009A482688F7F7AAFB002841F0418026F013
:103A600002039BB2B34223800AD0964B1421FF225B
:103A700002250E201D7059709A7025F02DF82688A9
:103A8000914BDFF884A21978DAF804000393B507A4
:103A900008BF81F00201C1F34001F6F7D5F82421F7
:103AA0008648F7F783FB30B9069A1378590744BF65
:103AB00023F004031370059B1B6813F00A0F1DD03D
:103AC00005217E48F7F772FB002800F094862588D0
:103AD0006F0740F1B18779480621F7F767FB0028A7
:103AE00000F076866E0640F1848707217348F7F769
:103AF0005DFB002840F02D83059B1B689D0600F1AF
:103B0000388327886D480C21F7F750FB002800F018
:103B1000C18147F48073BB42238009D0694B0225E1
:103B20001421FF220E201D7059709A7024F0D4FFCA
:103B3000664B1B78082B00F0B9810E2B00F0B68184
:103B4000049B1B685E0544D5614B1B79002B00F07C
:103B5000E18014215948F7F729FB002840F0DF8065
:103B600026F006F8012024F0F9FE90B3DFF89C81DE
:103B700000254FF0CC0902E0DDB2022D29D809FB67
:103B800005F76B1C58F80760002EF5D1C378514A31
:103B900090F9020052F8233001960322009201218D
:103BA000324624F0ABF8034605EB450000EB00106D
:103BB000049353B1314608EB8000CC222FF059FA20
:103BC000049B48F807300135EDB21FF019FF0028BB
:103BD000D3D1069B1B78DD0740F1B3803E493F4AB5
:103BE00001230B701370039BDAF80000197801F0C1
:103BF0000101F6F729F8059B1B685A0700F11181AE
:103C000013B0BDE8F08F364B364A1F68049307F4B3
:103C100080570392DFF8F8B0334C002F3FF4DBAD50
:103C200000212648F7F7C2FA00287FF4D4AD09F046
:103C300031FFD0E578023FF5F6AD069A127802F032
:103C400001022A4D002185F8A010002E3FF409AE94
:103C5000274901200870002A3FF414AEF9067FF5C9
:103C600011AE244A1278D2063FF50CAEB9F1000F1E
:103C70007FF408AE002B7FF405AE7B023FF502AE69
:103C80001D4B1B78002B01F01D841C4B9B78002ED4
:103C900041F055843BB11A4A1A4B12681B689B1AB3
:103CA000002BC1F287841020104D24F015FF012352
:103CB00085F8A130E6E500BF50570020C8B70020C6
:103CC00078660020746A00207CD00020FC4F002021
:103CD000106F0020F0620408956E0020582C002020
:103CE00070960020909800208066002064290020B3
:103CF000D02B00201CC40020B41E0020704F0020D8
:103D0000B4D000200C2E002080D00020EC540020E5
:103D100030B50020069B1B78D8077FF521AF3C20EB
:103D200021F0D6FE00283FF454AF0BF0ABF93C2055
:103D300021F070FE0028F8D1069B1B78DD073FF5C7
:103D40004DAFB94B93F80090B9F1000F5FD1DFF898
:103D50003883B64F18F8030C3E784146A8F10305A6
:103D60001EF0BAFC002800F02B84002E40F07D8469
:103D700005F1080168791EF0AFFC002841F02482AB
:103D8000AB49A87A1EF0A8FC002800F02C84022E73
:103D900041F01E82A749E87B1EF09EFC002841F0FE
:103DA0001B82A549287D1EF097FC002800F02C847A
:103DB000042E41F01582A149687E1EF08DFC00287A
:103DC00041F012829E49A87F1EF086FC002800F078
:103DD0002C84062E41F0F4819A4995F823001EF0B8
:103DE0007BFC002840F09387974995F828001EF047
:103DF00073FC002800F02C84082E40F07287934951
:103E000095F82D001EF068FC002840F02C84904BA3
:103E100001221A701EF0E3FE059B1B685A077FF50E
:103E2000EFAE03201EF082FC002800F0A18623885C
:103E300013F008047FF4E4AE082024F095FF8548D1
:103E4000854D8649864A874BBBF8066000682E8000
:103E5000086014601C6013B0BDE8F08F059B1B6800
:103E60009A077FF5DCAD804C2688F3073FF5F7AD68
:103E700046F001039E4223803FF4F1AD7B4B1421B9
:103E8000FF2202250E201D7059709A7024F024FE26
:103E90002688E4E527F480739BB2BB4223807FF43D
:103EA0003DAE734B1B78082B7FF447AE228822F07F
:103EB00040039BB29A4223803FF442AE6B4B0225F3
:103EC0001421FF220E201D7059709A7024F004FEF8
:103ED00036E60BB90123A370664B06931B201F78AF
:103EE00094F821601EF022FC012E07F001098246A1
:103EF00000F0258607F00203059394F82030DFF8E0
:103F00008C815D4D052B69D8DFE813F05B004F0015
:103F10000600DD000001C200012E04BF052384F865
:103F20002030B9F1000F00F05381039B534FB3F9D8
:103F30001810B8F80030002261F30F0263F31F423B
:103F4000002361F30F0361F31F43CBF804203968AA
:103F50006269CBF800308A42C0F06784012E41F0DC
:103F6000FE82032294F820300592CBE71EF00AFC73
:103F7000012807D1414FB8F802303A68642101FBAB
:103F800003232361BAF1000F04D098F80630002B08
:103F900040F09180012E21D0384F22693B689A422F
:103FA000C0F03186012384F82030012E70D098F8BB
:103FB0000730012B00F0158119F0D2F894F8203069
:103FC000A0E7B9F1000FD1D14FF48060BAF1000F32
:103FD00000F0FB8324F0C8FE00232361059B002B27
:103FE0003FF40DAC059824F077FD049B1F6817F48F
:103FF00080593FF40AAC1D212148F7F7D7F8002873
:104000007FF403AC1F4A039BD2881B8BBBF906606D
:10401000991A8E4240F3018613449E42B4BF002693
:104020000126FFF7FABB00BF956E00209E0000201E
:104030006C69002071690020766900207B6900208E
:1040400080690020856900208A6900208F6900202E
:10405000582C0020F8C30020382C0020442C0020CD
:104060003C2C0020342C002078660020746A00204C
:10407000FC4F0020946E0020D0B70020B4D0002068
:10408000C8B70020506A0020626900206C6A0020D6
:10409000B44F3A68B8F80230642101FB03234FF4AF
:1040A00080600022236184F82020E27024F044FE26
:1040B00094F8203026E719F053F803224FF47A736E
:1040C00084F82020E361A74F2B8843F002032B8064
:1040D00009F0E0FC3A68E36913440422A36184F820
:1040E0002020012E40F09C853B68A2699A42BFF4D3
:1040F00075AF9D4B187820B91EF018FB00287FF48F
:104100006DAF2B8823F002032B80C2E7954FE8E7C1
:10411000039A013BD27D3BF91330002A40F08083A3
:10412000A3F57A73B3F57A7FA8BF4FF47A7323EAC5
:10413000E37307EE903A9FED8D7AF8EEE77A67EE3B
:10414000877A8B4AFCEEE77A17EE903A1380FFF7F6
:104150004CBB884B884AB3F90430884982FB030280
:10416000DB17C3EBA202059B0A801B689D067FF547
:10417000C8AC834B1B78980704D5824E337D042B43
:1041800000F25485278817F0300F3FF4BBAC1020A5
:1041900024F0D2FD202024F0CFFD7B4B2788002285
:1041A0001A707A4A7A487B4E7B4D002111607B4A17
:1041B0003160002329604160816103608360436155
:1041C000C36113605160936053619161D36199E45D
:1041D000644F3B6847F230520323E26184F8203099
:1041E00072E718F0BDFF032240F6B83384F82020B0
:1041F000E3615C4F68E76A4F3B78002B00F09787DC
:10420000684BDFF8B481DFF8B4B1DFF8B4A10393F1
:1042100045465E46049099460EE019F8041098470A
:10422000032C28DC88B93B782AF8020F01349C4221
:1042300005F1040580F2EE80072CE1B23046DBF890
:104240000430EADD984700B2EDE738F824206B88A7
:10425000801A4FF47A719B1A01FB00F040F6CA02F3
:1042600090FBF3F00844904240F2EE23A8BF1046C2
:104270009842B8BF184600B2D5E7DFF848A1DFF88A
:104280004881494D0AF15A064FF0010951461AF882
:10429000010C1EF021FAF8B19AF804009AF80230E5
:1042A0009AF803E000EB400105EB8101013BD1F8F6
:1042B000B42003EB4303434493420DD095F8E02030
:1042C00081F8B0E009FA00F022EA0000C1F8B43049
:1042D000C1F8B87085F8E0000AF1060A5645D5D154
:1042E0003249204A324B334D09681B78D2F800908E
:1042F00008910793A5F1B00A00266B685BB31F789D
:104300004FB3AA68A9EB0202002A0ADB9AF8E02060
:104310000121B14022EA010209F5FA718AF8E02090
:10432000A960079ABAB12A7859780432D2B2002922
:1043300040F09A8203993BF91220098B01F1C800E1
:10434000824240F332849AF8E0109A7841FA06F3F8
:10435000D80740F1C1840136042E05F10C05CCD1FB
:10436000FFF752BBB4D00020B41E0020AAF1823F58
:10437000ACB70020FCC30020676666662C2C0020CA
:104380001CC4002020C40020E6510020D852002088
:1043900088520020A42B0020B42C0020B052002012
:1043A000B04B00209098002064290020807F0020DE
:1043B00049660020142A0020C44B00200858002021
:1043C000622900207968002024340408A84D95F85B
:1043D000AA3053B1069B1B78DE0706D5039BBBF9B9
:1043E00006205B8B9A4200F34D841121A148F6F719
:1043F000DDFE002800F0208295F8AE302BB995F84C
:10440000A83013B93223A5F8AC30012385F8AE30BB
:10441000FFF796BADDF81090974A04921146974A32
:104420000968A2FB092A42F201020A404FEA9A1ADD
:10443000059200F0FD81924D9248934C934A95F875
:1044400000E0007884F800E01070BEF1000F04D0A6
:104450008E4A92F800E08EF0010E854D0F2085F80F
:104460002400002B00F01283894B039E0C931B78D1
:10447000B6F826C00B931C463B78B78C039E854A42
:10448000368B0E962646A2FB0442520802EB4202ED
:10449000B21AD2B2CDF824C001F48051089295F836
:1044A0002580DFF808B2DFF824C20A900AF5967278
:1044B00076460F9105F1280400200692CDF834903D
:1044C000AE46002E00F037823EF910201FFA82F926
:1044D000B9454FEA400103D3099DA94540F26F82D7
:1044E0005CF82020924580F02F823BF90120059D49
:1044F000002D40F04382013098422BF8012004F156
:104500000604DEDB0A98644ADDF834908EF82580D4
:104510000F280CBF012100218EF82400117000F03B
:10452000BC825E4C5E4E5F4F35883868A168626819
:10453000E06045F00405401A9042524F3580534DDB
:104540004FF0010188BF00223970297088BF84F8BC
:104550002120002B00F0B382049A03991768524E71
:10456000B1F824C0B1F818E0504817F48057354628
:1045700040F0C78239460EE06A7802EB820202EB15
:10458000820202F2EE2292B201318B4220F8022B1B
:1045900005F102050ED016F81120002A00F0138252
:1045A000022AE9D00131028820F8022B8B4205F162
:1045B0000205F0D10C9A137801331370FFF708B994
:1045C00008F1050168791EF087F800283FF4D8ABA0
:1045D000012E40F0F98505F10D01A87A1EF07CF856
:1045E000002840F0F5853249E87B1EF075F8002878
:1045F0003FF4D7AB032E40F0EF852E49287D1EF007
:104600006BF8002840F0EC852B49687E1EF064F8BA
:1046100000283FF4D7AB052E40F0E6852749A87F58
:104620001EF05AF8002840F0CB85254995F8230064
:104630001EF052F800283FF4D7AB072E40F06783F6
:10464000204995F828001EF047F8002840F04983DB
:104650001D4995F82D001EF03FF800283FF4D7AB18
:10466000092E3FF4D4AB4FF009094B463CE300BFA1
:1046700064290020C8B7002070960020D34D621036
:1046800068490020E400002049660020E500002081
:104690005D4B0020ABAAAAAAA65700208066002086
:1046A000D0B70020B4D00020F84B002030B5002057
:1046B00071690020766900207B69002080690020F4
:1046C000856900208A6900208F690020604B0020E6
:1046D000CC4DD5F88830A9EB0303002BFFF685A855
:1046E000C94A95F88C30517C079AC5F88820013367
:1046F000C64A039E32F81120B17D03F00F0385F8FE
:104700008C302B4492B292FBF1F283F8902095F812
:10471000901095F8912095F8923095F89C000A44F5
:1047200095F89310134495F89420194495F8953012
:104730000A4495F89610134495F89720194495F873
:1047400098300A4495F89910134495F89A20194422
:1047500095F89B300A44134495F89D1095F89F20D6
:10476000184495F89E3001440B441A4442F30B124E
:10477000642AF17DA8BF642213B209B1C2F16403B7
:1047800007EE903A9FEDA27AF8EEE77AD7E402219D
:10479000A048F6F70BFD00283FF461A92580B70774
:1047A0003FF56EA946F00203B34223803FF468A9A7
:1047B000994B02201421FF2218700E2059709A7014
:1047C00024F08AF92688FFF75BB924F0B5FA03E4F0
:1047D00025F040039BB2AB4223803FF486A98E4B69
:1047E00002251421FF220E201D7059709A7024F0AA
:1047F00073F9FFF77AB9238823F00405ADB2AB4211
:1048000025803FF468A9844B02251421FF220E2045
:104810001D7059709A7024F05FF92588FFF75BB915
:10482000C3F53B6308331BB27AE403230593D1E459
:104830007A4A92F800E008E695F8A830002B3FF499
:104840007FA8069B1B7813F001037FF479A801224F
:1048500085F8A83085F8A920FFF772B8694D0121C5
:1048600085F8A010FFF7F4B9012900F002849AF846
:10487000E0200123B34001361343042E8AF8E030D0
:1048800005F10C057FF439ADFFF7BEB8069B644A0D
:104890001B781060DF0700F1038295F8A61000294D
:1048A0007FF445A8B5F9A430322B7FF740A895F8DE
:1048B000A2200120572A85F8A60000F09984049BC5
:1048C0001B6813F0040302D05A2A00F0E8855D2A21
:1048D00000F0E6845B2A00F026855E2A00F06C85F5
:1048E000562A00F0CD85972A00F08785A72A40F048
:1048F0009E844C49049B0A781B6842F004020A70AB
:10490000494A059203F00403FFF717B8B2F5FA7F9E
:10491000FFF60DA895F8A620002A7FF408A8069BAC
:104920001B780121D80785F8A61000F1C48408F08F
:1049300013FAFEF7FCBF002F3FD05CF82020924511
:104940004FEA4001FFF4D1AD384A384D525C05EBD7
:104950000109002A00F0B880022A47D199F8012005
:1049600002EB820202EB820202F2EE2292B20328F2
:1049700033DD059D12B2002D3FF4BDAD089D24F836
:104980001520B8F1000F03D10B9D022D7FF6B3ADBA
:104990002288B4F80290B4F804804A449044244A2F
:1049A0000FFA88F882FB0852224DA2EBE87225F834
:1049B000018012B24FF001089DE53A464100069D84
:1049C0004CF8205093E5CAB2022A04D9032A7FF496
:1049D000E9AD6246D8E57246D6E5012505FA00F94B
:1049E0000A9D25EA090512B20A9580E53BF80120E7
:1049F000BDE745F04003AB4223807FF4F0AEFFF704
:104A000074B800BF64290020AC7F0020C87F00205C
:104A100014AE2341C8B70020746A00204966002004
:104A2000102E00201CC4002018C40020F84B0020C9
:104A300056555555D429002045F004039D42238046
:104A40000AD0B54B02251421FF220E201D7059708B
:104A50009A7024F041F82588B04BB14AB3F904307C
:104A6000B04982FB0302DB17C3EBA2030B80FFF705
:104A700032B83946AC48F6F799FB00283FF406AF48
:104A800085F8A77008F068F9FEF74CBFA749A84A57
:104A90000C91DFF8C0B2012111701B21A2480593CF
:104AA000F6F784FB059B00287FF43BADA14CA24F99
:104AB000E2683B68A3609B1AC82B00F25A83049BF0
:104AC0001F6807F4805775E5C2B2022A40F2CF8210
:104AD000032A8BD10E9A0F9D002D08BF3A4646E758
:104AE00026F001039BB2B34223803FF458AE0E2060
:104AF0002F7085F8019085F8028023F0EDFF26885D
:104B00004DE600210FE06A7802EB820202EB82029E
:104B100002F2EE2292B20131994220F8022B05F105
:104B200002053FF447AD16F811201AB1022AEAD067
:104B30000288F0E7CAB2032AFAD87246EBE70023EC
:104B40000593FFF7DAB9B2F5FA7FFEF6F0AE95F805
:104B5000A630002B7EF4EBAE069B1B7801210B40A8
:104B600085F8A61000F0E78208F094FFFEF7DFBE9C
:104B7000082024F0E1F8FFF743B8704A7049106844
:104B8000B5F9A420C76981FB07018911FF17781ABD
:104B900000F5FF407F3082423EF7B7AEC91B0A44A2
:104BA00012B2A5F8A420FEF7B0BEC8398A425CDA7A
:104BB0009AF8E0109A7841FA06F3D9073FF5CBABA3
:104BC00052420120099224F09FF87B1E099A162B6D
:104BD00000F24281DFE813F0E301F901CA01220289
:104BE0000F0236029D01880171015A014301400103
:104BF0002202300136029D0188011A010401EE00F3
:104C0000B201D600C00018F0ABFA032240F6B83368
:104C100084F82020E361FFF757BA0126FEF7FDBDB7
:104C20003A68E3691344A361FFF7D8B90A201DF07D
:104C30007DFD27888046002800F05882F90640F163
:104C40004483404D95F8F080B8F1000F7EF45AAFE0
:104C50000D2023F041FF012385F8F0302788B8F1BB
:104C6000000F7FF49EAAFEF74DBF9AF8E0300122B4
:104C7000B24023EA020309F5FA728AF8E030AA602A
:104C8000FFF769BB00212848F6F790FA00287FF467
:104C9000ACAB322385F8AA00A5F8AC30FFF7A5BB72
:104CA000294B1B78002B3EF442AEE378002B7EF4B8
:104CB0003EAE95F8A7300133DBB2032B85F8A73061
:104CC0007EF635AE214B5B7813B9002E7EF42FAE05
:104CD00008F0E0FEFEF726BE002A0CBF01200220ED
:104CE00070E74FF008094B4603EB83031D4487F838
:104CF0000090A978687813F00BFA069B144A1B7889
:104D000001211170D9077FF585A8FEF76CBF4FF020
:104D100007094B46E8E700BF746A0020FCC3002087
:104D200067666666F8520020C8B700205D4B002019
:104D3000A657002080660020B4D0002094B900203F
:104D4000D34D62106429002049660020704F002076
:104D5000582C002030B50020DAF8E400DFF81C877A
:104D600090F8361098F8023011446429A8BF6421E5
:104D700021EAE17180F83610002B40F04B8426F0D8
:104D800089FB74E5DAF8E400DFF8F08690F8371074
:104D900098F802301144FE29A8BFFE2121EAE171F2
:104DA00080F83710002BEAD016201DF01DFDDAF830
:104DB000E400E4E7DAF8E400DFF8C0868178114423
:104DC000C829A8BFC82121EAE171817098F8023092
:104DD000002BD4D014201DF007FDDAF8E400CEE754
:104DE000DAF8E400DFF8948641781144C829A8BFB6
:104DF000C82121EAE171417098F80230002BBED041
:104E000013201DF0F1FCDAF8E400B8E7DAF8E4006A
:104E1000DFF8688601781144C829A8BFC82121EAB3
:104E2000E171017098F80230002BA8D012201DF01B
:104E3000DBFCDAF8E400A2E7DFF84086089898F88F
:104E40000230417911446429A8BF642121EAE1714B
:104E50004171002B40F09383DAF8E4008FE7DAF831
:104E6000E400DFF81886017A98F802301144C82966
:104E7000A8BFC82121EAE1710172002B3FF47FAF86
:104E80000B201DF0B1FCDAF8E40078E7DAF8E40072
:104E9000DFF8E885C17998F802301144C829A8BF25
:104EA000C82121EAE171C171002B3FF468AF0A20EB
:104EB0001DF09AFCDAF8E40061E7DAF8E400DFF8C4
:104EC000BC85817998F802301144C829A8BFC8214F
:104ED00021EAE1718171002B3FF451AF09201DF0EF
:104EE00083FCDAF8E4004AE7DAF8E400DFF88C85BE
:104EF000417998F802301144C829A8BFC82121EA95
:104F0000E1714171002B40F04183112F7FF456AFC6
:104F100035E7DAF8E400DFF86485017998F80230C3
:104F20001144C829A8BFC82121EAE1710171002BF1
:104F300040F07483102F7FF457AF20E70898DFF814
:104F40003C8541781144B1F5967FA8BF4FF4967126
:104F500021EAE171417098F80230002B3FF47CAFF8
:104F600015201DF041FCDAF8E40008E70899DFF8A5
:104F70000C850F791744642FA8BF642727EAE777C9
:104F80000F711DF04BFC98F80230002B3FF464AF1A
:104F9000032039461DF028FCDAF8E400EFE6089813
:104FA000DFF8D88401781144FA29A8BFFA2121EA50
:104FB000E171017098F80230002B3FF44DAF0120F1
:104FC0001DF012FCDAF8E400D9E60898DFF8AC84AA
:104FD000817811446429A8BF642121EAE1718170BC
:104FE00098F80230002B3FF437AF02201DF0FCFB95
:104FF000DAF8E400C3E60898DFF88084C17998F80D
:105000000230114481F30801C171002B3FF424AF39
:1050100005201DF0E9FBDAF8E400B0E6089BDFF8B4
:105020005C84997998F8020011446429A8BF64212E
:1050300021EAE1719971002840F0B0820D2F7FF4D0
:10504000FDAE09E7DAF8E400DFF83084C17898F8BB
:1050500002301144C829A8BFC82121EAE171C170FA
:10506000002B40F084820F2F7FF4D4AE87E60E9A97
:105070007DE43BF912209978B2F5617F4FF4966395
:1050800093FBF1F34ADB40F633019142A8BF11468E
:105090000C2FA1F5617191FBF3F100F08381182FC2
:1050A0007FF4E5ABC9B2C8290B46A8BFC823DAF81C
:1050B000E400C27DDFB297423FF4D9AB9A1ADFF821
:1050C000BC83C77548BF0732D71098F80230013744
:1050D000FFB23BB9002F3FF4CAAB384623F014FEB1
:1050E000FFF7C5BB18201DF07FFBF3E7FA0600F1C0
:1050F0004F810B201DF01AFB002840F01881BB06E1
:1051000000F15281C34D95F8F030002B3FF4A0AD73
:10511000B8F1000F7FF445A8FEF7F4BC0C2F00F0A7
:10512000EA80182F7FF4A3AB00210B46BFE7BA4AF1
:105130000392FFF771B9B949096811F4003140F0E1
:105140003F810B46B648C65C0F2E03F10C031ED000
:1051500001311529F7D1049BB2491B680591FA3A30
:10516000A5F8A420002203F0040385F8A620FEF78A
:10517000E4BBAD4A049B1F68138823F0040313802B
:10518000012307F4805784F82130FFF713BAA74EA4
:10519000D6F800E04B00BEF1000F07D05F1800EB1F
:1051A00087079EF801E07F787745D4D20B44A04F63
:1051B000A04900EB8300002330603B800B60CAE70E
:1051C0004FF006094B468FE54FF001094B468BE542
:1051D0004FF002094B4687E54FF003094B4683E544
:1051E0004FF004094B467FE54FF005094B467BE540
:1051F000914B92491A684FF47A73B3FBF2F3C3EB05
:10520000431203EB8203049A1268DB001206A1F832
:10521000B43000F1E580834B05931B685F0700F114
:10522000D680049B1B6803F00403FEF786BB0021B5
:10523000BB2A109100F08081B72A00F07981BE2A44
:1052400000F07481BD2A00F04D81792A00F0DB81E5
:105250007A2A00F0D1819E2A00F0C8819D2A00F0B0
:10526000BE81AE2A00F00182AD2A00F0F781EF2A5C
:1052700000F0EE81FD2A00F0E581FB2A00F0DC81E0
:10528000FE2A00F0D381F72A00F08E817B2A7EF47B
:105290004EAB4FF4FA61022008F052FFFEF747BB15
:1052A000674B00220120674D67492A700B6023F08D
:1052B0002BFDFEF73CBB049B64491B680A60594AFE
:1052C000059203F00403FEF738BB102023F04CFDD9
:1052D000202023F031FD5E494E4D081F12F01EFEC6
:1052E0005C4B02221A7095F8F030002B00F03B81E5
:1052F0002788FEF756BF00273946524B09915B7845
:10530000BB423FF4B4AADFF87481384609F0CAFA08
:1053100098F8023009991BB1C9B20C201DF064FA4B
:105320000137FFB2D6E64C4B01220220BBE74B4AC5
:105330004B4B528993ED007A07EE902AF8EEE77A0C
:10534000B0EEC77AB4EEE77AF1EE10FA7FF5D7AE99
:1053500093ED017AB0EEC77AF4EEC77AF1EE10FA67
:105360007FF7CDAEBB063FF5CDAE2A4D202023F012
:10537000FBFC29467268336841F8EC2F05F1E80020
:10538000C5F8E83012F0CAFD324B01221A70AAE7C4
:10539000102023F0D1FC2F4B278883F800804FF09A
:1053A0000108A6E6CFB2A8E7202023F0C5FC294BD0
:1053B000184D00221A7096E72A4B0222032072E74A
:1053C00029490978032900F0C5801946BAE6049BEB
:1053D000264A1B680A21118003F00403FEF7ADBAC8
:1053E000234B1B789B077FF516AF224B1B7D042BAD
:1053F0007FF611AF12F01DFD0DE7049B1E4A1B68DE
:105400004FF4C8711180074A059203F00403FEF7B8
:1054100094BA00BF64290020909800206C68002096
:10542000A054040818C40020D0B700207C2B002012
:105430001A2C00201C2C0020609600200CC7002095
:105440004A6B0020CC660020C8660020102E002089
:105450002C520020E6510020986B00207C52002046
:10546000206F0020E66B0020C4B700209E7F002044
:105470001CC4002020C40020A07F00208CB7002086
:105480000DF0E2FEF5F7D8F80DF0C6FEF9F7C2F917
:10549000012023F039FC95F8A220FFF724BA95F8F3
:1054A000A820002A40F0938095F8AA3083F00103E9
:1054B00085F8AA30002B40F085800C2023F00CFBEF
:1054C000FEF735BA002E3EF4EEAB6B4D95F8A130E9
:1054D000002B3EF4D7A923F0E3FA002385F8A1308E
:1054E000FEF7D0B94FF6FE73644A65489689059079
:1054F000D089334401449381D1810DF0A5FEF5F7A5
:105500009BF80DF089FEF9F785F9012023F0FCFBEB
:10551000049BB5F8A4201B68FA3A0021A5F8A42042
:1055200003F0040385F8A610FEF707BA0223DBE7B1
:105530000B464FF6FE71D7E70B460221D4E7002B4E
:10554000C3D05049504A09684FF47A7000FB0313E6
:105550001360BAE723F0A4FAB5F9A420FBE503230E
:105560000593FEF73FBD4FF00108FFF771BB0F2019
:1055700009921DF039F9DAF8E400099A73E50E2072
:105580001DF032F9DAF8E400FFF7F9BB11200992B7
:105590001DF02AF9DAF8E400099AB6E40D20099220
:1055A0001DF022F9099A49E50021042008F0C8FD00
:1055B000FEF7BDB9304D08F06DFA002385F8A13033
:1055C000FEF760B90B2023F087FAFEF7B0B92C4A3A
:1055D00085F8A81085F8A9000592FEF7AEB900215C
:1055E000FF202BF0E1F995F8A2203AE601202BF0FC
:1055F000DBF995F8A22031E6244A137A43F001033F
:105600001372FEF794B9214A137A23F0010313723F
:10561000FEF78DB917201DF0E7F81DE41020099260
:105620001DF0E2F8DAF8E400099A83E4002103208F
:1056300008F086FDFEF77BB90021022008F080FD0E
:10564000FEF775B90021012008F07AFDFEF76FB969
:105650000021084608F074FDFEF769B9FF2100201B
:105660002BF0A2F995F8A22001E6012100202BF0F1
:105670009BF995F8A220F7E564290020544F0020FB
:1056800018C40020B4D000200C2E00208C5700201D
:105690002DE9F0478C4B1B78DB07074644D58B4B35
:1056A0008B4D1C788B4E012C59D01CD3022C07D16A
:1056B00089498A4A09881288914201D901241C70BB
:1056C000EB7AE3B12B89D3B1854B1B78BBB109F0E1
:1056D000FDF8002800F09B802B7B83422CBF01212A
:1056E000002131700CE07C497E4A098810886A7B71
:1056F000801A8842E2DAEB7A0024002BE2D131787A
:105700002A79632A06D8022C774E00F0BA803378C3
:10571000002B5DD1754AAB7A8C4238BF0C461470B1
:10572000002B4CD1BDE8F0876B4B694D19885B8825
:10573000E878CB1A83EAE3728142A2EBE3721DD3CD
:105740002B788B421AD3614B1C78E01E012861D95B
:105750006749097802294FD0012C5E4EA5D15F4AD6
:105760005D491288687B0988121A914239DD5D4AC9
:1057700012888A42A4D200241C70A1E7B1EB400F2A
:10578000E1DC524B1C78E11E012940F29480022A90
:10579000DEDC57494F4E0878DFF84481DFF844C11A
:1057A000DFF838E100210324022834701C7088F8E7
:1057B0000010ACF80010AEF8001081D11FE0012CF1
:1057C00071D0022C0BD10720BDE8F04723F084B93B
:1057D0007068381A474B984258DD72709AE7BDE8F6
:1057E000F08702241C706BE7022AD2DD4049097859
:1057F00002294FF0040464D13949364E09783E48F5
:10580000022ACCBF00220122C28081804BE7022104
:10581000317075E7022A9BDC95F800C091FBFCFC17
:105820000CF1010CBCF1080FDFF8B4A0304EA878E1
:1058300095F801E096F800802A4CDFF8A090254EFC
:10584000A8BF4FF0080C8AF800C01FFA8CFA10FBB2
:105850000AF01EFB0AFE80B2DFF88CA02080A9F8B7
:1058600000E000244FF0640EB8F1020F34701C7099
:10587000CAF804408AF801E07FF439AF0FFA8CF1DE
:10588000BDE73078A0B9012377603370C2F16402BC
:105890001A4B00FB02F083FB0023C017A0EBA350C0
:1058A0006430707036E70820BDE8F04723F014B983
:1058B0007368F81A8EE7032C96D10D4909780229EE
:1058C0009AD0044EFCE600BF946E00209C2E00206F
:1058D00004C40020A22E0020086F0020A02E00206B
:1058E0001E6F00209E2E0020242C0020C4B7002014
:1058F000246E00207F969800286E00206BCA5F6B94
:105900002DE9F04F2DED0A8B404B1B7893B0012B06
:10591000039001F0C4803E4C94F80021002A41F02D
:10592000CF80072B01F0D6804FF0000ADFF8ECB0F3
:10593000DBF8043058469847002800F06F81BBF828
:10594000B46000228BF85520002E40F06887BBF928
:105950003C50DBF82410BBF93E00DBF82820BBF9F3
:105960004030691ACBF830102A490191821ADBF8CD
:105970002C00CBF834200D461B1A9BF85610CBF8A0
:1059800038300BF130000FF049FF2B68990040F1DF
:10599000E980DBED0D5ADBED0C7A1F4A94ED416A8C
:1059A000D4ED426A94ED437AD4F810311268B8EE1F
:1059B000E58ADBED0E5AF8EEE77AF8EEE58A013378
:1059C00077EE867A38EE268A78EE878A9342C4ED9F
:1059D000417A84ED428AC4ED438AC4F8103101F063
:1059E000FD820A4B1E78142E02F0B1840023D4F8F5
:1059F00018510293062D00F2A880DFE815F0071376
:105A0000F6121B128B1211003114CA13246E0020DF
:105A1000582A002070960020244C00200CC700203B
:105A2000D74B1A78D4F81C71DFF8BCE39FEDD57A18
:105A3000F8000EEB000383ED007A002A7AD0D249F9
:105A4000B0EE476AF0EE476A0023F1EC017A0133C9
:105A500067EEA77A05EE903AB4EEE77AF1EE10FA27
:105A6000F8EEE55AB8BFB0EE677A9A4276EEA76ACA
:105A7000A7EEA56AE9D1F5EEC06A0EEB0003F1EEE0
:105A800010FA83ED007A55DDC6EE265ABF4BC04AA8
:105A90001288F7EE007A75EEE75AD3ED007A65EEDC
:105AA000A77AFDEEE77A17EE903A812B43F327832E
:105AB0009342A8BF134607EE903AF8EEE77AB54B4B
:105AC000C11903EB810393ED057AD3ED003A93ED11
:105AD000066A93ED014AD3ED046AD3ED034A93EDD0
:105AE000025AA3EEA77AA4EE276A66EEC76AA7EE6B
:105AF000646ABDEEC77AE5EE276A17EE101A8129AF
:105B000083ED056AC3ED066A43F3F6828A42A8BFB5
:105B10000A4607EE902AF8EEE77AFCEEE77ACDED3A
:105B2000047ABDF810300EEB0002938017B9132EE3
:105B300003F0B687152E42F0CF817044DFF8AC82B7
:105B4000838828F81730D4F81851934B013583FB1C
:105B500005235A19EB17C3EBA203C3EBC303ED1ADA
:105B6000C4F818518D4B1B78002B01F0EF808C4D41
:105B7000CDF808A0DFF87882DFF87092DDF804A095
:105B800005F2DC670026874BDBED087A1B78172BC4
:105B900001F04E8495ED007AB8EEC78A082B28EE06
:105BA000278A07D1B0EE480A01932BF055F9019BE3
:105BB00029F81600DAF8002092000BD5002E04F028
:105BC0001981B0EE480ADBF8783707F17000984782
:105BD000B0EE408AB0EE480ADBF89836A7F17000C4
:105BE0009847DBF80837384698476E4B1B78032BED
:105BF000B0EE408A01F0FB83D5F85C06DBF8B830E4
:105C0000B0EE480A98470136032E07F12407A8ECA6
:105C1000010A05F10405B6D1DDF808A0614B1F7833
:105C2000072F00F0BC8694F828310493002B40F035
:105C3000C4865D4B5B79002B40F0EB850123594A0C
:105C400084F828311278072A01F08486002306930D
:105C5000564B94ED4C9A93ED007A554BDFF89481B6
:105C6000D3F800A0534B0293F7EE007A37EEC9BA8F
:105C700008F11C032BEE07BA0025B4EEE7BAF1EEEB
:105C800010FA0593D4ED4BBA4B4BDFF86CB1DFED56
:105C90004B8A9FED4BAADFED3BAADFED4A9ADFF876
:105CA0005C91494F019388BFB0EE67BA2E46474BCF
:105CB00098ED008A2B44D3ED007AF5EE407AF1EEB0
:105CC00010FA17D0424B2B44D3ED006A38EE667AB7
:105CD000B0EEC76AF4EEC67AF1EE10FA08D5B5EE6A
:105CE000C07AF1EE10FACCBF37EEA68A36EEE78A1C
:105CF00083ED008A374B1A88930700F08180022ECB
:105D00007ED0354B9AF82E1033F9163007EE103A44
:105D1000059B07EE901A2B44F8EEE76AB8EEC77AB7
:105D2000D3ED007A4B42A6EEA77A700007EE903AC8
:105D3000F8EEE77AB4EEE77AF1EE10FA0AD407EE5D
:105D4000901AF8EE677AF4EEC77AF1EE10FA88BF8F
:105D5000F0EE477A214B22490344085EB3F90C3038
:105D6000C01A07EE100AB8EEC77AD007E7EE687AD5
:105D700040F12B861B4B93ED008A27EE888A3FE08B
:105D80002A4C002000000000582A00202C4C002043
:105D9000284C0020604E0020932449921C4C002087
:105DA0003CC70020246E00204C96002064C00020D8
:105DB000C866002060960020744F0020CDCCCC3DFA
:105DC000AE47813F0000C842804F002058C00020ED
:105DD000982B002078660020A42B0020544F002030
:105DE000FCC3002040C00020484E0020286E002048
:105DF000649600208C2B0020B8BB00208C4F002024
:105E0000029B94F868212B44D3ED01CA38EE6CCA8A
:105E1000002A3DD0D34BD4F86C2103991B688A1A11
:105E20009A4235DD9AF84830022B01F0CA85022EDD
:105E300003F06787CC4B1B68990740F16E87CB4B0B
:105E4000CB49DFF8A0E331F916C09EED008ADFF8F8
:105E500098E3C7ED00AA03EB460028EE288AB0F9C4
:105E60000C00A0EB0C0007EE900AF8EEE77ADEF8E3
:105E7000000027EE888A904238EE6CCAC1F2838017
:105E8000F7EE007AB4EEE79AF1EE10FA01F15280E3
:105E9000B84B2B4493ED000A019B2BEE800A022E97
:105EA00020EE0C0AA3EC010A019303F05287B24BD7
:105EB0009BED007AD3ED007AB04BD7ED006A93EDFD
:105EC000006AAF4B67EE277A2B4427EE8B7AD3ED2F
:105ED000007A67EE277AF0EE665AECEE275AB1EEBA
:105EE000467AF4EEC75AF1EE10FA08D4F4EEC65A28
:105EF000F1EE10FA8CBFB0EE467AB0EE657A94ED12
:105F00004C6AF7EE007AB4EEE76AF1EE10FAACBF35
:105F10000123002343B1F0EEE66AF0EEC77AF4EE17
:105F2000E67AF1EE10FA01D587ED007A022E03F041
:105F3000E186944A944B52F826001B68B0EE6C0A36
:105F40009847924A924B52F826001B6898479AF855
:105F5000373023B18F4B1B88002B00F0C085B0EE8B
:105F60006A8A8D4B9BED007A38EE400A2B4493ED04
:105F7000008A83ED000A9AF8483030EE480AC0EEF5
:105F8000077A2BB3854B1B78DB0721D5B7EE007A58
:105F9000B4EEC79AF1EE10FA04DB94F86831002BE6
:105FA00000F06F87D4F86C31039AD31A6D4A1268E7
:105FB0009A420DDD7A4B93ED007AB0EECCCAB4EE86
:105FC000C7CAF1EE10FA40F1FA87002384F868316D
:105FD000744B94F878212B4493ED007A2BEE877A5A
:105FE00067EE277AC9ED007A32B9019BC7ED00AAA6
:105FF00043ED01AAC9ED00AA0136032E08F10408F9
:1060000009F1040907F1040705F104057FF44FAE17
:10601000654B1B78072B01F02182012B01F09F8437
:106020000023029394F88031002B40F0A1855F4B50
:106030005F4A1B68126813F4805C92F82C2040F0D1
:10604000AE865C495C4891ED006A408B5B4984ED0B
:10605000646A91ED007A5A4984ED657A07EE900AF8
:10606000F8EEE76AD1ED037A564984ED626A37EEBD
:10607000467A77EEE67AD1ED006A84ED617A012105
:1060800084F89811C7EEA65A4F48504990ED005A2F
:106090004F489FED506A90ED004A4F48DFED4F6A40
:1060A000D0ED004A91ED007A35EE045AF7EE007A11
:1060B000F4EEE75A35EE245AF1EE10FA88BFF0EE0E
:1060C000675A25EE065AF4EEE65AB1EE476AF1EE4B
:1060D00010FAB4EEC65AB8BFF0EE665AF1EE10FAF6
:1060E000C4ED675A01F10780B4EEC75AF1EE10FA19
:1060F00088BFB0EE475A3449DFED366AD1ED017AF8
:10610000334991ED014A344977EE847AD1ED014A61
:1061100077EEA47A67EEA67AB4EEE76AF1EE10FAAB
:1061200008DCB4EEE77AF1EE10FA8CBFB0EE676AE5
:10613000B0EE476A2449DFED276AD1ED027A24499F
:10614000D1ED024A264977EEA47A91ED007A67EE06
:10615000A67AB1EE473AF4EEC37AF1EE10FA4ED4D5
:1061600044E000BF6CC0002018C40020544F002041
:10617000FCC3002014C00020A000002088C0002024
:1061800020C00020C0BB0020BCBB002014BC0020ED
:1061900010BC002078660020C82B0020946E0020E0
:1061A00078C000202CC00020246E002070960020B3
:1061B000C866002058C5002090980020384F002065
:1061C000206F0020586A0020744F00208CC00020EF
:1061D000804F00206F12833A8C4F00200000000097
:1061E00090C0002040C0002068C00020F4EEC77AB4
:1061F000F1EE10FA8CBFB0EE473AB0EE673AED49D7
:10620000497809B9B1EE433A002A41F04B82F7EEE2
:10621000003ADFF8C8B39BF80020002A02F045825C
:10622000E549DFEDE67AD1ED024AD1ED016A91ED63
:10623000037A66EE244AE5EE264AE3EE074A63EE69
:10624000A44AF4EEE74AF1EE10FAB4BFB0EE674AA2
:10625000B0EE644A98BFF0EE647A012ACDED0A4AA6
:1062600002F0448291ED067AD1ED052AD1ED076A5C
:1062700026EE077AA5EE227AA3EE267A23EE877A17
:10628000B4EEE77AF1EE10FAB4EEC47A8CBFF0EE19
:10629000676AF0EE476AF1EE10FA88BFF0EE676ABF
:1062A000B4BFF0EE447AF0EE477A022A8DED0B7A15
:1062B00000F0DE8091ED0A7AD1ED092A91ED0B4ACA
:1062C00026EE077AA5EE227AA3EE047A23EE877AE9
:1062D000B4EEE67AF1EE10FAB4EEE77A8CBFB0EEE7
:1062E000664AB0EE474AF1EE10FA98BFF0EE446A03
:1062F000A8BFF0EE477A032A8DED0C7A00F0B88043
:1063000091ED0E7AD1ED0D2A91ED0F4A26EE077A26
:10631000A5EE227AA3EE047A23EE877AB4EEE67A2B
:10632000F1EE10FAB4EEE77A8CBFB0EE664AB0EE4A
:10633000474AF1EE10FA98BFF0EE446AA8BFF0EEBB
:10634000477A042A8DED0D7A00F0928091ED124A81
:10635000D1ED112A91ED137A26EE044AA5EE224AD8
:10636000A3EE074A23EE844AB4EEE64AF1EE10FAB1
:10637000B4EEE74A8CBFB0EE667AB0EE447AF1EE46
:1063800010FA98BFF0EE476AA8BFF0EE447A052AEB
:106390008DED0E4A6CD091ED164AD1ED152A91ED96
:1063A000177A26EE044AA5EE224AA3EE074A23EE08
:1063B000844AB4EEE64AF1EE10FAB4EEE74A8CBF36
:1063C000B0EE667AB0EE447AF1EE10FA98BFF0EED5
:1063D000476AA8BFF0EE447A062A8DED0F4A47D0EF
:1063E00091ED1A4AD1ED192A91ED1B7A26EE044A55
:1063F000A5EE224AA3EE074A23EE844AB4EEE64A0B
:10640000F1EE10FAB4EEE74A8CBFB0EE667AB0EE69
:10641000447AF1EE10FA98BFF0EE476AA8BFF0EEAA
:10642000447A072A8DED104A22D091ED1E7AD1EDE3
:106430001D2A91ED1F4A26EE077AA5EE227AA4EED8
:10644000037A27EE237AB4EEE67AF1EE10FAB4EE90
:10645000E77A8CBFB0EE666AB0EE476AF1EE10FAEA
:106460008DED117A98BFF0EE466AA8BFF0EE477A3C
:1064700077EEE67AF7EE006AF4EEE67AF1EE10FADD
:10648000C4ED4C7A43F3A88286EEA77A022ADDEDAA
:106490000B7A67EE244A67EE877ACDED0A4ACDED96
:1064A0000B7A2DD0DDED0C7A67EE877A032ACDEDDD
:1064B0000C7A25D0DDED0D7A67EE877A042ACDEDD2
:1064C0000D7A1DD0DDED0E7A67EE877A052ACDEDC7
:1064D0000E7A15D0DDED0F7A67EE877A062ACDEDBC
:1064E0000F7A0DD0DDED107A67EE877A072ACDEDB1
:1064F000107A05D0DDED117A27EE877A8DED117ACD
:106500002F49096811F0805800F0A387F6EE005A71
:10651000C4ED675A002A02F0BF8094F99801D4EDC7
:10652000654A284D284994ED646A284E284FDFF8C3
:10653000B0E0B5F81AA0C978B6F9069097ED005A00
:106540009EF800E0D4ED616AD4ED627A07EE100A9D
:10655000FDEEE44A1F4814EE905A0078FDEEC64A5C
:1065600003F0100603F4800300F00107B8EEC77AC9
:1065700014EE900A0193002941F0D4800E49002EB8
:1065800040F0898791ED006A9DED0A5A124B25EE85
:10659000866AA5EE076AB0EE675AA6EE265ABDEEE9
:1065A000C56A16EE10EA16EE106AAE45A8BF2E4672
:1065B00018E000BFFC4F0020C86900200000000068
:1065C000C8B70020909800208066002030B50020D9
:1065D000A4690020946E0020D44F0020056E002096
:1065E000409300207045C8BF064606EE106AB8EE1C
:1065F000C66A012A83ED006A00F0DC8091ED046A2E
:106600009DED0B5A25EE866AA5EE076AB0EE675A35
:10661000A6EE265ABDEEC56A16EE10EA16EE106A10
:10662000AE45A8BF2E467045C8BF064606EE106AA6
:10663000B8EEC66A022A83ED016A00F0BB8091EDD4
:10664000086A9DED0C5A25EE866AA5EE076AB0EE43
:10665000675AA6EE265ABDEEC56A16EE10EA16EE89
:10666000106AAE45A8BF2E467045C8BF064606EE66
:10667000106AB8EEC66A032A83ED026A00F09A80B7
:1066800091ED0C6A9DED0D5A25EE866AA5EE076A1E
:10669000B0EE675AA6EE265ABDEEC56A16EE10EAAF
:1066A00016EE106AAE45A8BF2E467045C8BF064616
:1066B00006EE106AB8EEC66A042A83ED036A79D042
:1066C00091ED106A9DED0E5A25EE866AA5EE076AD9
:1066D000B0EE675AA6EE265ABDEEC56A16EE10EA6F
:1066E00016EE106AAE45A8BF2E467045C8BF0646D6
:1066F00006EE106AB8EEC66A052A83ED046A59D020
:1067000091ED146A9DED0F5A25EE866AA5EE076A93
:10671000B0EE675AA6EE265ABDEEC56A16EE10EA2E
:1067200016EE106AAE45A8BF2E467045C8BF064695
:1067300006EE106AB8EEC66A062A83ED056A39D0FD
:1067400091ED186A9DED105A25EE866AA5EE076A4E
:10675000B0EE675AA6EE265ABDEEC56A16EE10EAEE
:1067600016EE106AAE45A8BF2E467045C8BF064655
:1067700006EE106AB8EEC66A072A83ED066A19D0DB
:1067800091ED1C6A9DED115A65EE865AE7EE055AA9
:10679000E6EEA57AFDEEE77A17EE901A8D42A8BFD5
:1067A0000D468842C8BF054607EE905AF8EEE77AD4
:1067B000C3ED077A2FB922B19200D649D6482AF004
:1067C00041F9D64B1B68002B40F0AE84D44B1B78AC
:1067D00093B19BF8000060B1CF4ED24F0025E8B2D4
:1067E0003B68B6EC010A98479BF8000001358542EA
:1067F000F5DBCD4B1B689847CC4B1B78072B00F083
:106800004286012384F8003113B0BDEC0A8BBDE849
:10681000F08FC74B1B78013BDBB2FFF710BAC54BBB
:1068200002934FF47A751B68B5FBF3F3C3EB431582
:10683000C149DFF8388391F80190BC49B8F90600E6
:106840000F7803EB8503DD00ADB2AE4201F0938615
:10685000DBF88810BBF93CE0DBF86C304A1C07EE33
:1068600090EA7344012ACBF88820CBF86C30F8EE1C
:10687000E77A01F08D86DBED1E5ADBED206A07EE2C
:10688000102A37EEE56AB8EEC75A012E86EE057A71
:1068900037EE257A77EEC77A8BED1F7AE7EE866AB8
:1068A0008BED1E7AF0EE667ACBED216ACBED206A95
:1068B00002F05E80DBF89C10BBF93EE0DBF8703044
:1068C0004A1C07EE90EA7344012ACBF89C20CBF8CF
:1068D0007030F8EEE77A01F07686DBED235ADBEDD7
:1068E000256A07EE102A37EEE56AB8EEC75A012E80
:1068F00086EE057A37EE257A77EEC77A8BED247A25
:10690000E7EE866A8BED237AF0EE667ACBED266AA7
:10691000CBED256A02F05580DBF8B010BBF940E002
:10692000DBF874304A1C07EE90EA7344012ACBF876
:10693000B020CBF87430F8EEE77A01F05F86DBED3B
:10694000285ADBED2A6A07EE102A37EEE56AB8EE20
:10695000C75A012E86EE057A37EE257A77EEC77A8A
:106960008BED297AE6EE276A8BED287AF0EE667ACF
:10697000CBED2B6ACBED2A6A02F04C80A8F806001A
:10698000BBF8B430694A013B1778ABF8B4300299D0
:106990000023072F4B608B60CB607FF444A9F8F78E
:1069A00017FADFF8C88194F828310493A0EB0A00A5
:1069B000A8F80000002B3FF43CA9013B84F82831E3
:1069C00013B0BDEC0A8BBDE8F08F94ED577AB1F9A6
:1069D0000000D4ED586AB1F902E0584AF4EEC76AF3
:1069E00080EAE0738EEAEE71A3EBE073F1EE10FA49
:1069F000A1EBEE71B4BFB0EE476AB0EE666A8B42AF
:106A0000B8BF0B4607EE103A1378B8EEC77A27EEF8
:106A1000287A002B40F00682494BD3ED005AF4EE61
:106A2000CA5AF1EE10FA40F19087B7EE005A75EEAF
:106A3000654ADFED446A9FED445A444B36EEC77A0F
:106A400024EE855AD3ED006AE7EE055A65EEA65AA4
:106A5000F5EEC05AF1EE10FA40F2F784C9EEA56ADD
:106A6000B7EE007AF0EE475AE6EE665AF0EE656A47
:106A7000F4EEC76AF1EE10FA88BFF0EE476AF5EE61
:106A8000C06AF1EE10FAB8BFF0EE6A6A304B93EDCF
:106A9000007A67EE877AA7EEA68AFFF7B1B92D4B89
:106AA0002D4C19682D4ADFF8C48094F80031C9696B
:106AB0001288A8F80010A8F80220002B3EF434AF8A
:106AC00003F012FA002384F80031184B1B78072BCF
:106AD0007EF42AAFF8F77CF98246FEF727BF204BF9
:106AE000204A2B4493ED007AD2ED007A1E4B67EEDC
:106AF000277AF7EE006AF4EEE67AF1EE10FA93EDFB
:106B0000007A88BFF0EE667A67EE877A27EE888A89
:106B1000FFF727BAA8690020D44F0020B0BB00209F
:106B200048960020349300203C930020246E0020DF
:106B3000484F0020609600204C9600204CC000205A
:106B400054C0002000003443610BB63B48C0002015
:106B500044C0002094B90020582A0020A8470020F3
:106B6000B42B00203CC0002038C00020286E00203C
:106B7000D94BDFF8B8B31B789BF80020DD077FF511
:106B80001AAE002A3FF41DAED4ED583A94ED574AA0
:106B9000D24BD4ED627A93ED005A94ED617AD4ED44
:106BA000555A94ED546ACE49CE4BF4EEC43AF3EE06
:106BB000046AF1EE10FA77EEA64A00F15B8791EDD8
:106BC000026A26EE656AB0EE674AA6EE074AB4EEA0
:106BD000E44A34EE666AF1EE10FA48BFB0EE456A58
:106BE000012A83ED006A3FF4ECAD91ED066A26EED2
:106BF000656AB0EE674AA6EE074AB4EEE44A34EEA0
:106C0000666AF1EE10FA48BFB0EE456A022A83EDDB
:106C1000016A3FF4D6AD91ED0A6A26EE656AB0EEE0
:106C2000674AA6EE074AB4EEE44A34EE666AF1EE2D
:106C300010FA48BFB0EE456A032A83ED026A3FF4BA
:106C4000C0AD91ED0E6A26EE656AB0EE674AA6EE1B
:106C5000074AB4EEE44A34EE666AF1EE10FA48BF31
:106C6000B0EE456A042A83ED036A3FF4AAAD91EDC4
:106C7000126A26EE656AB0EE674AA6EE074AB4EEDF
:106C8000E44A34EE666AF1EE10FA48BFB0EE456AA7
:106C9000052A83ED046A3FF494AD91ED166A26EE61
:106CA000656AB0EE674AA6EE074AB4EEE44A74EEAF
:106CB000666AF1EE10FA48BFF0EE456A062AC3EDA7
:106CC000056A3FF47EADD1ED1A6A66EEE56AB0EE74
:106CD000674AA6EE874AB3EE046AB4EEE44A74EE5D
:106CE000466AF1EE10FA48BFF0EE456A072AC3ED96
:106CF000066A3FF466ADD1ED1E6A66EEE55AE5EE32
:106D0000877AF4EEE74A77EEC67AF1EE10FAC8BF5A
:106D1000F0EE457AC3ED077A53E5734BC7ED00AA51
:106D20001B689342BFF6ACA8704B1A88002384F806
:106D30006831002A41F015846D4A6E4B117818684D
:106D400081F00101F2F780FFFFF7A2B86A4EDFF889
:106D5000E08106F24C7506F5F767F6EC017A9BEDDB
:106D6000080ADBF87837F8EEE77A284627EE800A3B
:106D70009847A5F1E000DBF898369847A5F1700038
:106D8000DBF808379847D6F85806DBF8B83098474C
:106D90002435AF42A8EC010ADFD1FEF73FBF4E49D0
:106DA0000978C80703D45549098BA4F88C115449B4
:106DB0005448098890ED037A07EE901AF8EEE77AC6
:106DC000B4EEE77AF1EE10FA40F20C864E480088F5
:106DD00007EE900AF8EEE77AB4EEE77AF1EE10FAF1
:106DE000C0F2D08549484A49D0ED006A91ED006A69
:106DF0004848C4ED646ABCEEC75A76EE665A15EE92
:106E0000101AC4ED626AC4ED615A84ED656AA4F893
:106E10008C110121D0ED006A84F8981177EE677A21
:106E2000FFF730B93C4B93ED005AB5EEC05AF1EE86
:106E300010FA40F30A83394BD3ED006AF5EEC06ACD
:106E4000F1EE10FA40F3018336EEC77A66EE695A26
